S02B0000433A2F55736572732F4D53492F446F63756D656E74732F576F726B53706163652F6769742F41444DEB
S214400000A55AA55A0100000000000000001040005C
S21440100000F0422021144400E55C4500E75C4500C2
S214401010E95C4500EB5C4500ED5C450000000000E7
S214401020000000000000000000000000EF5C4500EB
S214401030235D450000000000255D4500275D450016
S21444010047573334342056302E322E352032303250
S214440110332E31312E362031323A30300A0D00003B
S20C4401803412AA5500000000E9
S214440200A55AA55A01000000000000000010440052
S2144402100000000000104400000000000000000041
S2144402200000000000000000000000000000000085
S2144402300000000000000000000000000000000075
S2144402400000000000000000000000000000000065
S2144402500000000000000000000000000000000055
S21444100000F0422021144400E55C4500E75C4500BE
S214441010E95C4500EB5C4500ED5C450000000000E3
S214441020000000000000000000000000EF5C4500E7
S214441030235D450000000000255D4500275D450012
S214441040295D4500295D4500295D4500295D45002B
S214441050295D4500295D4500295D4500295D45001B
S214441060295D4500295D4500295D4500295D45000B
S214441070295D4500295D4500295D4500295D4500FB
S214441400295D4500295D450000BF00BF00BF00BF01
S214441410FFF7FABF000000000000000000000000D4
S21444142072B64FF000004FF000014FF000024FF04C
S21444143000034FF000044FF000054FF000064FF055
S21444144000074F4801684FF0807201EA0201002904
S2144414501CD14C4801684FF0807241EA0201016099
S214441460494801684FF0010241EA020101604748D9
S21444147045F6F02101604AF20F5101604048016888
S2144414804FF0807201EA02010029F7D040484149F2
S2144414900160414801684FF00000814200D003E0FB
S2144414A03E4880F3088803E03D4880F3088822E0FD
S2144414B03C484CF2205101604DF6281101603A48F0
S2144414C03A4901600AE03A484CF2205101604DF630
S2144414D028110160374835490160FFE7364800283F
S2144414E009D03649364A521A013A04DD0020002310
S2144414F009C1083AFCDA3348002810D03249086853
S2144415004FF0010240EA020008603049304A521A5D
S214441510013A04DD0020002309C1083AFCDA2D48CC
S214441520002810D02C4908684FF0010240EA020017
S21444153008602A492A4A521A013A04DD0020002348
S21444154009C1083AFCDA274800684FF05A31884205
S214441550F9D0114801684FF00000814200D001E004
S21444156014F0E4FB14F00EFC62B614F009FC00F030
S2144415703BF800BFFEE700BFAFF30080AFF3008048
S21444158010C32D4030C32D4004C32D4000C02D4011
S21444159008ED00E0001043200400264000F04220FE
S2144415A0000043201000274000002740400000FF72
S2144415B010C0464000C046400100000000004020E5
S2144415C0004044200100000094EF00E000000020AA
S2144415D0000001200100000090EF00E00000000041
S2144415E000800000F02440202DE9F04F87B05B4C8B
S2144415F005F0BAF95A4816F0E7F85A494E2000253D
S21444160026F092FA58481DF06FFA58481DF090FAA2
S21444161005F01DF94CF24453E05803F079FE05F00A
S21444162059FB03F09DFF03F079FF03F0F7FE5049A2
S214441630002020F0D5FB4F49002020F0E7FB002196
S214441640084620F08DFC002144F62062084620F02F
S21444165043FC2846013505F0B7FC062DF9D105F0C4
S214441660F3F84CF23853444D4FF47A7054F80380F0
S214441670E75805F1040BE25854F803900592E258F3
S2144416800292E2580392E2580492E25854F803A0B5
S214441690E6582C46019205F09EF800F0B9F8374813
S2144416A005F0CAF900F0C4F82A6806F57A739A4237
S2144416B002D32E680BF0E7FE22680AF1C8039A426A
S2144416C003D3D4F800A00BF0D7FE019B2268643302
S2144416D09A4203D3236801930BF0BBFE049B226813
S2144416E032339A4201D323680493039B226814330B
S2144416F09A4203D32368039307F0F2F8029B2268C6
S2144417000A339A4203D3236802930BF066FE226898
S21444171009F105039A4203D3D4F800900BF0DBFD9D
S214441720059B226802339A4203D32368059300F04C
S21444173080F822687B1C9A4200D32768DBF8002096
S21444174008F101039A4203D3DBF800800BF070FEE5
S21444175000F064F80DF072FDA6E700BFEC4B4120A4
S21444176028964600E80340206CA346009C9E46000C
S2144417707417402068174020241142208C8C460061
S214441780024B586800F00300704700BF0000264034
S214441790024600F03F00931010B583EA5203540803
S2144417A0534084EA121483EA121384EAD2049B0157
S2144417B084EA521403F0400314F0010F43EA000392
S2144417C00CBF80240024234319B99A4218BFFF2033
S2144417D010BD01290CBF1846FF20F9E73C2A0CD05F
S2144417E07D2A0AD0FE2A08D0BF2A06D092B20144E7
S2144417F0814204D1D043C0B270470022F7E710F8C4
S214441800013B1A4492B2FF2A84BFFF3A92B2EFE7F2
S2144418100149002026F00CBB90A74600002026F085
S2144418200BBB00221146104626F0FEBA704700BF96
S214441830704703F0CBBC704710B50C4C002004F046
S2144418402DFF2080012004F029FF094B22881880B0
S214441850084B1A8003F019F803F03AF803F05CF8E2
S21444186003F07EF8BDE8104003F09EB85A184020B6
S21444187058184020041840207047704770477047F7
S2144418802DE9F04FB84CD9B0D4E904230DF580784F
S214441890CDE92A23DDE92A01D4E950230DF05EFF81
S2144418A0A1A3D3E900230EF00FF906460F46A0A3E2
S2144418B0D3E90023D4E952010EF006F902460B465A
S2144418C0304639460DF04AFF9BA3D3E900230EF079
S2144418D025FA95A3D3E90023D4E94856D4E94AAB7C
S2144418E0CDE94C23CDE9005695A3D3E90023D4E9AA
S2144418F04C45CDE91001CDE95223002000220023B7
S2144419009A49CDE9024546AC0325CDE94601CDE9E1
S2144419104823CDE94A23CDE94E01CDE95023CDE90C
S2144419205423CDE95601CDE90A01CDE90623A14663
S214441930504659460834D9E906230EF0C5F80646FB
S2144419400F46D9E90023DDE900010EF0BDF8024652
S2144419500B46304639460DF001FF06460F46D4E99D
S2144419600A23DDE902010EF0AFF802460B46304684
S21444197039460DF0F3FE013DE8E80201D7D17A4C32
S214441980236D0293636D0493DDE94223DDE940ABA6
S214441990CDE90023DDE94423CDE90823DDE9080148
S2144419A0002200230EF090F8002280468946002349
S2144419B0DDE900010EF088F852465B460DF0CEFE97
S2144419C042464B460DF0CAFE02460B460298049920
S2144419D00DF0C2FE002206460F46002350465946E6
S2144419E00EF072F8DDE900230DF0B8FE42464B4691
S2144419F00DF0B4FE02460B46DDE910010DF0ACFED8
S214441A0002460B46CDE90C234FA3D3E900230EF040
S214441A105BF880468946304639464DA3D3E90023D1
S214441A200EF052F802460B46404649460DF096FEE6
S214441A3052465B460DF092FE00220023C4E948015C
S214441A40304639460EF040F88046894642A3D3E9EC
S214441A500023DDE90C010EF037F802460B464046FB
S214441A6049460DF07BFEDDE900230DF077FE024685
S214441A700B46CDE91201C4E94A233046394638A319
S214441A80D3E900230EF020F806460F460022002332
S214441A90DDE90C010EF018F802460B46304639468E
S214441AA00DF05CFEDDE908230DF058FED4E91A2358
S214441AB0D4E902ABC4E94C01CDE9182350460022D0
S214441AC02B4B59460EF086FA002840F00182D4E9A2
S214441AD01267D4E90C453046394622462B460EF06A
S214441AE06FFA08B926462F4600224FF08043DDE9B8
S214441AF018010EF051FA0022002800F0EC81002371
S214441B00304639460DF0E0FF02460B46CDE9082341
S214441B10154BD3E9A44522462B460DF01DFE06463A
S214441B200F4627E0AFF30080FCA9F1D24D62603F38
S214441B30D9D6F61FCE4EE43F2DBA9CBB926FE43FF7
S214441B4049DC63E9431794BF7B14AE47E17A843F8C
S214441B50E71DA7E8482ED33F386744696FF0EF3F48
S214441B603CBD5296218EB5BFC04740200000F03F92
S214441B7000004940ACA3D3E900230EF035FA002810
S214441B8000F0AB8120462946A7A3D3E900230DF0F5
S214441B90E5FDCDE90801DDE90834B74E0022C6E983
S214441BA0A434D6E95445B54B204629460EF01CFAD3
S214441BB0002840F0A4810022B14B204629460EF06E
S214441BC0F5F9002840F09E8196F8EA320BB1C6E952
S214441BD05645A94B20462946D3E9566732463B46E6
S214441BE00DF0BAFD04460D4691A3D3E900230EF04A
S214441BF0FBF9002840F08981204629468EA3D3E984
S214441C0000230EF0D3F9002840F0838122462B4669
S214441C10304639460DF0A2FD02460B46CDE92E234A
S214441C2087A3D3E900230DF04FFF06460F4612F074
S214441C3043FF04460D463046394612F0AFFE914BFC
S214441C4006460F4620462946D3E900230DF03CFFBE
S214441C5004460D46304639467BA3D3E900230DF0AF
S214441C6033FF002200230DF02FFF02460B4620468A
S214441C7029460DF073FD76A3D3E900230DF024FF27
S214441C8075A3D3E900230DF01FFF00227E4B0446C4
S214441C900D460EF0A9F9002840F03F8100220023AB
S214441CA0204629460EF082F908B100240025724BDE
S214441CB093F8EB220AB1C3E95845D3E9586720465E
S214441CC0294632463B460DF047FD04460D4664A37E
S214441CD0D3E900230EF088F9002840F021812046FD
S214441CE0294661A3D3E900230EF060F9002840F0AA
S214441CF01B8122462B46304639460DF02FFD0246C0
S214441D000B46CDE93A235AA3D3E900230DF0DCFE73
S214441D10594BCDE93001D3E90E45D3E95A12204652
S214441D200023CDE90012002229460EF035F900289A
S214441D3000F0FE8000220023029804990EF040F939
S214441D4050B10022514B504659460EF043F918B153
S214441D5000230024CDE90034474CD4E90023CDE9E0
S214441D600C2394F8E832002B40F0318140F2011302
S214441D70A4F8E832DFF800810022454DDDE9063458
S214441D80DDE90001C8E9C434424B0EF005F9031EF0
S214441D904FF00002594618BF0123504616933E4B57
S214441DA00EF00EF9041E4FF000024FF0804318BFA9
S214441DB00124DDE908010EF003F9169B00280CBF48
S214441DC02046601C002418440DF014FE0022334BB9
S214441DD00DF0C4FCD8E9C6230DF0C0FC0022304BFD
S214441DE00EF0F8F80022D8E9B267002800F0108117
S214441DF00023304639460EF0CFF818B1DDE9062305
S214441E00C8E9B8231C4EDDE90A23C6E9B445D6E939
S214441E10B845C6E9B223204600221E4B29460EF09A
S214441E20C5F800284BD03DE0FCA9F1D24D62703F86
S214441E30FCA9F1D24D62603FFCA9F1D24D6260BF6D
S214441E40399D52A246DF913F407EFCF8F14B7B40E1
S214441E50E3A59BC420B0D23F578C22C76075B53FDC
S214441E60FCA9F1D24D62903F7B14AE47E17AC4BFE1
S214441E709A9999999999E93FC04740200000204093
S214441E80000020C0A880460000004E400000594094
S214441E9000408F4000000840000034400000F03FFF
S214441EA00000144020462946DDE93023C6E9B6231F
S214441EB073A3D3E900230DF051FCC6E9B801DDE96C
S214441EC00A34C6E9C4340023814CCDE90E3419E102
S214441ED00026002708E67F4B12E66BA3D3E90023CF
S214441EE0304639460EF062F800283FF454AE204699
S214441EF0294667A3D3E900230DF02EFC49E60024C7
S214441F00754D61E60024754D5EE663A5D5E900454A
S214441F107CE663A5D5E9004578E60024704DC6E620
S214441F2061A5D5E90045E4E661A5D5E90045E0E6C6
S214441F30DDE900010EF078F803283FF60DAFDFE840
S214441F4000F002191D1900220023029804990EF08D
S214441F5037F800283FF400AF00225E4B204629465F
S214441F600EF01AF878BB00225E4B204629460EF047
S214441F7013F840BB00224FF080431AE000220023AF
S214441F80029804990EF01CF800283FF4E5AE0022AF
S214441F90554B504659460EF01DF800283FF4DCAE2B
S214441FA000224C4B204629460DF0F6FF40B900224D
S214441FB04C4B204629460DF0EFFF00283FF4CCAEAC
S214441FC0CDE90045C8E600234FF08044C2E694F8C5
S214441FD0E932012B0FD10022444BDDE90C010DF010
S214441FE0E5FF18B1022384F8E932C3E6DDE90623A7
S214441FF0C4E9C623BEE630A3D3E90023DDE90C01D9
S2144420000DF0F2FF08B10123EDE7DDE90A23EFE71F
S214442010304B304639460DF0BFFF002801F03F8173
S214442020D8E9B623D8E910010DF0D4FF002861D0D2
S214442030D8E9B44522A3D3E90023204629460DF027
S21444204043FD02460B46204629460DF085FB0446D2
S2144420500D461DA3D3E900230DF0A8FF28B9C8E90F
S214442060B445234BD3E9B4342FE7DDE90634C8E955
S214442070B434C8E9B234C8E9B634C8E9B834F0E789
S2144420807B14AE47E17A743FFCA9F1D24D6280BF1F
S214442090FCA9F1D24D62803FFCA9F1D24D62603F6B
S2144420A0FCA9F1D24D6260BFFCA9F1D24D62903FCB
S2144420B07B14AE47E17AC4BF0000000000C0624013
S2144420C09A9999999999A93F7B14AE47E17A843FA6
S2144420D000408F400000F03F00002040000020C039
S2144420E000004E400000084000005940000049C02F
S2144420F0C0474020DDE90A23C8E9B445C8E9C423FB
S214442100CDE90E45049C029824F000410024B6A371
S214442110D3E900230DF04AFF002841F0C480C24DA5
S214442120DFF80C83B2A3D3E90023DDE910010DF0F8
S214442130CBFC02460B46002000210DF00DFB224648
S2144421402B460DF0C1FC02460B46CDE92C2300225B
S214442150B64B0DF0B9FCA8A3D3E90023CDE9320170
S214442160D8E95C010DF0B0FC06460F46A4A3D3E9BB
S2144421700023DDE92C010DF0A7FC02460B46304651
S21444218039460DF0EBFA06460F46D8E95E23DDE9FC
S21444219032010DF0E1FA002200230DF095FC0246D0
S2144421A00B46304639460DF0D9FA02460B46CDE981
S2144421B01A2395A3D3E900230DF016FF002841F017
S2144421C0758093A3D3E90023DDE91A010DF0EEFEF2
S2144421D0002841F07080DDE91A23CDE91423DDE9B7
S2144421E01423204629460DF06FFC914B04460D46B9
S2144421F0D3E9A66732463B460DF0AEFA00224FF0CE
S2144422008043804689460DF0EFFE0022002801F008
S21444221057804FF08043304639460DF09FFA0446C7
S2144422200D46834B0022C3E9A645DDE90001814BF8
S2144422300DF0B2FE002801F0558000207A4922466F
S2144422402B460DF041FC02460B46CDE90A230022FC
S21444225000230DF0BFFE18B900230024CDE90A344C
S21444226073490022744BD1E960010DF02DFC002225
S214442270724B0DF029FC002204460D466A4BDDE9FC
S21444228000010DF089FE169B00284FF00002204600
S214442290294608BF1E466A4B18BF4FF0FF360DF05E
S2144422A0A3FE002841F0228000220023204629462F
S2144422B00DF07CFE08B10024002530460DF09AFB54
S2144422C022462B460DF000FC594B80468946D3E9FE
S2144422D0A84522462B460DF03FFA0022554B0646AB
S2144422E00F460DF081FE0022002801F00380514B7A
S2144422F0204629460DF032FA804689464C4B002249
S21444230040464946C3E9A8894D4B0DF06DFE00286A
S21444231041F0008000220023404649460DF046FE28
S21444232018B14FF000084FF0000900224FF08043E8
S214442330DDE918010DF030FE002800F0F187002298
S214442340404B029804990DF0BFFB06460F4632A355
S214442350D3E900230DF048FE002840F0E987002228
S2144423600023304639460DF021FE08B100260027EA
S21444237000222D4BDFF8B8A0DDE908010DF02AFE57
S21444238048B927A3D3E90023DAE932010DF022FE47
S214442390002800F0E78700222B4BDAE91045204658
S2144423A029460DF017FE002800F0DC8712A3D3E977
S2144423B00023DDE910010DF00DFE002800F0D28761
S2144423C00022224B029804990DF004FE002800F0E7
S2144423D0C98700221C4B304639460DF0F1FD0028D3
S2144423E000F0C08734E000BF9A9999999999B93F0B
S2144423F000000000007097409A9999999999C93FAE
S214442400EC51B81E85EBB13F00000000008AAB409B
S214442410000000000088A3C0000000000088A3401D
S2144424207B14AE47E17A843F0000F03F00407F4093
S214442430C0474020000008400000B03F000054C0A1
S21444244000408F4000005940000024400000F83F00
S214442450DAE9B023DAE90801CDE90623ACA3D3E9E7
S21444246000230DF031FBDDE912230DF077F9AAA322
S214442470D3E900230DF028FB02460B4620462946A6
S2144424800DF04CFC04460D460022C14BCAE94E45AD
S2144424900DF0AAFD002800F05B870022BD4B2046C5
S2144424A029460DF083FD002800F052872046294631
S2144424B0DDE906230DF050F921F0004CDDE9062352
S2144424C061460DF02BFC96A3D3E900230DF06EFD78
S2144424D0002800F03D8794A3D3E90023DDE90601F4
S2144424E00DF0F2FA92A3D3E90023CDE9120129466E
S2144424F020460DF0E9FA02460B46DDE912010DF0DE
S2144425002DF902460B46CAE9B023DDE906230DF051
S21444251023F921F0004500229F4B29460DF046FD45
S214442520002800F00A8701238AF8EE329B4B0020ED
S2144425304FF08041C3E9E001984CD4E9B023C4E9A4
S214442540BC67C4E9DE23C4E9DA677BA3D3E9002386
S214442550DDE90A01C4E9CC890DF0B6FA78A3D3E9DB
S21444256000230DF0DBFB00220023C4E9CE01DDE9A5
S21444257000010DF011FD0646002840F0FA860022C0
S2144425804FF08043DDE900010DF006FD58B9844B59
S2144425900022DDE900010DF0FFFC169B00280CBF6D
S2144425A01E464FF0FF3600227E4BDDE908010DF053
S2144425B08BFA65A3D3E900230DF0B0FB60A3D3E9FF
S2144425C000230DF081FA0022774B0DF07DFA60A3CC
S2144425D0D3E900230DF0A2FB04460D4630460DF029
S2144425E009FA02460B46204629460DF06DFA024685
S2144425F00B46CDE90A23694BD3E9AA4522462B4626
S2144426000DF0AAF806460F4653A3D3E900230DF06F
S214442610EBFC002800F0B086204629464EA3D3E9BA
S21444262000230DF09BF8CDE90A015C4CDDE90A2352
S214442630DDE90A01C4E9AA23D4E962230DF08EF841
S21444264047A3D3E900230DF03FFA06460F4646A3B8
S214442650D3E90023D4E964010DF036FA02460B466A
S214442660304639460DF07AF841A3D3E900230DF0FD
S21444267055FB02460B46CDE90623D4E966230DF006
S2144426806BF80022474B0DF01FFAD4E968230DF08F
S21444269063F802460B46CDE91C23D4E96A230DF0C1
S2144426A05BF800223F4B0DF00FFAD4E96C230DF093
S2144426B053F802460B46CDE91E23D4E96E230DF0AB
S2144426C04BF80022374B0DF0FFF9D4E970230DF098
S2144426D043F829A3D3E90023CDE93401DDE9060113
S2144426E00DF0F2F906460F4625A3D3E90023DDE9AB
S2144426F01C010DF0E9F932463B460DF02FF88046B2
S214442700894621A3D3E9002350E000BFAFF30080FD
S2144427107B14AE47E17A843F8462BF15623E973F9E
S2144427209A9999999999C93F5C8FC2F5285CEF3F6D
S2144427307B14AE47E17A943F0E9F7422C154D13F36
S2144427405C8FC2F528DC2740000000000020AC4027
S214442750B46155D0CC38FB3F9A9999999999D93F09
S214442760FCA9F1D24D62603FB428207983A6BA3FD3
S21444277054434F56A8ACBB3F9A999999999963404C
S2144427809A99999999996A40CDCCCCCCCCCC354081
S21444279000407F4000409F4000001440C047402017
S2144427A00000F03F00408F4000004E40DDE91E012F
S2144427B00DF08AF902460B46404649460CF0CEFFD9
S2144427C0DDE934230CF0CAFFBFA3D3E900230DF0A0
S2144427D07BF9D4E97223CDE92001104619460CF062
S2144427E0BDFFDDE920230CF0B9FFD4E938230CF013
S2144427F0B5FFB7A3D3E900230DF066F980468946B2
S214442800B5A3D3E90023D4E974010DF05DF902467B
S2144428100B46404649460CF0A1FF80468946B0A385
S214442820D3E90023D4E93C010DF04EF902460B46A9
S214442830404649460CF090FFABA3D3E900230DF085
S2144428406DFA02460B46CDE92223D4E976230CF0F2
S21444285085FFA7A3D3E900230DF036F980468946C1
S214442860A5A3D3E90023D4E978010DF02DF9024657
S2144428700B46404649460CF071FFA1A3D3E900231A
S2144428800DF04CFADDE90C23CDE93601DDE906010D
S2144428900CF062FF0022B44B04460D460DF0A4FB38
S2144428A0002840F07C852046294697A3D3E9002398
S2144428B00DF07CFB002840F085850022AB4B20467B
S2144428C029460DF091FB002800F06D850022A74BA9
S2144428D0204629460CF040FF82468B46A44CDDE950
S2144428E00601D4E97A230CF037FF0022A14B0DF001
S2144428F0EBF8D4E97C230CF02FFF02460B46CDE9D7
S2144429002423D4E97E230CF027FF0022994B0DF0B4
S214442910DBF8D4E980230CF01FFF02460B46CDE9D2
S2144429202623D4E982230CF017FF0022914B0DF0A6
S214442930CBF8D4E984230CF00FFF75A3D3E9002326
S214442940CDE93801DDE924010DF0BEF832463B46B8
S2144429500CF004FF06460F466FA3D3E90023DDE9D7
S21444296026010DF0B1F802460B46304639460CF0C7
S214442970F5FEDDE938230CF0F1FE53A3D3E900233A
S2144429800DF0A2F8D4E9AC230CF0E6FE02460B4662
S214442990CDE93C23D4E986230CF0E0FE54A3D3E9E6
S2144429A000230DF091F806460F465DA3D3E90023B5
S2144429B0D4E988010DF088F802460B46304639467D
S2144429C00CF0CCFE58A3D3E900230DF0A7F9D4E9C4
S2144429D08A23CDE91201104619460CF0BFFEDDE904
S2144429E012230CF0BBFED4E940230CF0B7FE50A3F0
S2144429F0D3E900230DF068F806460F464EA3D3E904
S214442A000023D4E98C010DF05FF802460B463046AD
S214442A1039460CF0A3FE06460F4649A3D3E90023E5
S214442A20D4E944010DF050F802460B463046394688
S214442A300CF092FE44A3D3E900230DF06FF9002274
S214442A404D4BCDE92801029804990DF0AFFA0028C1
S214442A5040F0C2840022484B029804990CF07CFE55
S214442A603BA3D3E900230DF02FF80022434B044642
S214442A700D460DF0AFFA08B10024404D36A3D3E915
S214442A800023DDE928010DF01FF800223C4B884660
S214442A9006460DF08BFA8146002840F0A1840022B9
S214442AA0384B304641460DF09FFA002840F09E844D
S214442AB0B14608F100485046594629A3D3E90023B5
S214442AC00DF002F860E000BFE3F36EFB79D0E33E1E
S214442AD0277845D92444D93FFB50D7647BD71C403C
S214442AE03043BB3975F104406D0D4BFEC9AF1840F9
S214442AF0FCA9F1D24D62603FEBF33CDE4AA2813F33
S214442B00E9C8B5C771D3893F0000000000409FC0A4
S214442B109A99999999996A40CDCCCCCCCCCC3540ED
S214442B205ED817C2038C9E3F6F216A9B4B52A13FCF
S214442B302ED7D19C0A49373F7119ABB745FF1F4082
S214442B40ECBC164D8E930F401988C921F3361040BD
S214442B509A9999999999C93FCDCCCCCCCCCCEC3F99
S214442B603B08AA2A23DCA63F00409F400000494079
S214442B70C047402000408F40000014400000F03F13
S214442B8000003EC000003E40DDE936230CF0E6FD82
S214442B9006460F4622462B46484641460CF094FFCE
S214442BA032463B460CF0DAFD02460B46CDE90C2392
S214442BB00022B74B0DF018FA002840F01B84002280
S214442BC0B44BDDE90C010DF0F1F918B10023B14C1A
S214442BD0CDE90C3400224FF08043DDE918010DF0B6
S214442BE0DBF90446002800F00984AB4C0022AB4BCA
S214442BF0D4E920010DF0D0F9002800F02A84002200
S214442C00A64BD4E922010DF0C7F9002800F0218430
S214442C1002980026049994A3D3E900230DF07EF885
S214442C2000229F4B0DF0E0F9002800F01384994FE2
S214442C30994C0022994BD4E91E010DF0ADF90028B9
S214442C4040F00F8432463B46C4E9DC67C4E9C223FD
S214442C50DDE91A01DDE914230CF07EFDDDE90E23DF
S214442C60CDE93E01C4E9CA23DDE90023DDE92A01B2
S214442C70C4E9D423DDE93023C4E9C023DDE92E23A7
S214442C80C4E9C823D4E98E230CF068FD78A3D3E9BD
S214442C9000230CF019FF06460F4677A3D3E900231A
S214442CA0D4E990010CF010FF02460B4630463946F4
S214442CB00CF054FD72A3D3E900230DF02FF8D4E9A9
S214442CC09223CDE91801D4E906010CF047FD68A328
S214442CD0D3E900230CF0F8FE06460F4666A3D3E974
S214442CE00023D4E994010CF0EFFE02460B4630462E
S214442CF039460CF033FD62A3D3E900230DF00EF8F9
S214442D00D4E99623CDE90401D4E908010CF026FD64
S214442D1057A3D3E900230CF0D7FE06460F4656A326
S214442D20D3E90023D4E998010CF0CEFE02460B46C4
S214442D30304639460CF012FD51A3D3E900230CF07B
S214442D40EDFFCDE90E01DDE90423104619460CF0EB
S214442D50BBFE04460D46DDE90E23104619460CF02C
S214442D60B3FE02460B46204629460CF0F7FC11F00B
S214442D70E9FE0022002304460D460DF00DF948B93D
S214442D8022462B46DDE918010CF0C8FF11F07CFC06
S214442D9004460D46404E20462946424FD6E9542323
S214442DA0CDE9142338A3D3E900230CF08DFE024664
S214442DB00B46DDE914010CF0CFFCD6E90A34CDE924
S214442DC01A01CDE91634DDE91601D6E99C230CF048
S214442DD0C5FC27A3D3E900230CF076FE04460D4633
S214442DE025A3D3E90023D6E99E010CF06DFE0246E6
S214442DF00B46204629460CF0B1FC21A3D3E9002318
S214442E000CF08CFFD6E91445CDE92A0122462B4620
S214442E10DDE908010CF0A0FC0022234BCDE930018B
S214442E20204629460CF050FE02460B4600201F4919
S214442E300CF092FC00221B4B0C4605460DF0B6F8EF
S214442E40002808BF28460AA3D3E9002316BF00205B
S214442E50214639460CF038FE96F8EC3282468B46CC
S214442E6026E000BFAFF30080CDCCCCCCCCCC0C401D
S214442E70FCA9F1D24D62603FFEF2469F2892AF3FD6
S214442E801F94D22C39CFB03FF8C1631ADCA54C400E
S214442E9000005440000054C0C04740200000F03FAB
S214442EA00000E03F0080614000001A400000794086
S214442EB0D6E916010BB1C6E9A001D6E9A089424677
S214442EC04B460CF049FC002206460F46A04B2846CB
S214442ED021460DF06BF8002840F0C78204F1004408
S214442EE032463B46504659460DF060F8002840F0BE
S214442EF0BF822846214694A3D3E900230CF0E4FD80
S214442F0002460B46CDE90201304639460DF04EF8EE
S214442F1008B1DDE9026732463B46404649460CF076
S214442F201DFC8C4B0A46CDE902010146C3E9BE129C
S214442F30C3E9D81293F8ED22D3E918010AB1C3E9DC
S214442F40A201D3E9A28942464B460CF005FC06464C
S214442F500F4602460B46504659460DF027F878B9B8
S214442F602846214678A3D3E900230CF0ADFD32462B
S214442F703B4682468B460DF037F808B9B246BB4608
S214442F8052465B46404649460CF0E8FB714C0246C6
S214442F900B46C4E9D02300220023CDE90801C4E946
S214442FA0D623D4E91C0100226B4B0CF0F5FF68B91C
S214442FB00022694BD4E91E010CF0EEFF30B9002222
S214442FC0654BD4E928010CF0E7FF18B10022624BA8
S214442FD0C4E9D6235F4C00225F4BD4E92A010CF0A7
S214442FE0DBFFA0B900225C4BD4E92C010CF0D4FFE3
S214442FF068B90022584BD4E92E010CF0CDFF30B905
S2144430000022554BD4E930010CF0C6FFA8B1514E0E
S21444301000220023D6E91A45204629460CF0BCFF78
S21444302038B900224FF08043204629460CF0B4FFBE
S21444303018B10023484CC6E9D634464C0022464BC9
S214443040D4E920010CF0A8FF40B90022424BD4E951
S21444305022010CF0A1FF002800F00D823D4B002118
S2144430603D4AC3E9D612DFF8ECA00022DAE99A67B3
S214443070DDE91034DAE90489CAE952343046374B7C
S2144430803946CAE950890CF01FFD04460D46002215
S214443090334BDDE91A010CF017FD02460B46204679
S2144430A029460CF05BFB02460B46DDE92A010CF090
S2144430B053FB25A3D3E900230CF006FDDDE91423D6
S2144430C00CF04CFBDDE92E34CAE95401CAE9563407
S2144430D0DDE93A34DDE92C01CAE95834DDE9003447
S2144430E0CAE95A34DAE9AE230CF036FB16A3D3E920
S2144430F000230CF0E9FCDAE95C230CF02FFB0022F9
S214443100DDE93234CAE95C01CAE95E34DAE96001D1
S214443110144B0CF0D9FCDDE930230CF01FFBDDE941
S2144431200A34CAE96001CAE96234DDE90634CAE908
S2144431306434CAE96634DDE91C34CAE96834CAE949
S2144431406A34DDE91E340FE0FCA9F1D24D62603FDB
S21444315000806140C04740200000F03F000014401B
S214443160000059400000EE3FCAE96C34CAE96E34A8
S214443170DDE93434CAE97034DDE92034CAE972340E
S214443180DAE93A23CAE93823DDE92034CAE93A348D
S214443190DDE92234CAE97434DAE93E23CAE93C2339
S2144431A0DDE92234CAE93E34CAE97634DDE9363408
S2144431B0CAE97834DDE90C34CAE9AC34DDE90634CE
S2144431C0CAE97A34DDE92434CAE97C34CAE97E346F
S2144431D0DDE92634CAE98034CAE98234DDE9383484
S2144431E0DDE91A01CAE98434DDE93C34CAE98E894A
S2144431F0CAE98634DDE91234CAE98834CAE98A342D
S214443200DAE94223CAE94023DDE91234CAE9423402
S214443210DDE92834CAE98C34DAE94623CAE944238A
S214443220DDE92834CAE94634DDE93E34CAE9AE3439
S214443230DDE91834CAE99034DAE90623CAE9922368
S214443240DDE90434CAE99434DAE90823CAE9962362
S214443250DDE90E34CAE9983491A3D3E900230CF08F
S21444326033FC3B4632460CF079FADDE91634CAE9BB
S2144432709A01CAE99C34DDE92A34CAE99E34DDE978
S2144432800234CAE9A0340023AAF8EA32AAF8EC3297
S214443290DDE90834CAE9A23459B0BDE8F08F00230A
S2144432A00024FEF712BE0025FEF73ABF7EA3D3E9FC
S2144432B00023FEF792BF7EA3D3E90023FEF78DBF1B
S2144432C04FF04043404649460CF070FE00283EF41A
S2144432D0A8AF00224FF08043304639460CF03CFA03
S2144432E0FEF79DBF00200021FEF7A9BF00247A4DBB
S2144432F0FEF7E3BF794B304639460CF057FE0028BC
S2144433003EF4FCAF0022764B204629460CF024FAC5
S214443310FEF7F2BF4FF00008DFF8BC91FFF705B8A0
S21444332042464B46DDE90E010CF018FAFFF70DB89D
S21444333061A7D7E90067FFF71BB89AF8EE32002B6F
S2144433407FF4F4A80023674CCAE9E034FFF7F4B8E6
S2144433500022654B002183F8EE22624AC3E9E0125C
S214443360FFF7EAB80022604B83F8EE22DDE9061246
S214443370F4E70026FFF717B951A3D3E900233046F4
S21444338039460CF013FE00283FF44FA92046294640
S2144433904DA3D3E900230CF0DFF9FFF744B900242A
S2144433A0524DFFF793BA0022514B204629460CF063
S2144433B011FE58B900224F4B204629460CF0CEF950
S2144433C0FFF78ABA42A5D5E90045F3E74FF0000A6D
S2144433D04FF0000BFFF782BA00240025FFF74EBBE0
S2144433E04FF00009DFF81881FFF765BBDFF814815A
S2144433F0FFF761BB0023404CFFF7EABB00220023E3
S214443400DDE900010CF0C8FD054630BB00224FF054
S2144434108043DDE900010CF0BFFD00BB314B0022C8
S214443420DDE900010CF0B8FD0028169B18BF4FF0EC
S214443430FF3318460CF0DEFADDE90C230CF044FBAF
S2144434400022002306460F460CF0B0FD00283FF449
S214443450EFAB00260027FFF7EBBB2046EAE72846FB
S214443460E8E700220023FFF7EFBB0025234C37E5AF
S21444347056465F464FE500221A4BD4E924010CF029
S2144434808BFD00283FF4EFAD0022164BD4E926010D
S2144434900CF082FD00287FF4E1ADE4E5AFF3008054
S2144434A0FCA9F1D24D62603F00000000008AAB40A8
S2144434B0000000000088A3C0000000000088A3406D
S2144434C09A9999999999E9BF9A9999999999E93FB5
S2144434D00000000000409FC000408F40000008C02D
S2144434E0000008400000F03FC047402000409F4096
S2144434F0000049C00000494000005440008061C0BC
S21444350000003E4000003EC0094B40F2011206A1B6
S214443510D1E90001A3F8EA22A3F8EC22C3E9B001FA
S214443520704700BFAFF30080000000000070974073
S214443530C0474020F8B56A4B00266A4C00271868F6
S2144435400CF06AFA684B1D68C4E9000128460CF082
S21444355041FA664BC4E91A0118680CF05DFA644BEC
S214443560C4E9140118680CF057FA624BC4E9040124
S21444357018680CF051FA604BC4E9060118680CF060
S2144435804BFA5E4BC4E9080118680CF045FA5C4BEC
S214443590C4E90A0118680CF03FFA5A4BC4E93201F0
S2144435A018680CF039FA584BC4E9360118680CF020
S2144435B033FA564BC4E9020118680CF02DFA544B02
S2144435C0C4E91001C4E9346718780CF003FA514B87
S2144435D0C4E92A0118780CF0FDF94F4BC4E92C01D4
S2144435E018780CF0F7F94D4BC4E92E0118780CF016
S2144435F0F1F94B4BC4E9300118780CF0EBF9494B20
S214443600C4E91C0118780CF0E5F9474BC4E91E01DF
S21444361018780CF0DFF9454BC4E9200118780CF013
S214443620D9F9434BC4E9220118780CF0D3F9414B3D
S214443630C4E9240118780CF0CDF93F4BC4E92601BF
S21444364018780CF0C7F9C4E9280125BB3B4B186829
S2144436500CF0E2F93A4BC4E9020118680CF0BAF9E6
S2144436600022384BC4E91223374BC4E90C01C4E9A1
S214443670326718680CF0AEF9344BC4E90E0118688A
S2144436800CF0CAF9324BC4E9160118680CF0C4F9B8
S214443690C4E91801F8BD012D1CD12E4B18680CF056
S2144436A099F92D4BC4E90C01C4E9326718680CF04B
S2144436B091F92A4BC4E9120118680CF08BF9284B8F
S2144436C0C4E90E0118680CF0A7F9C4E91867C4E900
S2144436D01601DFE7023D012DDCD8C4E90C67D9E7C3
S2144436E06C1E4020C0474020541C4020741C402080
S2144436F01C1F40203C1F4020001F40200C1F402021
S2144437008C1F40204C1C4020A01F4020681E402098
S2144437108217402081174020801740207F17402082
S214443720521F4020511F4020241C4020231C402070
S214443730221C4020211C4020501F4020B41D402005
S214443740BC1D4020000044408C1D4020A81D402045
S214443750A41D4020881F4020541F4020701F402036
S214443760941F40202DE9F04F774C85B0774EDFF814
S21444377038A2DFF838B2D4E900010CF09DFC744B53
S21444378080461860D4E906010CF096FC3060D4E913
S21444379004010CF091FC6F4B1860D4E902010CF064
S2144437A08BFC6D4A6D4B074610601860D4E91401D3
S2144437B00CF082FCCBF80000CAF800008146D4E93D
S2144437C018010CF059FC664905460860D4E9220104
S2144437D00CF052FC63490880D4E924010CF04CFCFC
S2144437E061490870D4E91A010CF046FC5F49087038
S2144437F0D4E920010CF060FC5D490860D4E91E0160
S2144438000CF05AFC5B490860D4E91C010CF054FCEB
S2144438105949086038465949096803910CF066FFCF
S2144438204D4A4E4B029616461C460399CDF804A0C4
S21444383060B111601960524F484639460CF056FF45
S214443840B8B1019BCBF800701F6019E001F1004A43
S214443850384651460CF02CFF20B1C6F800A0C4F8F8
S21444386000A0E8E7514638460CF022FF0028E2D094
S214443870F5E7444F484639460CF01AFF0028E0D195
S214443880414B424F1B6853B9414B25F0020519681A
S214443890012D08D140460CF065FC386004E0012B4D
S2144438A043D13C4BF1E739603B4D386829460CF030
S2144438B013FF00B13D603B680022DFF8F480374FC9
S2144438C0374DC8F800303B60364BD5E920010CF044
S2144438D063FB10B10023C8F800300022314BD5E911
S2144438E022010CF059FB08B100233B6000222D4B0B
S2144438F0D5E924010CF050FB08B1002333600022C4
S214443900284BD5E926010CF047FB08B10023236079
S2144439100022244BD5E928010CF03EFB10B10023CD
S2144439203360236005B0BDE8F08F022B03D1194BFA
S21444393041461868AFE7032BB6D10023029A1360BA
S214443940144B1B683B60AFE7B04A4020581B4020EE
S214443950901F4020B4174020B81940201419402026
S214443960581C40207C1740207A174020A817402037
S214443970A4174020A01740209C174020AC17402096
S21444398000004843000048C3541C4020981F402071
S214443990B41D4020A01F402000401C45081940206C
S2144439A0C04740200000F03F8C184020A418402018
S2144439B0AC19402000000000F8B5174B174C1E68A1
S2144439C0174D66B1012E19D00021002001F0DEFC0F
S2144439D00021012001F0DAFC00232B700CE026784D
S2144439E0002EF1D10021304601F0D0FC0D490120D3
S2144439F001F0CCFC01232E702370F8BD2F78002FE5
S214443A00E2D10849384601F0C1FC0021304601F0B5
S214443A10BDFC2E702770F0E7541C4020E817402069
S214443A20E91740200000C84208B5114B18680BF04F
S214443A30F3FF0DA3D3E900230CF0C2FA90B90D4B63
S214443A404FF07E5118680CF047FE003818BF01202E
S214443A50094B1860094B1B685A1E53425341084A87
S214443A60136008BD0120F3E7666666666666E6BFD1
S214443A701C1F4020A01F4020901B4020581C402064
S214443A807C1B402008B5FFF7CFFF104B1A68104B3D
S214443A901A60104B1A68104B1A60104B1A68104B79
S214443AA01A60104B1A68104B1A60104B1A68104B69
S214443AB01A60104B1A68104B1A60104B1A68104B59
S214443AC01A60104B1A68104B1A6008BD5C1A4020E6
S214443AD0701B4020741A4020881B4020701A4020D7
S214443AE0841B4020601A4020741B4020781A4020D3
S214443AF08C1B40206C1A4020801B4020641A4020B7
S214443B00781B4020581A40206C1B402008B5FFF70D
S214443B108BFF104B1A68104B1A60104B1A68104BE8
S214443B201A60104B1A68104B1A60104B1A68104BE8
S214443B301A60104B1A68104B1A60104B1A68104BD8
S214443B401A60104B1A68104B1A60104B1A68104BC8
S214443B501A6008BD5C1D4020701B4020741D402028
S214443B60881B4020701D4020841B4020601D402040
S214443B70741B4020781D40208C1B40206C1D402028
S214443B80801B4020641D4020781B4020581D402048
S214443B906C1B402000230B4A012113600A4A136021
S214443BA00A4A13600A4A13600A4A13600A4A1360B0
S214443BB00A4A13600A4A13600A4A11600A4A1360A2
S214443BC0704700BF901B40208C1B4020881B402021
S214443BD0841B4020801B40207C1B4020781B4020B8
S214443BE0741B4020701B40206C1B402002230B4A51
S214443BF013600B4A136000230A4A13600A4A136090
S214443C000A4A13600A4A13600A4A13600A4A13604F
S214443C100A4A13600A4A1360704700BF901B40204C
S214443C208C1B4020881B4020841B4020801B402047
S214443C307C1B4020781B4020741B4020701B402077
S214443C406C1B40202C4B2D491A6810B542B90A68A3
S214443C50012A05D12A4802602A4802602A4802609E
S214443C602A4A502010602A4A2A4810602A4A126873
S214443C701A602A4B1B780B60294B1C6874B9294B75
S214443C80002118680CF00AFD88B1274B07221A60F9
S214443C900122264B1C60264B1A6008E0012C07D1F3
S214443CA00223214A1360214A1360214A136010BD3F
S214443CB0022C0FD11B4B002118680CF0EFFC002897
S214443CC0F5D0194B03221A600022184B1A60184B81
S214443CD01C60ECE7032CEAD1124B002118680CF068
S214443CE0DDFC0028E3D0104B04221A6001220F4B5F
S214443CF01A6002220E4BCFE7381B4020341B40206C
S214443D00441B4020481B4020501B4020301B402072
S214443D102C1B4020000048C2FC1940201A1E40209C
S214443D20581C4020741C4020401B40203C1B402014
S214443D30601B40200000000038B5174B00211C686B
S214443D4020460CF0B5FC08B104F10044134D20465F
S214443D502C600BF061FE0CA3D3E900230BF0DEFFCE
S214443D600BA3D3E900230BF0AFFE00220C4B0BF061
S214443D70ABFE0C4B00220BF0D1FF0CF09DF90A4B26
S214443D806860186038BD00BF5C8FC2F528DC2740E9
S214443D90B4A766033D39FB3F6C1E4020A41F402059
S214443DA000004E4000408F40741C402008B5074B2E
S214443DB018680CF087FA064B064918600CF082FC2B
S214443DC010B1054B01221A7008BD00BF141E4020D6
S214443DD0501840200000F04154184020FE28D4BF1C
S214443DE001300020704770B50022FF23064ED4B23F
S214443DF0551C8C4202D3D843C0B270BD025D5340BA
S214443E002A46F35CF3E700BFB8804600072101303A
S214443E1008B5FFF7E8FFC0B208BDB0F5447F38B533
S214443E20144617D1244D204695F8EC32FF2B14BF88
S214443E3001330023DBB285F8EC3253701F4A13700B
S214443E40FFF7E4FF1E4BC0B285F8ED0220701870F1
S214443E50012038BD402818D0B0F5547FF8D1164D0F
S214443E60204695F8E832FF2B14BF01330023DAB21C
S214443E7085F8E8226270134A1360FFF7C7FFC0B2A2
S214443E80114B85F8E902207014E00B4D204695F856
S214443E90E032FF2B14BF01330023DAB285F8E02268
S214443EA062700A4A1360FFF7B1FF094BC0B285F847
S214443EB0E10220701860CBE7608740203B19402021
S214443EC03A1940203419402030194020C019402067
S214443ED0BC194020402838B5144616D1254D2046F6
S214443EE095F81833FF2B14BF01330023DAB285F854
S214443EF018236270204A1360FFF788FF1F4BC0B236
S214443F0085F819032070186005E0B0F5547F04D096
S214443F10B0F5447F17D0012038BD164D204695F89D
S214443F202033FF2B14BF01330023DAB285F8202355
S214443F306270134A1360FFF769FFC0B2114B85F8ED
S214443F4021032070DFE70B4D204695F82433FF2BE2
S214443F5014BF01330023DBB285F8243353700A4A76
S214443F601370FFF753FF094BC0B285F82503207042
S214443F701870D0E7608740201C194020181940204C
S214443F80C4184020C0184020CB184020CA184020EF
S214443F90402838B5144617D1254D204695F8183391
S214443FA0FF2B14BF01330023DAB285F85423627022
S214443FB0204A1360FFF72AFF1F4BC0B285F855030B
S214443FC020701860012038BDB0F5547F18D0B0F585
S214443FD0447FF7D1164D204695F86033FF2B14BF27
S214443FE001330023DBB285F860335370134A1370F1
S214443FF0FFF70CFFC0B2124B85F86103207014E043
S2144440000B4D204695F85C33FF2B14BF0133002339
S214444010DBB285F85C3353700A4A1370FFF7F6FE3A
S214444020094BC0B285F85D0320701870CAE700BF1C
S21444403060874020AC184020A8184020A018402094
S2144440409F1840209C1840209B184020402838B594
S214444050144616D1254D204695F86433FF2B14BFDD
S21444406001330023DAB285F864236270204A136071
S214444070FFF7CCFE1F4BC0B285F86503207018606E
S21444408005E0B0F5547F04D0B0F5447F17D0012046
S21444409038BD164D204695F87033FF2B14BF0133B8
S2144440A00023DAB285F870236270134A1360FFF770
S2144440B0ADFEC0B2114B85F871032070DFE70B4D9F
S2144440C0204695F86C33FF2B14BF01330023DBB234
S2144440D085F86C3353700A4A1370FFF797FE094B02
S2144440E0C0B285F86D0320701870D0E76087402012
S2144440F09418402090184020801840207C18402077
S2144441008718402086184020502870B50546144627
S21444411016D18C4A92F8A831FF2B14BF01330023E2
S214444120D9B282F8A811884A2171136040F28533C7
S2144441309D4200F0DD80162D00F0F080012070BD19
S214444140642826D065283BD032284FD0702863D0C8
S214444150712877D0332800F08C806A2800F09F803E
S214444160B0F5617FE2D1774D204695F8F032FF2BCB
S21444417014BF01330023DBB285F8F0325370734A20
S2144441801370FFF743FEC0B2714B85F8F1022070FE
S2144441906DE06C4E204696F8AC32FF2B14BF0133CC
S2144441A00023DBB286F8AC3253706A4A1370FFF7CA
S2144441B02DFE694BC0B286F8B00220701870B5E781
S2144441C0604E204696F81033FF2B14BF013300236D
S2144441D0DBB286F810335370604A1370FFF716FE4E
S2144441E0C0B25F4B86F814032070E7E7554E20466E
S2144441F096F8C432FF2B14BF01330023DBB286F893
S214444200C4325370574A1370FFF700FEC0B2564B81
S21444421086F8C5022070D1E74A4E204696F8B83252
S214444220FF2B14BF01330023DBB286F8B832537039
S2144442304E4A1370FFF7EAFDC0B24D4B86F8B902FA
S2144442402070BBE73F4D204695F80433FF2B14BF40
S21444425001330023DBB285F804335370454A1370A8
S214444260FFF7D4FD444BC0B285F8050320701870A0
S21444427064E7344D204695F82833FF2B14BF0133AA
S2144442800023DBB285F8283353703C4A1370FFF79B
S214444290BDFDC0B23A4B85F829032070E7E7294DA7
S2144442A02046D5F8D832D5F8D822C3F3C733FF2BE7
S2144442B014BF01330023DBB263F3D632C5F8D822E9
S2144442C06370D5F8D8322F4AC3F3C7331360FFF769
S2144442D09DFDB5F8DA32C0B22B4A60F3CE13A5F88A
S2144442E0DA322070B5F8DA32C3F3C713136025E721
S2144442F0144D2046254A95F84033FF2B14BF01330E
S2144443000023DBB285F8403363701370FFF77EFDFD
S214444310C0B21F4B85F841032070A8E70949B1F89D
S2144443209022C2F34313013303F00F0363F348129E
S214444330A1F890226370B1F89032164AC3F343133F
S214444340D4E700BF60874020281C40202C1940201A
S2144443502B1940207C1940207D19402010194020FC
S21444436011194020C6194020C51940205D19402027
S2144443705C194020ED184020EC18402022194020BB
S21444438021194020701940206C194020B91840204B
S214444390B8184020C41A40200F28D4BF013000204B
S2144443A0704770B50022FF23074ED4B2551C8C428A
S2144443B005D3DB4383EA131303F00F0070BD025D9D
S2144443C053402A46F35CF0E7B881460007210130A3
S2144443D008B5FFF7E6FFC0B208BDB0F5AE6F70B5DE
S2144443E0054614461AD1C04D204695F805221309B1
S2144443F0013363F3071203F00F0385F80522BB4A23
S2144444001360FFF7E3FF95F8063260F3030300F00A
S2144444100F0085F80632B64B1860C0E0B0F5B06FB2
S2144444201DD0B0F5B26F35D1AF4D204695F8162263
S21444443002F00F03013363F3030203F00F0385F81E
S2144444401622AC4A1360FFF7C1FF95F8163260F3A4
S214444450071300F00F0085F81632A74BDCE7A24D91
S2144444602046B5F80C22C2F38313013363F3891252
S21444447003F00F03A5F80C22A04A1360FFF7A6FF2B
S21444448095F80D3260F3850300F00F0085F80D3281
S2144444909B4BC1E740F29553984222D040F2855355
S2144444A0984258D050287CD0512835D18E4D20463D
S2144444B095F8302202F00F03013363F3030203F04E
S2144444C00F0385F830228F4A1360FFF77FFF95F875
S2144444D0303260F3071300F00F0085F830328A4B11
S2144444E09AE7814E204696F81B22C2F38303013393
S2144444F003F00F0363F3850286F81B22834A137086
S214444500FFF764FF96F81C3200F00F0060F30303D5
S21444451086F81C327E4B1870602D5DD0612D35D1E7
S214444520714D204695F8402202F00F03013363F3A1
S214444530030203F00F0385F84022764A1360FFF720
S21444454045FF95F8403260F3071300F00F0085F8F6
S2144445504032714B60E7644E2046D6F82022C2F3C0
S2144445608333013363F3913203F00F03C6F82022FA
S2144445706A4A1360FFF72AFF96F8223260F38503EF
S21444458000F00F0086F82232654B1860132D3ED09B
S214444590142D57D0152D70D0162D00F0898001208B
S2144445A070BD514D204695F8282202F00F03013382
S2144445B063F3030203F00F0385F82822594A136075
S2144445C0FFF704FF95F8283260F3071300F00F0056
S2144445D085F82832544B1FE7434D204695F8382239
S2144445E002F00F03013363F3030203F00F0385F86D
S2144445F038224E4A1360FFF7E9FE95F8383260F3E6
S214444600071300F00F0085F83832494B04E7364D5F
S2144446102046B5F84A22C2F38313013363F3891262
S21444462003F00F03A5F84A22424A1360FFF7CEFE72
S21444463095F84B3260F3850300F00F0085F84B3253
S2144446403D4BE9E6284D204695F8522202F00F03EA
S214444650013363F3030203F00F0385F85222374A0B
S2144446601360FFF7B3FE95F8523260F3071300F079
S2144446700F0085F85232324BCEE61B4D204695F855
S2144446805A2202F00F03013363F3030203F00F03CD
S21444469085F85A222B4A1360FFF798FE95F85A324B
S2144446A060F3071300F00F0085F85A32264BB3E642
S2144446B00D4D2046B5F89022C2F34313013363F3FD
S2144446C0481203F00F03A5F89022204A1360FFF720
S2144446D07DFE95F8913260F3440300F00F0085F8B0
S2144446E091321B4B98E600BF60874020101A40204A
S2144446F00C1A4020301E40202C1E4020E81D40202E
S214444700E41D4020A41A4020A01A4020DB19402073
S214444710DA194020841A4020801A4020E4194020A8
S214444720E0194020B41A4020B01A4020941A402081
S214444730901A4020001B4020FC1A4020E41A4020D7
S214444740E01A4020CC1A4020C81A4020C41A402000
S214444750C01A40200D4B0E490E4810B51C680E4B2F
S2144447601A78A2421A460BD10B8801339BB2312BDE
S2144447700B8008D932230B8001230370147010BDBC
S21444478000230B80F9E70023F7E700BF541D4020C1
S2144447909A174020821740208A1740200D4B0E4916
S2144447A00E4810B51C680E4B1A78A2421A460BD116
S2144447B00B8801339BB2312B0B8008D932230B80F4
S2144447C001230370147010BD00230B80F9E7002307
S2144447D0F7E700BFB01D40209817402081174020BF
S2144447E0891740200D4B0E490E4810B51C680E4BD9
S2144447F01A78A2421A460BD10B8801339BB2312B4E
S2144448000B8008D932230B8001230370147010BD2B
S21444481000230B80F9E70023F7E700BFA01D4020E4
S2144448209617402080174020881740200D4B0E498D
S2144448300E4810B51C680E4B1A78A2421A460BD185
S2144448400B8801339BB2312B0B8008D932230B8063
S21444485001230370147010BD00230B80F9E7002376
S214444860F7E700BF841D4020941740207F17402060
S2144448708717402008B5FFF76DFFFFF78FFFFFF758
S214444880B1FFBDE80840FFF7D1BF0D4B0D490E48B8
S21444489010B51C780D4B1A78A2421A460BD10B88D9
S2144448A001339BB2312B0B8008D932230B80012372
S2144448B00370147010BD00230B80F9E70023F7E75C
S2144448C00C1D402092174020241C40208617402070
S2144448D00D4B0E490E4810B51C780E4B1A78A24262
S2144448E01A460BD10B8801339BB2312B0B8008D967
S2144448F032230B8001230370147010BD00230B80F9
S214444900F9E70023F7E700BF981C402090174020A3
S214444910231C4020851740200D4B0E490E4810B5E9
S2144449201C680E4B1A78A2421A460BD10B880133E8
S2144449309BB2312B0B8008D932230B8001230370A2
S214444940147010BD00230B80F9E70023F7E700BF7F
S214444950501D40208E174020221C402084174020A3
S2144449600D4B0E490E4810B51C680E4B1A78A242E1
S2144449701A460BD10B8801339BB2312B0B8008D9D6
S21444498032230B8001230370147010BD00230B8068
S214444990F9E70023F7E700BFCC1C40208C174020E3
S2144449A0211C4020831740201D4B1B78012B30D1FF
S2144449B01C4B1B78003B18BF01231B4A13701B4B30
S2144449C01B78012B27D1174B1B78003B18BF0123BC
S2144449D0174A1370174B1B78012B1ED1114B1B78AB
S2144449E0003B18BF0123144A1370144B1B78012B49
S2144449F00CD0134B1B78012B08D0124B1B78012B81
S214444A0004D0114B1B785A1E534253410F4A13701D
S214444A1070470023D1E70023DAE70023E3E700BF2B
S214444A20521F4020A8174020261C4020511F4020DB
S214444A30251C4020501F4020201C40208217402028
S214444A4081174020801740207F1740207E17402043
S214444A500B4B1B68012B09D10A4A11680A4A106895
S214444A6088420ABF094A116013607047022B06D178
S214444A70074B1B68012B02BF044B00221A60704789
S214444A80541C40205C1F4020801F4020781F40203C
S214444A90681F4020094B0A491A6801328A4288BF77
S214444AA000221A601A792AB19A68054901328A4264
S214444AB09A6001D900229A60704700BFAC1F40201C
S214444AC07F510100024B187100B99860704700BFCF
S214444AD0AC1F4020014B9868704700BFAC1F402075
S214444AE0194B30B51C68194B012C03D11A780AB9F6
S214444AF002225A70164A1178012903D19A780AB9C3
S214444B0003225A70134D0022012913482A7012D1E9
S214444B10012C0CD15A782970032A18BF022202703D
S214444B200A461A704A1E51425141997030BD0324B8
S214444B3004705C70F5E7012C04D1022202705A70AE
S214444B402246EEE70124F3E7741F4020B81F4020B6
S214444B50601F402078174020FA1A402070B5FFF7AF
S214444B60BFFF6C4B1C78012C2CD06B4B1C78012C53
S214444B7028D06A4B1C78012C24D0694B1C78012C15
S214444B8020D0684B1C78012C1CD0674B1C78012C19
S214444B9018D0664B1C78012C14D0654B1C78012C1D
S214444BA010D0644B1C78012C0CD0634B1B78012B23
S214444BB015D0624B1C78012C04D0614B1C78631EC4
S214444BC05C425C415F4B604A1968604B12881B68C4
S214444BD03CB101291AD15E4B02221A7010E001241E
S214444BE0F0E70129F7D0012A00F09180012B0FD07D
S214444BF0584B1B68012B03D0574B1B78012B12D103
S214444C0000240225FFF736FE002043E0012B02D1A4
S214444C104F4B0322E1E7012A02D14D4B0422DCE745
S214444C204B4B0122D9E74D4B494E1B68013B022BA7
S214444C3009D84B4B002234701C704A4B1A604A4BBE
S214444C401C700325E0E7494B34701D78484B1C78AC
S214444C50022C27D0032C37D0012C4BD1454B1B6854
S214444C60012B0BD0444B4FF07E5118680BF020FDBF
S214444C7040BB05230224337002250BE015BB3E4B94
S214444C804FF07E5118680BF013FD03462846002B60
S214444C9018BF0324354B1D60384B1C70BDE870406C
S214444CA0FFF710BF344B4FF07E5118680BF000FDF1
S214444CB018B935BB06233370DEE7EDB92D4B1B68B8
S214444CC0012B1CD00024BCE72B4B4FF07E511868B8
S214444CD00BF0EEFCA8B1032D13D1264B1B68012B19
S214444CE011D0FFF7F7FE1E2835BF03240224012007
S214444CF00020CFE7002487E70024012584E7032427
S214444D0082E7012480E700252C462846C2E7012B8B
S214444D1083D17DE7781740208217402081174020B2
S214444D20801740207F174020241C4020231C40200E
S214444D30221C4020211C4020201C4020251C4020B2
S214444D40261C4020681F402004184020881D402010
S214444D50F81A4020781F4020A8174020201E4020E4
S214444D6025184020581B402024184020541C40201E
S214444D70FA1A4020981D4020741C4020F91A4020FE
S214444D801A4B1A781A4B1B7813432DD1194B1B78A0
S214444D90013B18BF0123184A1370184B184A1B6866
S214444DA0003B18BF01231370164B1A78164B1B781A
S214444DB01343164B14BF012200221A70144B154A93
S214444DC01B78013B18BF01231370134B134A1B78FF
S214444DD0003B18BF01231370114B124A1B78003B4B
S214444DE018BF0123137070470123D4E7E21D402007
S214444DF0E11D4020181E4020671840208C1E40208D
S214444E0064184020D11D4020D01D40206518402005
S214444E10191E4020661840201A1E40206318402061
S214444E20241E40206218402038B52A4B2A4D1B6861
S214444E30012B30D1294B1C68294B012C1B6814D1FB
S214444E40002B42D1274B4FF07E5118680BF03AFCAA
S214444E5000283AD0244B002118680BF01FFC002889
S214444E6033D02C60214B1C7038BD1C432DD11D4BB8
S214444E704FF07E5118680BF025FC30B31A4B0021D6
S214444E8018680BF00BFC00B32C60194B1C68003CF4
S214444E9018BF0124E6E7C3B9164B1C68164B012C11
S214444EA01B6810D18BB90F4B4FF07E5118680BF02E
S214444EB009FC50B1114B002118680BF0EFFB20B1F0
S214444EC00B4B1C6001E01C43EDD02B68002BDCD060
S214444ED00124C7E7541C4020601C4020641F402027
S214444EE0881F4020741C40208C1F40207917402087
S214444EF0101B4020941D4020BC1D4020B81D40205F
S214444F0038B50124204B00251C70204B1C70204BC8
S214444F101C70204B1C70204B1D70204B1D70204B6A
S214444F201C70204B1C70204B1D70204B1D70204B5A
S214444F3018680BF0E5FB1F4B18601F4B1C601F4B9B
S214444F401C601F4B1C601F4B1A681F4B1A601522AF
S214444F501E4B1C701E4B1C701E4B1C701E4B1C7034
S214444F601E4B1D701E4B1D701E4B1A7006221E4B88
S214444F701D701E4B1D701E4B1A7018221D4B1D7043
S214444F801D4B1A7038BD00BFC4194020201940205C
S214444F903919402038194020C9184020C8184020E4
S214444FA09D1840209E184020841840208518402094
S214444FB0581B4020A8194020A4194020941940208A
S214444FC0F8184020581C402000194020B4194020AE
S214444FD012194020A1184020881840202A19402041
S214444FE029194020281940202719402026194020F6
S214444FF0251940202419402023194020064B01221D
S2144450001A70064B1B78934204D1054A13707822D3
S214445010044B1A80704700BF271B4020631840206B
S214445020261B4020241B402008B5FFF7E7FFFEF769
S2144450306DFD054B1B68012B1EBF044B00221A60F6
S214445040BDE80840FFF716BC881D4020041B4020DE
S21444505008B5FFF7D3FFFEF715FD064B1B68012B7B
S2144450601EBF054B00221A60044B1A68044B1A6094
S21444507008BD00BF681F40205C1C4020541F4020D1
S214445080701C40200D4B1A780D4B32B90D4A1278DD
S214445090012A02BF1A8801321A801A88B2F5FA7FAA
S2144450A006D300221A80074B1A700522064B1A7044
S2144450B00023064A1370064A13807047621840203D
S2144450C01A184020271B402068184020261B4020E2
S2144450D0241B402008B5FFF7D5FFFEF75BFD0023F1
S2144450E0024A1360024A136008BD00BF5C1C40209D
S2144450F0041B402038B5154A0223154D1360154A43
S214445100154C136001232B602360FFF7BBFFFEF7AB
S2144451106DFD124B1B88BBB9114B124A1B681268B3
S2144451201343114A126813430ED1104B104A1B788E
S2144451301278134308D10F4A2B6013600E4A23603B
S214445140136003220D4B1A6038BD00BF601B40201D
S2144451505C1C4020581C4020041B4020041840205F
S214445160681F4020881D4020781F40207817402024
S214445170A8174020901B40208C1B4020541C4020E5
S21444518008B5FFF7BDFEFFF7E9FCFEF7D3F9FCF7D9
S21444519077FBFEF7E7FA0C4B1B68032B13D8DFE8C4
S2144451A003F002060A0EBDE80840FFF73DBFBDE81F
S2144451B00840FFF74DBFBDE80840FFF79BBFBDE87A
S2144451C00840FFF787BF08BD541C402010B5314C3B
S2144451D0FFF7D6FD2378052B5AD8DFE803F00316ED
S2144451E038474F5300F078F8FEF7E0FD2A4B1B781B
S2144451F0012B3AD1294A1178294A12780A4334D1E4
S214445200284A1360284A137018E0274B1A78511E10
S2144452104B424B4125490B7025490B7025490B7071
S21444522025490B70254B1B78012B254B08D1012AA9
S21444523006D11A700022234B1A700223237014E0FE
S21444524000221A70144B1B787BB90323F6E7FFF74A
S21444525097FFFEF7F7FCFEF76FFD0F4B1B7823B95D
S214445260194B1B68023B012BEFD910BD174B00228C
S2144452701A800122164B1A700423DFE7BDE810405B
S214445280FFF700BF134B1B88042BEED80023B9E767
S2144452900023D3E768184020691840206718402048
S2144452A0631840204C1B4020281B40206E1840208A
S2144452B06D1840206C1840206B1840207018402011
S2144452C07518402072184020541C40201A1840205C
S2144452D074184020C21D4020074B1A221A6003232C
S2144452E0064A1360064A13600122064B1A60064BB0
S2144452F0064A1A60704700BFA41B4020A01B4020EB
S2144453009C1B4020981B4020941B4020EFAB03007E
S214445310002110B50446084615F010FC0121002073
S21444532015F00CFC0221002015F008FC0321002097
S21444533015F004FC002015F0FDFA0E49002015F087
S2144453400FFA0D4BA2B20020197815F047FB0B4913
S214445350002015F0B9FE0A49002015F0B5FE0949AB
S214445360002015F0B1FE08490020BDE8104015F0B5
S214445370ABBE00BFE49A46001C9B46006C9C4600AD
S2144453804C9C46002C9C46000C9C4600F8B50D46AA
S21444539006461F4928461F4F0BF09EF9044670B137
S2144453A04CF24453F85806F54553123307EB83073B
S2144453B07D60032E2BD8DFE806F01A21242700212F
S2144453C028460BF07FF980B94CF24453F8580AF05B
S2144453D079FF29460AF0CEFF0AF01EFB00220E4B48
S2144453E00AF09CFC0AF048FEDDE72046DBE782B282
S2144453F000210020BDE8F84016F0B0B882B2012182
S214445400F7E782B20221F4E782B20321F1E7F8BD5E
S2144454100000C842EC4B41200000594008B5034800
S2144454201AF054FD024B187008BD00BF64A646002F
S2144454304C4B4020F7B50123104C114D6370A21C11
S214445440EB68A91C0F480235009335F8023C1AF065
S214445450DFFB00222073A01C6178134615F8017BFD
S214445460013310F8016BDBB2B7421CBF01220021A6
S2144454700A2BF3D102B1617003B0F0BD4C4B40200F
S214445480C01F402078A646004B7C062B0AD101223A
S214445490054B1A74CA7B1A2A04D1032203F111015C
S2144454A01AF0F6BE704700BFC01F40204B7C062B48
S2144454B00AD10122054B1A74CA7B2A2A04D1032234
S2144454C003F111011AF0E4BE704700BFC01F40202C
S2144454D01FB500231A210446039301238DF8073091
S2144454E01BF01CF80B4B03930B4B1A7C002AFCD086
S2144454F01B7C63B102A920461AF014FF8DF80700FE
S214445500039B5A1E039213B19DF80730F1E704B08B
S21444551010BD00BF006A1800C01F402008B5A12077
S21444552019F028FB00220A49A12019F022FB094B56
S214445530094902220120C3F8F413C3F8982DC3F88E
S214445540F813C3F8902D0549BDE808401AF012B880
S2144455506BF945000000294004002800D8A5460001
S21444556008B5A22019F006FB00220B49A22019F028
S21444557000FB0A4B0A4A01210020C3F8E023C3F883
S214445580AC1DC3F8E42302220649C3F8A42DBDE8A3
S214445590084019F02FBD00BF71F9450000002940AE
S2144455A002002800FCA5460010B508221749012031
S2144455B04FF480341AF09AF8012308221449002044
S2144455C019F004FE0021084619F04EFF022801D1C6
S2144455D0013CF7D14FF48034002101201AF090F8B2
S2144455E0022801D1013CF7D1094A0823A2F1080058
S2144455F012F8011B013B10F8014BA14204BF0131D4
S21444560002F8011C13F0FF03F2D110BDD41F402052
S214445610DC1F402082B00190019B5A1E0192002B51
S214445620FAD102B07047044B4FF400224FF4FA709C
S214445630C3F8C022FFF7EEBF00002940044B4FF4E6
S21444564020124FF4FA70C3F8C022FFF7E3BF00BF3E
S214445650000029402DE9F04104460D461046002935
S2144456603ED1DFF8908050260B46C1B2564308F12F
S21444567010072846BA19B04416F080FF1C484FF469
S214445680FB534FF4FB62D8F81410083603FB0403AC
S2144456903744D3F8FC3802FB043203F17A0602F5A9
S2144456A0107C02F5427240F82C1098F8581040F8D6
S2144456B02210FB2212FB046200EB4212A94211D8CC
S2144456C04FF4FB520133642102FB0404B3FBF1F2B2
S2144456D001FB1233C4F8FC3804F52154012323603B
S2144456E0BDE8F08117F8016B013502F8016BE5E778
S2144456F0EC4B41204C4B40202DE9F04104460D46EE
S214445700104600293ED1DFF8908050260B46C1B2A1
S214445710564308F521670120BA19B04416F02EFF07
S2144457201C484FF4FB534FF4FB62D8F8141A08365F
S21444573003FB04033744D3F8FC3802FB043203F17A
S2144457407A0602F5107C02F5427240F82C1098F85E
S214445750581A40F82210FB2212FB046200EB421255
S214445760A94211D84FF4FB520133642102FB0404CE
S214445770B3FBF1F201FB1233C4F8FC3804F52154B0
S21444578001232360BDE8F08117F8016B013502F868
S214445790016BE5E7EC4B41204C4B40202DE9F041B2
S2144457A004460D46104600293ED1DFF89080502628
S2144457B00B46C1B2564308F546770220BA19B044A0
S2144457C016F0DCFE1C484FF4FB534FF4FB62D8F84B
S2144457D01C13083603FB04033744D3F8FC3802FB97
S2144457E0043203F17A0602F5107C02F5427240F860
S2144457F02C1098F8601340F82210FB2212FB046227
S21444580000EB4212A94211D84FF4FB5201336421F3
S21444581002FB0404B3FBF1F201FB1233C4F8FC3878
S21444582004F5215401232360BDE8F08117F8016B89
S214445830013502F8016BE5E7EC4B4120445C40201F
S2144458402DE9F04104460D46104600293ED1DFF8C6
S214445850908050260B46C1B2564308F6185703208C
S214445860BA19B04416F08AFE1C484FF4FB534FF462
S214445870FB62D8F81C1D083603FB04033744D3F8F0
S214445880FC3802FB043203F17A0602F5107C02F57A
S214445890427240F82C1098F8601D40F82210FB2203
S2144458A012FB046200EB4212A94211D84FF4FB5299
S2144458B00133642102FB0404B3FBF1F201FB12330F
S2144458C0C4F8FC3804F5215401232360BDE8F08174
S2144458D017F8016B013502F8016BE5E7EC4B412004
S2144458E0445C40202DE9F04104460D46104600290C
S2144458F03ED1DFF8908050260B46C1B2564308F599
S214445900C4670420BA19B04416F038FE1C484FF455
S214445910FB534FF4FB62D8F82416083603FB040303
S2144459203744D3F8FC3802FB043203F17A0602F516
S214445930107C02F5427240F82C1098F8681640F82D
S2144459402210FB2212FB046200EB4212A94211D839
S2144459504FF4FB520133642102FB0404B3FBF1F21F
S21444596001FB1233C4F8FC3804F5215401232360A8
S214445970BDE8F08117F8016B013502F8016BE5E7E5
S214445980EC4B41203C6D40202DE9F04104460D4649
S214445990104600293ED1DFF8908050260B46C1B20F
S2144459A05643A8F1D8070520BA19B04416F0E6FDC8
S2144459B01C484FF4FB534FF4FB6258F8D41C08368B
S2144459C003FB04033744D3F8FC3802FB043203F1E8
S2144459D07A0602F5107C02F5427240F82C1018F84C
S2144459E0901C40F82210FB2212FB046200EB421289
S2144459F0A94211D84FF4FB520133642102FB04043C
S214445A00B3FBF1F201FB1233C4F8FC3804F521541D
S214445A1001232360BDE8F08117F8016B013502F8D5
S214445A20016BE5E7EC4B4120347E40204FF4FB52BB
S214445A30054B02FB0033D3F8F808D3F8FC38C31AF6
S214445A4058425841704700BFEC4B41202DE9F74F70
S214445A50D14D0021D14E4FF4FB692C4641F698783F
S214445A6037464FF0640A0846FFF7E0FF58BBD6F8BF
S214445A70F83809FB013202F5427257F822C008FB97
S214445A80014200924FF4FB524A4302EB43123A441B
S214445A90019200F1010EC0B2844500F2A88009FBD1
S214445AA00132013385F820C002F5107257F82220DF
S214445AB06A624FF0010285F82120B3FBFAF20AFB32
S214445AC01233C6F8F8380131454406F5FB56062924
S214445AD0C9D194F82130012B19D1002384F8213000
S214445AE0636AB3F5407F00F0CF8000F29F80B3F541
S214445AF0BA7F00F0D28000F28B80422B00F0D9802F
S214445B007FD8402B00F0C380412B00F0C38041F681
S214445B10B973E25C012A0FD10022E25441F6BC7309
S214445B20E358932B00F0D68000F2C680912B00F009
S214445B30CB80922B00F0CB8043F65173E25C012A73
S214445B4014D10022E25443F65473E358962B00F0E3
S214445B50E98000F2CA80822B00F0E18000F2BD802A
S214445B60722B00F0E580732B00F0E58045F6E96380
S214445B70E25C012A14D10022E25445F6EC63E35871
S214445B809B2B00F0F98000F2E4808D2B00F0088116
S214445B9000F2D780722B00F0F880732B00F0F88068
S214445BA047F68163E25C012A0BD10022E25447F6B1
S214445BB08463E358722B00F0F980732B01D102F012
S214445BC0ADFD49F61963E25C012A40F0F7800022F5
S214445BD0E25449F61C63E358722B00F0EA80732BB8
S214445BE040F0EC8003B0BDE8F04F02F0C7BD019A28
S214445BF002EB000B009A9BF840BF02F800B07046D8
S214445C0047E740F25512934281D101F0F9FC7EE712
S214445C10B3F5BE7F44D040F22122934243D0B3F53D
S214445C20BC7F7FF474AF01F035FD70E740F28552D7
S214445C30934226D00DD8B3F5AE6F19D0B3F5B06FF6
S214445C4019D040F2013293427FF461AF01F0E2FD95
S214445C505DE740F29552934210D040F277729342F9
S214445C6024D0B3F5B26F7FF452AF01F0A1FE4EE7F5
S214445C7001F0DCFD4BE701F029FE48E701F0AAFEFF
S214445C8045E701F06DFE42E701F0A4FD3FE701F071
S214445C903CFC3CE701F04CFC39E701F0D9FC36E724
S214445CA001F01AFD33E701F035FD30E701F0AAFEB6
S214445CB02DE701F05FFC2AE740F2511293427FF44D
S214445CC03BAF01F007FF37E701F0AEFE34E701F0E3
S214445CD0D1FE31E701F0E0FE2EE78C2B25D0922B47
S214445CE07FF444AF02F058F840E7AA2B26D007D8F2
S214445CF09A2B0ED0A02B7FF439AF02F06DF935E71E
S214445D00C82B09D0B3F5F36F7FF430AF02F02EFA08
S214445D102CE702F021F929E702F0EAF926E701F038
S214445D20A9FF23E702F0C0F820E701F0CDFF1DE706
S214445D3001F026FF1AE701F06BFF17E702F098F927
S214445D4014E7932B2FD0972B7FF42AAF02F0FEFA5A
S214445D5026E7C92B13D007D8A12B13D0AA2B7FF440
S214445D601FAF02F0C3FB1BE740F2997293427FF4E5
S214445D7017AF02F0A1FC13E702F040FB10E702F075
S214445D80F5FB0DE702F07AFB0AE702F003FA07E7B1
S214445D9002F048FA04E700BFD88A4020EC4B412082
S214445DA002F022FCFCE602F06FFAF9E602F098FCF8
S214445DB007E703B0BDE8F04F02F0C2BC03B0BDE84D
S214445DC0F08FEB4BEB4A5969DFF8CCC30A40EA49FB
S214445DD02DE9F0475A610022E84D4FF00008E84E9E
S214445DE04FF000095A6583F86F201A67E54CDFF8D0
S214445DF0ACE3DFF8ACA3C3E90212197C21F0070137
S214445E001974596A29405962196C01F000411964A1
S214445E10596C31405964996C01F0604141F4C82191
S214445E209964D949C3E91312996D01F07041996593
S214445E30D96D2940D965196E01F000411966B3F849
S214445E40641001EA0C01A3F86410B3F8681001EA80
S214445E500C01A3F86810596F01F07F415967986F99
S214445E60CA49D3F89870084083F88C209867D3F8CA
S214445E70800000F07F40C3F88000D3F8840000F030
S214445E807F40C3E92102D3F890002040C3F8900035
S214445E90D3F8940000F07C40C3F89400BC48074014
S214445EA0C3F89870D3F89C7007F04047C3F89C70CA
S214445EB0D3F8A0703740C3E92872D3F8A8700F40CF
S214445EC0C3F8A870D3F8AC7007F04047C3F8AC707A
S214445ED0D3F8B47007F04047C3F8B470D3F8B8703A
S214445EE007F07F47C3F8B870B3F8B07083F8BB20A8
S214445EF062F30D07A3F8B07093F8BC7027F003075D
S214445F0083F8BC70D3F8C070C3F8D4A007F0004739
S214445F10C3F8C070D3F8C4700740C3F8C470D3F84D
S214445F20C87007F07047C3F8C870D3F8CC7007F051
S214445F307F47C3F8CC70B3F8D07007EA0E07A3F8CF
S214445F40D070D3F8D87007F04047C3F8D870D3F869
S214445F50DC7007F07847C3E9377293F8E47062F36D
S214445F60000783F8E470D3F8E87007F07E4747F4F8
S214445F708037C3F8E870D3F8EC703740C3F8EC7059
S214445F80D3F8087107F04047C3F80871D3F80C718A
S214445F903740C3E94372D3F814710F40C3E9402233
S214445FA0C3E93E89C3F81471D3F81871A3F82821BD
S214445FB007F0404783F85421A3F86C21C3F838A16E
S214445FC0C3E9467293F8207127F0030783F82071DB
S214445FD0D3F8247107F06047C3F82471D3F82C71C2
S214445FE007F07047C3F82C71D3F8307107F07F4739
S214445FF0C3F83071B3F8347107EA0E0ED3F83C7127
S2144460000740A3F834E1C3F83C71D3F8407107F075
S2144460107847C3F84071B3F8447107F47847A3F857
S2144460204471D3F8487107F07E4747F48037C3F885
S2144460304871D3F84C713E40C3F84C61D3F8506174
S21444604006F06046C3F85061D3F868612E40C3E951
S2144460505689C3F86861D3F87061A3F874212E405A
S214446060C3F8782183F88021C3F87061D3F87C6143
S21444607083F8E42106F07F46A3F8A021C3F8A421C0
S214446080C3F87C61D3F88461A3F8A8212640C3F8FA
S214446090AC2183F8B021C6F30747C3F88461C3F83C
S2144460A0B42107F0E10683F8B821C3F8BC2183F88D
S2144460B08661D3F8C46183F8C02106F07C46354F28
S2144460C0C3F8C461D3F8C8610640C3E97722C3E97C
S2144460D06222C3E96422C3E96622C3F8C861D3F8DE
S2144460E0D06183F8942206F00046C3F82C2283F845
S2144460F03022C3F8342283F8382283F85222C3F875
S2144461003C2283F84022C3F8442283F82822C3E979
S2144461107462D3F848620640C3F84862D3F84C62C7
S21444612006F07F46C3F84C6293F8986226F01F0642
S21444613046F0010683F89862B3F89C6262F3090657
S214446140A3F89C6293F8A06226F00F0683F8A06238
S21444615093F8A46262F3020683F8A462D3F820623A
S2144461603040C3E9880293F8A80262F3030019E0BA
S2144461706087402000E01FE00000E2810000F0FF5E
S214446180000080FF0000FEFF0080204E0000FCFF61
S2144461900000C0FF00E0FFFF00C0FFFF00F0FFFF6D
S2144461A00000C04B83F8A802D3F8000200F0704009
S2144461B0C3F8000283F80422D3F80802D3F8F8623E
S2144461C000F00040C3F8102206F07846A3F8DC221C
S2144461D0C3F80802B3F80C02C3F8E02200EA0C0C39
S2144461E0D3F8140200F07F40A3F80CC2C3F814029C
S2144461F0D3F818020840C3F81802D3F8C402204063
S214446200C3F8C402D3F8AC0200F07E40C3F8AC0234
S214446210D3F8B00200F00040C3F8B00293F8B402DA
S21444622020F00F0083F8B402D3F8B80200F07840A8
S214446230C3F8B802D3F8BC0200F07F40C3F8BC02EF
S214446240B3F8C0023840C3E9BE62A3F8C002D3F82C
S214446250D86293F8000306F0004662F30000C3F8E1
S214446260D86283F8000393F8E402D3F8EC6262F34E
S21444627000000E4083F8E402D3F8E802C3F8EC6268
S2144462800540D3F8F00200F04040C3F8E852C5F3A6
S2144462900745C3F8F002D3F8F40262F3071500F09A
S2144462A0784083F8EA52C3F8F402D3F8040300F0C3
S2144462B07840C3F80403D3F8080300F07F40C3F8DB
S2144462C00803B3F80C033840A3F80C03D3F81003C0
S2144462D000F07E40C3F81003D3F814032040C3E90B
S2144462E0C50293F81C0362F3000083F81C03D3F83A
S2144462F0200300F07F40C3F82003D3F82403014072
S214446300C3F82413D3F828130C40D3F8401301F0F1
S2144463107F40090EC3F8284321F03F01C3E9B28900
S214446320C3F8400383F84313D3F84413D3F848031D
S21444633001F07841C3F8542300F07840C3F864234E
S214446340C3F8441393F8581362F3000183F85813C0
S214446350D3F85C1301F07F41C3F85C1393F86213DF
S21444636021F00301C3E9D20283F8621393F8500381
S21444637093F8681362F3000062F3000193F86E2307
S21444638083F8500322F0030283F86813C3E9CC89E8
S21444639083F86E23BDE8F08741F6987308490022D7
S2144463A058430B182830DA64084483F848202023DE
S2144463B0013B00F8012B13F0FF03F9D1704700BFEF
S2144463C0D88A402041F6987310B558430B4C41F692
S2144463D092732218D35A28225A4300231118503055
S2144463E0104421441A46204481F870304B670133E8
S2144463F000F8012BDBB2202BF9D110BDD88A4020FF
S2144464002DE9F8439946234B0546884603EB00138B
S2144464109B6A402B31D820494FF4FB5303FB0013AF
S21444642042F644015B5843B341F698761B4C00272A
S2144464304FF0280C06FB00F3E11801F5FC5110312F
S214446440F8B248451BD328467543FFF7A5FF41F6E7
S2144464509071601928260122435A06FB03551344BB
S2144464602C4484F87120C4F8748084F87090C8244E
S214446470B3FBF4F204FB12334352BDE8F8830888B6
S21444648012F807E00CFB003020443844013780F80B
S21444649050E0D5E7C01F4020EC4B4120D88A40202E
S2144464A041F6987241F692732DE9F34102FB00F1EE
S2144464B04E4D04466A18D05A282202FB00122A443B
S2144464C092F87020082A31D8494B082203EB04136B
S2144464D09A62282341F6947603FB00F241F69873B9
S2144464E020466343D118EF18503329441344414A95
S2144464F02B4402EB041200934B6FB95D15F0C6FFB4
S214446500012C80462FD143F62C711C206B5C013342
S214446510B3FBF0F200FB12336B54B8F1000F2BD0F0
S214446520B8F1020F40D002B0BDE8F081102A04D87A
S2144465302F4B102203EB0413CAE7182A05D82C491C
S214446540182301EB04118B62C3E7202A04D8284998
S214446550202301EB0411F6E7402ABAD82449402305
S21444656001EB0411EFE7BB5D0E210133B3FBF1F2FF
S21444657001FB1233BB55D0E72046FFF723FF41F615
S214446580987041F69271604328242E18735A04FB7F
S21444659003040133C8202544B3FBF0F200FB123356
S2144465A085F871807352BEE72046FFF70BFF41F62D
S2144465B0987041F692710022444328202E19735A4B
S2144465C000FB03440133C820254485F87120B3FBFF
S2144465D0F0F200FB1233064A7352D2E922310133F9
S2144465E041F10001C2E922319DE700BFD88A40202C
S2144465F0C01F4020E41F4020F8B500240A4D41F651
S21444660098760A4F06FB04F22821E0B2D35B01FBDE
S21444661003232B4493F87130012B01D1FFF740FF3D
S2144466200134062CEED1F8BDD88A40206AAA402010
S21444663008B50B21034821F0BFF9034B83F828091A
S21444664008BD00BF02172940347E402001290A466F
S21444665028BF0122072819D8DFE800F004070B0DED
S2144466601012141600210A4801E00A21094821F0B4
S2144466706AB90C21F7E702210748F8E70D21F2E74B
S2144466800E21F0E70F21EEE70021F5E7704700BF43
S21444669002172940101729400017294007281AD8FE
S2144466A0DFE800F004070B0E1013151708210B48FB
S2144466B001E00B210A4821F07FB901210948FAE795
S2144466C00B21F4E704210848F5E70521FBE70821F8
S2144466D0F9E70A21F7E7FF20704700BF061729406D
S2144466E002172940121729400417294001284FF061
S2144466F002010CBF0022012210B50446034821F0D3
S21444670022F9034A4CF24053D45010BD081729408E
S214446710EC4B412005281DD8DFE800F003080C1098
S21444672014180D4A4CF27453D05A70470A4A4CF225
S2144467307653F9E7084A4CF27853F5E7064A4CF2A2
S2144467407A53F1E7044A4CF27C53EDE7024A4CF2A2
S2144467507E53E9E7FF207047EC4B412008B50621FD
S21444676000200FF070FE024A4CF27453D05208BD1B
S214446770EC4B412010B5022101200FF064FE064C7C
S2144467804CF276532B21E05201200FF05CFE4CF283
S2144467907E53E05210BD00BFEC4B412010B50321A0
S2144467A002200FF050FE094C4CF278530421E0527C
S2144467B002200FF048FE4CF27A530521E0520220A4
S2144467C00FF041FE4CF27C53E05210BDEC4B41209E
S2144467D000210FF025BD084A4CF2385382B00749D1
S2144467E0D35800930B68009A9B1A0193019B8342EB
S2144467F0F8D902B0704700BFEC4B41202411422028
S21444680038B50F4D0F4C95F890305BB901234CF2D8
S2144468103C5285F89030A3580133A350BDE8384025
S21444682006F006BE07F0C2FA4CF23C52002385F846
S2144468309030A3580133A3504CF23852EBE700BFD4
S214446840C01F4020EC4B41200020FFF74FBF10B53F
S2144468508D20244C18F08EF9002223498D2018F000
S21444686088F98F2018F086F9002220498F2018F0E6
S21444687080F9972018F07EF900221D49972018F0D9
S21444688078F99A2018F076F900221A499A2018F0D6
S21444689070F9194900201AF0B5FC184902201AF07C
S2144468A0B1FC17490A201AF0ADFC16490D201AF01F
S2144468B0A9FC2146012200201AF026FF04F5967111
S2144468C0012202201AF020FF04F26C5101220A2011
S2144468D01AF01AFF04F28C5101220D20BDE8104034
S2144468E01AF012BFF84E4120111C4600171C4600F1
S2144468F01D1C4600231C460064A7460038A74600D5
S2144469000CA74600E0A6460010B48AB90949D1F857
S2144469106C3891F8B848CA18013301F6B801DBB2AE
S21444692082F8584610BC012241F84C3C1BF03CB857
S21444693010BC7047EC4B412010B48AB90949D1F8D1
S214446940743891F8D848CA18013301F6D801DBB236
S21444695082F8584710BC012241F8643C1BF024B826
S21444696010BC7047EC4B4120194B012142F64400C1
S2144469700022195044F2A470195046F2047019507B
S21444698048F2646019504AF2C45019504CF22450EC
S214446990195042F648015A5044F2A8715A5046F2E9
S2144469A008715A5048F268615A504AF2C8515A50CF
S2144469B04CF22851C3E9C1225A504CF248524CF288
S2144469C0503199504CF244524FF4486199507047B4
S2144469D0EC4B412010B5064B4FF4FB5404FB0030FF
S2144469E042F64803C15042F64C03C25010BD00BFA5
S2144469F0EC4B4120094BD3E9C1218A420BD01A44BF
S214446A0092F8042202700020D3F804230132D2B252
S214446A10C3F8042370470120704700BFEC4B412065
S214446A2007B501220DF107018DF8070000201AF082
S214446A30BFFC03B05DF804FB0FB470B5C2B00024CD
S214446A4046AA02AE52F8041B304601920BF064FD8F
S214446A50304608F025FEC5B2E3B29D4204D842B0A3
S214446A60BDE8704004B07047305D0134FFF7D8FF8E
S214446A70F2E708B58E2018F07DF8962018F07AF8DC
S214446A800748FFF7D9FF0749002019F03BFB0120D0
S214446A90054919F037FB0548BDE80840FFF7CCBF69
S214446AA0E08A4600B4A6460088A64600E88A460021
S214446AB00B2938B5044614D142F644030E4D002241
S214446AC00E48EA50FFF7B8FF42F64803EB581BB1AE
S214446AD042F64C02A85898472046BDE8384016F07F
S214446AE04BBA074B1A6832B1002206481A60BDE812
S214446AF03840FFF7A1BF38BDEC4B4120EE8A460034
S214446B002C7441200A8B46000B2938B505460E4C9A
S214446B1013D144F2A47300220C48E250FFF78CFFD2
S214446B2044F2A873E3581BB144F2AC72A058984799
S214446B302846BDE8384016F01FBA44F2A073E2581F
S214446B400AB10022E25038BDEC4B4120298B460066
S214446B500B2938B5044614D146F204730E4D002270
S214446B600E48EA50FFF768FF46F20873EB581BB12D
S214446B7046F20C72A85898472046BDE8384016F0AE
S214446B80FBB9074B1A6832B1002206481A60BDE8C2
S214446B903840FFF751BF38BDEC4B4120458B46008B
S214446BA0ECB24120618B46000B2938B504464FF4BD
S214446BB0FB55134815D105FB040542F64403002251
S214446BC01048EA50FFF738FF42F64803EB581BB12B
S214446BD042F64C02A85898472046BDE8384016F07E
S214446BE0CBB905FB040404F52154236833B10023D0
S214446BF005482360BDE83840FFF71EBF38BD00BFD8
S214446C00EC4B41207F8B46009B8B46000B2938B5C6
S214446C1004464FF4FB55134815D105FB040542F6CC
S214446C20440300221048EA50FFF706FF42F64803A2
S214446C30EB581BB142F64C02A85898472046BDE88C
S214446C40384016F099B905FB040404F5215423682A
S214446C5033B1002305482360BDE83840FFF7ECBE57
S214446C6038BD00BFEC4B4120BA8B4600D68B46005D
S214446C700B2938B504464FF4FB55134815D105FB8C
S214446C80040542F6440300221048EA50FFF7D4FEB7
S214446C9042F64803EB581BB142F64C02A8589847B4
S214446CA02046BDE8384016F067B905FB040404F5F1
S214446CB02154236833B1002305482360BDE8384097
S214446CC0FFF7BABE38BD00BFEC4B4120F58B4600FB
S214446CD0118C460038B50A243C4D294600200FF056
S214446CE0C3FF38B1013C14F0FF04F6D121463848BE
S214446CF0FFF7A2FE0A24374D294601200FF0B4FFC1
S214446D0038B1013C14F0FF04F6D101213048FFF7B6
S214446D1093FE0A24304D294602200FF0A5FF38B1D1
S214446D20013C14F0FF04F6D102212948FFF784FE03
S214446D3000222A49B4200A2417F01BFF00222849BF
S214446D40B52017F016FF00222649B62017F011FF8B
S214446D50B42017F00FFFB52017F00CFFB62017F03D
S214446D6009FF00200FF016FC38B1013C14F0FF0474
S214446D70F7D121461C48FFF75FFE0A2401200FF096
S214446D8009FC38B1013C14F0FF04F7D10121164840
S214446D90FFF752FE0A2402200FF0FCFB38B1013CF8
S214446DA014F0FF04F7D102210F48FFF745FE0121F6
S214446DB000200FF071FC012108460FF06DFC012104
S214446DC00220BDE838400FF067BC00BF509A46002A
S214446DD04C8C4600F4994600989946004572450006
S214446DE04B72450051724500308C460038B51C4CF9
S214446DF00546206804302044FFF7FCFD012801D1F5
S214446E00012038BD2368E21810790A2810D00D28CE
S214446E100ED0082815D123B1013B12482360FFF752
S214446E200BFE2368AB42EBD325440020E87006E013
S214446E300D48FFF701FE23680020234418712060A4
S214446E40DFE7A0F120035E2BEBD8FFF7E9FD2368CC
S214446E50E11801330A792360303A81F80421E0E7E7
S214446E60EC4B4120618C4600708C460010B5802067
S214446E70FFF7BCFF90B90A4C23797BB10949201D22
S214446E8008F004FC20B90848BDE81040FFF7D4BD1C
S214446E90211D0648BDE81040FFF7CEBD10BD00BF1B
S214446EA0EC4B4120658C46006B8C4600738C460048
S214446EB02DE9F04F082389B0002492463B4A054604
S214446EC089464FF064081068EDB2516802AF012657
S214446ED022468DF810408DF81C40DFF8E8B0CDE926
S214446EE005346B4403C35146484620F02CFD04AA9F
S214446EF0214640F255532846CDF8048000978DF835
S214446F001C608DF81040059415F024FF284B04AA05
S214446F102146284602934FF607738DF81060ADF865
S214446F200C300623CDE9007805935B4615F012FF36
S214446F30204A0623214602924FF6FF7205932846BE
S214446F405B46ADF80C2004AA8DF81060CDE90078B5
S214446F5015F000FF184A062321460292284604AA42
S214446F6005935B46ADF80C408DF81060CDE900788B
S214446F7015F0F0FE114B124A214628468DF8106053
S214446F80CDE90232082304AA05935B46CDE900788E
S214446F9015F0E0FE0A20FFF71EFC324651464846EE
S214446FA020F0D1FC09B0BDE8F08F00BFB88246009F
S214446FB01000500010019FFF1002C000710203042D
S214446FC005060708F100DA182DE9F04104460028C2
S214446FD055D16D2017F0CEFD2246C0496D2017F0DE
S214446FE0C8FD6E2017F0C6FD2246BD496E2017F038
S214446FF0C0FD01220821BB4820F0A5FC0122052142
S214447000B84820F0A0FCB84AB849204615F034F9F0
S2144470100121204616F0F2F822460E21204615F0AD
S21444702049FF204616F0C8F82346B14A0E212046AA
S21444703015F060FA2346AF4A0E21204615F09EFA14
S214447040FEF7BFFE2046FFF7A7F9AB4B012242F6F8
S21444705044015A5003F521531A6041F698700023B0
S214447060A64A4443A648A35004441A46013384F827
S21444707071202834C82BF9D10020BDE8F0810128BE
S21444708046D0022840F0898074209E4F17F072FD47
S21444709000229D49742017F06CFD752017F06AFD98
S2144470A000229A49752017F064FD0122042198486D
S2144470B020F049FC01220621964820F044FC002595
S2144470C0954A20469549DFF8B88215F0D5F820460B
S2144470D016F072F805F10E0658F83530904A02203C
S2144470E0F6B223F060430135314615F003FA3A46CA
S2144470F0002331460220503715F040FA0B2DE9D1D3
S2144471007D4B012246F204715A5003F5CE43A3E761
S2144471107120844F17F02EFD00228349712017F00A
S21444712028FD722017F026FD00228049722017F0B1
S21444713020FD22460721774820F005FC22460221FE
S214447140734820F000FC0025794A20467949DFF848
S214447150348215F091F8204616F02EF805F11C06F8
S21444716058F83530744A0120F6B223F060430135AE
S214447170314615F0BFF93A460023314601205037D0
S21444718015F0FCF9042DE9D144F2A4715A4B0122BE
S2144471905A5044F2A0715A505FE7032859D0042845
S2144471A000F0F48005287FF458AF7B20634D17F039
S2144471B0E1FC002262497B2017F0DBFC7C2017F0C0
S2144471C0D9FC00225F497C2017F0D3FC01220E2113
S2144471D0504820F0B8FB01225B48114620F0B3FB30
S2144471E05A4A5B49204615F047F8204615F0E4FF16
S2144471F0012255492046FFF75BFE564A544920462D
S21444720015F03AF8204615F0D7FF2B68524A0E215F
S21444721023F06043204615F06DF900234F4A0E21B3
S214447220204615F0ABF9AB684B4A0F2123F0604378
S214447230204615F05FF90023494A0F21204615F0F1
S2144472409DF94CF224512C4B01225A504CF22051B9
S214447250A1E77720434F17F08DFC00224249772060
S21444726017F087FC782017F085FC00223F497820E9
S21444727017F07FFC012200213D4820F064FB0122E8
S2144472803B4800251146DFF8008120F05CFB394A74
S2144472903949204614F0F0FF204615F08DFF05F1DD
S2144472A00E0658F83530354A0320F6B223F06043CC
S2144472B00135314615F01EF93A460023314603207F
S2144472C0503715F05BF90A2DE9D148F264610A4B50
S2144472D001225A5048F260615DE700BF75E94500F7
S2144472E07BE9450008172940449E460088414020D3
S2144472F054204020BC4F4020EC4B412068AA4020FC
S214447300D88A4020BC634020BDE94500C3E9450017
S2144473100E1729400C172940949D460038384020C3
S214447320742040201C5E40209FE94500A5E94500A6
S214447330EC9D4600E03C402064204020D885460032
S214447340FFE9450005EA450010172940C08246007B
S214447350402A40208C9C4600A4204020BC814020EB
S2144473600C824020BC6D4020DBE94500E1E9450045
S214447370061729403C9D46009033402084204020F8
S21444738048864600A0864600F88546007920294D62
S21444739017F0F0FB00222849792017F0EAFB7A2000
S2144473A017F0E8FB002225497A2017F0E2FB012279
S2144473B00A21234820F0C7FA01220921204820F058
S2144473C0C2FA204A2049204614F056FF204615F0BB
S2144473D0F3FE09221A492046FFF76AFD1B4A1A495A
S2144473E0204614F049FF204615F0E6FE2B68184A5E
S2144473F00E2123F06043204615F07CF80023154AFE
S2144474000E21204615F0BAF8AB68114A0F2123F036
S2144474106043204615F06EF800230F4A0F2120469D
S21444742015F0ACF84AF2C4510C4B01225A504AF2B9
S214447430C051B0E6E8854600EDE94500F3E945006D
S21444744008172940C0824600E82E4020E49C4600A7
S21444745094204020BC7740200C784020EC4B4120C0
S21444746041F69872084B02FB003310B503EB8104D7
S214447470E278A07800EB0220627802EB002213F850
S214447480210000EB022010BDD88A402010B5094BDD
S21444749041F6987404FB0030130A00EB810181F82E
S2144474A0282081F82930130C120E81F82A3081F8EE
S2144474B02B2010BDD88A402013B502AB044603E9FE
S2144474C0060041F69871094A9DF8043001FB0022F3
S2144474D0009903F03F0321F06041FEF791FF2046F8
S2144474E002B0BDE81040FEF757BF00BF008B4020F7
S2144474F0FAF7C4B97047704770477047704770478B
S21444750070477047704770477047074B074A19687B
S21444751058799160197941EA002191819979DB790A
S2144475209173D373704700BFD88A40206087402049
S2144475300E490F4810B54A780B7802F0010443EA26
S2144475400423C2F34104C2F3C10243EA442343EA98
S214447550C2238A7843EA4233CA7843EA42534269AA
S21444756002F060421343436110BD00BFD88A4020F6
S21444757060874020074B08491B7803F003021B0929
S21444758003F0040313430A7C22F0070213430B74EC
S214447590704700BFD88A4020608740200549064B84
S2144475A00A7E1B7822F01F0203F01F0313430B7658
S2144475B0704700BF60874020D88A40200549064B64
S2144475C00A7F1B7822F01F0203F01F0313430B7736
S2144475D0704700BF60874020D88A40200649074B42
S2144475E091F820201B7822F00F0203F00F03134378
S2144475F081F82030704700BF60874020D88A4020FA
S214447600114B124810B55A78997802F003041B7847
S21444761043EA0423C2F3810443EA8423C2F30114F5
S214447620920943EA043343EA823301F00302C1F386
S214447630810143EA0243426A120D43EA814312053A
S2144476401343436210BD00BFD88A40206087402061
S2144476500E4B0F4A5878197841EA0021587911851B
S214447660997801F00F0182F82A10D97882F82B1005
S214447670197941EA002191859979DB7901F00F0166
S21444768082F82F3082F82E10704700BFD88A4020E8
S214447690608740200E4B0F4A5878197841EA0021FB
S2144476A058791186997801F00F0182F83210D9780A
S2144476B082F83310197941EA002191869979DB7969
S2144476C001F00F0182F8373082F83610704700BF59
S2144476D0D88A4020608740200C4B0D4A5878197849
S2144476E041EA002158791187997801F00F0182F810
S2144476F03A10197941EA002191879979DB7901F0AA
S2144477000F0182F83F3082F83E107047D88A4020F6
S214447710608740202D492E4A10B50B78487803F0F0
S2144477207F0343EAC013887843EAC033C87843EA01
S214447730C053106C00F00040034348791364C0F310
S21444774040040B79897982F8443000F001031B0227
S21444775043EA4423C0F3800443EA8423C0F3C004CA
S21444776043EAC423C0F3001443EA0433C0F340148A
S21444777043EA4433C0F38014C00943EA843343EAFB
S214447780C03301F0010043EA0043C1F3400043EA3A
S2144477904043C1F3800043EA8043C1F3C00043EA58
S2144477A0C043C1F3001043EA0053C1F34010C1F391
S2144477B0801143EA405343EA8153516C21F4FF015C
S2144477C021F4FE410B43536410BD00BFD88A4020C9
S2144477D0608740200D4A0E4810B55178137801F062
S2144477E00F04C1F3001143EA042343EA01339178BA
S2144477F043EA4133D17843EA4153816C01F0604116
S2144478000B4383645368C36410BD00BFD88A4020CA
S21444781060874020034A044B1168526819655A65CC
S214447820704700BFD88A402060874020244A2549B4
S21444783070B55578137805F003069078D47843EA03
S2144478400623C5F3810643EA8623C5F30116AD092C
S21444785043EA063343EA8533C0F3011543EA054356
S214447860850900F00F0043EA854304F0030543EA24
S2144478700553C4F3810543EA8553C4F30115A409AB
S21444788043EA056343EA84638C6D04F070442343FF
S21444789054798B651379D27981F85C30230104F0EE
S2144478A0030403F4706343EA0233CA6D43EA0050A8
S2144478B0054B40EA046013401843C86570BD00BFDA
S2144478C0D88A402060874020FF0000FC70B5224DD7
S2144478D0224A2C78E878C4F3401604F00F0329793A
S2144478E043EA0613C4F38016E40943EA461343EA1C
S2144478F084136C7843EAC413AC7843EAC43300F088
S214447900030443EAC453C0F3810443EA4463C0F324
S2144479100114800943EAC46343EA4073106E00F0DE
S2144479200040034301F0030013668B0803F004038E
S2144479300343880800F0080003438808C90900F098
S2144479401000034343EA411392F8641021F03F01C8
S2144479500B4382F8643070BDD88A4020608740204C
S214447960114A124810B55178137801F0030443EADB
S2144479700423C1F3810443EA8423C1F3011489092F
S21444798043EA043343EA8133A0F868305388A0F8C6
S2144479906A309388A0F86C30937980F86E30D37947
S2144479A080F86F3010BD00BFD88A402060874020E2
S2144479B0064B074A1968587911671979DB7941EA01
S2144479C0002182F87630A2F874107047D88A402096
S2144479D060874020084A09491378907881F87830BF
S2144479E053781843D378064A9B0443EA0023886FA7
S2144479F0024013438B677047D88A402060874020F4
S214447A00FF0000FC08B5054B188808F05FFC0449E5
S214447A1008F0B0FC034BD86708BD00BFD88A4020A6
S214447A20CDCCCC3D60874020104B41F69871104A2F
S214447A30595C82F8801041F69B71585C41F69A7105
S214447A40595C41EA0021A2F8811041F69D71585CC8
S214447A5041F69C71595C41EA0021A2F8841041F633
S214447A609F715B5C82F88630704700BFD88A40209E
S214447A7060874020064A41F69871064B5158C3F831
S214447A80881041F69F71525C83F88C20704700BF83
S214447A90D88A4020608740200C4A41F69F730C49A0
S214447AA010B541F69974D05C41F69873D35C125D78
S214447AB002F0010243EA0223D1F89020520C43EA32
S214447AC0402352041343C1F8903010BDD88A402056
S214447AD060874020284941F69973284A70B5C85CA7
S214447AE041F69A73CD5C41F69B7300F00306CC5C7A
S214447AF041F69873CB5C43EA0623C0F3810643EA17
S214447B008623C0F30116800943EA063343EA8033EA
S214447B1005F00300C5F3810543EA004304F003007F
S214447B2043EA854343EA0053C4F38100A40943EA85
S214447B308053D2F8940043EA046300F07C40034345
S214447B4041F69F70C2F8943041F69C73CB5C82F841
S214447B50983041F69D73CB5C095C1B0203F47C535E
S214447B6043EA8133D2F8981021F47F1121F47C51F2
S214447B700B43C2F8983070BDD88A402060874020B6
S214447B80214843F63073214930B5C35A5BBAA1F84D
S214447B909C3043F63373C25C43F63273C2F301152A
S214447BA0C45C930943EA850304F00F05240943EAB9
S214447BB0051343F63675455DED0843EA0523C2F3DF
S214447BC0800543EA4533B1F89E5005F440452B43BF
S214447BD0A1F89E3043F63473C55C43F63573C35CF4
S214447BE043EA0523A1F8A030C2F3C003520143EA96
S214447BF0440302F060021A4391F8A23023F07F0354
S214447C001A4381F8A22030BDD88A4020608740209D
S214447C10164A43F63073164910B5D35A5BBAA1F8E0
S214447C20A43043F63273D05C43F63373D35C43EAF2
S214447C300023A1F8A63043F63673D05C43F634737B
S214447C40D45C43F63573D35C43EA042200F0010364
S214447C50C0F3400043EA4203D1F8A820920C43EA1A
S214447C60404392041343C1F8A83010BDD88A40203C
S214447C7060874020124A43F63071124B515A49BA33
S214447C80A3F8AC1043F63271505C43F63371515C42
S214447C9041EA0021B3F8AE0061F30D0043F63671B5
S214447CA0A3F8AE0043F63770515C125C42EA0122F8
S214447CB0B3F8B01062F30D01A3F8B010704700BFDC
S214447CC0D88A40206087402030B543F63073304C25
S214447CD03049E35A5BBAA1F8B43043F63673E05CF5
S214447CE043F63773E25C43F63273E55C00F0030315
S214447CF043EA8503C0F3800543EA8523C2F380053F
S214447D0043EAC523850943EA0533B1F8B65005F47A
S214447D1040452B43C2F3C005A1F8B63043F633734F
S214447D20E35C81F8B830C0F3C0031B0243EA452342
S214447D3002F0030543EA852343F63475655D43EA5A
S214447D400533C0F30015C0F3401043EA0553C2F3AD
S214447D50001543EA45539509120943EA8553D1F879
S214447D60B85002F0020225F47F05024325F47F450D
S214447D702B43C1F8B83043F63573E35C81F8BB3027
S214447D8091F8BC3023F003031A4381F8BC2030BD7D
S214447D90D88A402060874020F0B543F63273404F7F
S214447DA0404DFE5C43F63473F95C43F63373C6F3D6
S214447DB0801CF85C43F63573FC5C43F63673FA5C19
S214447DC0F30943EA4C0343F6317C42EA042217F8AB
S214447DD00CC043EA8C03C6F3401C43EA8C23C6F328
S214447DE0001C43EACC23C1F3400C43EA0C3343F66D
S214447DF0307C17F80C7043EA4733C6F3C00743EAAF
S214447E004753C6F3800743EA8753C0F3001743EA51
S214447E10C753470943EA0763C4F30117A40943EA6F
S214447E20C763C6F3400706F0010643EA477343EACE
S214447E308673D5F8C06006F00046334301F0010669
S214447E40C5F8C030C2F30903C0F3C00243EA862330
S214447E5043EAC223C0F3800243EA0233C0F340023B
S214447E6000F0010043EA4233C1F3C00243EA8033E0
S214447E7043EAC433C1F3001443EA44438C09C1F3D0
S214447E80800143EA844343EA025343EA4151D5F826
S214447E90C4309B0D9B051943C5F8C410F0BD00BF04
S214447EA0D88A402060874020284843F6307343F6FB
S214447EB036722749F0B5C35A43F63275845C43F6A6
S214447EC035725BBA455D825CA709A1F8C83043F6B3
S214447ED0337347EA820743F63772C65C43F6347315
S214447EE0825CC35CB009B1F8CAC042EA042240EAE4
S214447EF08500C6F3810543EA0623C6F3011640EA25
S214447F008520144DC3F309030CEA050C43EA862383
S214447F1040EA0C0043EA0733A1F8CA00C4F38100E0
S214447F20C4F3011443EA8053D1F8CC0000F07F40F8
S214447F300343C1F8CC30C2F30903B1F8D02043EA76
S214447F40842315402B43A1F8D030F0BDD88A402076
S214447F506087402000F0FFFF1D4943F630731D48FC
S214447F60F0B5CB5A43F632745BBA0E5DA0F8D43003
S214447F7043F63373CA5C43F63573CD5CC2F381046F
S214447F8043F634732F09CB5C44EA870443F63677CA
S214447F9043EA0223C95D41EA052144EA8111A0F877
S214447FA0D610C3F30901C2F3001343EA410391090F
S214447FB0C2F3401243EAC62343EAC16343EA427328
S214447FC0D0F8D82002F040421343C0F8D830F0BD71
S214447FD0D88A40206087402070B5234943F63674DB
S214447FE043F6357543F630730C5D4E5DCB5AA509A2
S214447FF01E485BBA45EA860543F63776A0F8DC3079
S21444800043F633738E5DCA5C43F6347346EA0424FF
S21444801043F63276CB5C8E5D910943EA022341EA0D
S2144480208601C2F38006C3F3090341EA8621B0F809
S214448030DE6006F478463143A0F8DE10C2F3C00191
S21444804043EA8123C2F30011520943EAC52343EAB3
S214448050415343EA8453C0F8E03090F8E43062F386
S214448060000380F8E43070BDD88A40206087402002
S2144480701D4A43F630731D4870B5D35A5BBAA0F810
S214448080E83043F63273D45C43F63473D55C43F637
S2144480903373D15C2B09C5F3C00543EA011143F69B
S2144480A03673D65C43F63573D35CDB0043EA56122C
S2144480B0C4F3400343EA450304F00105A40843EA35
S2144480C0850343EAC403B0F8EA4004F47E442343F9
S2144480D0A0F8EA3041EA0233D0F8EC20D20DD205BB
S2144480E01343C0F8EC3070BDD88A402060874020E7
S2144480F01B4943F631731B4830B5CB5C80F8F030EF
S21444810043F63273CA5C43F63573CD5C43F6347338
S214448110CC5C43F63073C95C93091B0243EA812363
S214448120C2F3401143EA8143C2F38001C2F3C00262
S21444813043EAC143D0F8F01043EA02532A0905F053
S2144481400F0543EA4253084A43EA45630A40134349
S214448150C0F8F030230943EA041480F8F44030BDF4
S214448160D88A402060874020FF0000E0074943F655
S2144481703073074ACB581BBAC2F8003143F63473FF
S214448180CB581BBAC2F80431704700BFD88A402087
S21444819060874020214845F6C863214930B5C35A14
S2144481A05BBAA1F8083145F6CB63C25C45F6CA63B0
S2144481B0C2F30115C45C930943EA850304F00F0532
S2144481C0240943EA051345F6CE65455DED0843EAC2
S2144481D00523C2F3800543EA4533B1F80A5105F452
S2144481E040452B43A1F80A3145F6CC63C55C45F6B9
S2144481F0CD63C35C43EA0523A1F80C31C2F3C00344
S214448200520143EA440302F060021A4391F80E31E5
S21444821023F07F031A4381F80E2130BDD88A4020CC
S21444822060874020164A45F6C863164910B5D35AA7
S2144482305BBAA1F8103145F6CA63D05C45F6CB6309
S214448240D35C43EA0023A1F8123145F6CE63D05CF2
S21444825045F6CC63D45C45F6CD63D35C43EA04224E
S21444826000F00103C0F3400043EA4203D1F814216E
S214448270920C43EA404392041343C1F8143110BDB0
S214448280D88A402060874020F0B545F6CA632D4F13
S2144482902D4CFD5C45F6CC63F95C45F6CB63C5F3E3
S2144482A0801CFE5C45F6CD63F85C45F6CE63FA5C0E
S2144482B0EB0943EA4C0345F6C96C42EA002217F838
S2144482C00CC0C2F3090243EA8C03C5F3401C43EADC
S2144482D08C23C5F3001C43EACC23C1F3400C43EA89
S2144482E00C3345F6C86C17F80C7043EA4733C6F3AC
S2144482F00017760943EA475343EA8653C0F3011608
S214448300800943EA4663C5F3400605F0010543EA9F
S214448310C66343EA0573D4F8245105F060452B43FD
S214448320C4F8243101F0010342EA832242EAC02021
S214448330C1F30012890940EA423040EA8131A4F888
S2144483402811F0BDD88A402060874020284845F64A
S214448350C86345F6CE622749F0B5C35A45F6CA65A2
S214448360845C45F6CD625BBA455D825CA709A1F89C
S2144483702C3145F6CB6347EA820745F6CF62C65CA6
S21444838045F6CC63825CC35CB009B1F82EC142EAC0
S214448390042240EA8500C6F3810543EA0623C6F371
S2144483A0011640EA8520144DC3F309030CEA050C74
S2144483B043EA862340EA0C0043EA0733A1F82E0139
S2144483C0C4F38100C4F3011443EA8053D1F8300166
S2144483D000F07F400343C1F83031C2F30903B1F8DB
S2144483E0342143EA842315402B43A1F83431F0BDAD
S2144483F0D88A40206087402000F0FFFF1D4945F69C
S214448400C8631D48F0B5CB5A45F6CA645BBA0E5DE0
S214448410A0F8383145F6CB63CA5C45F6CD63CD5CEF
S214448420C2F3810445F6CC632F09CB5C44EA870447
S21444843045F6CE6743EA0223C95D41EA052144EA8C
S2144484408111A0F83A11C3F30901C2F3001343EAB9
S21444845041039109C2F3401243EAC62343EAC143A7
S21444846043EA4253D0F83C21920D92051343C0F898
S2144484703C31F0BDD88A402060874020184845F6F5
S214448480C863184930B5C35A5BBAA1F8403145F6BB
S214448490CC63C55C45F6CA63C45C45F6CB63C35C33
S2144484A043EA042245F6CD63E409C35CB1F84201CD
S2144484B043EA0523ED09C3F3090343EA85230A4D3A
S2144484C028400343A1F84231C2F30903B1F84421DA
S2144484D043EA84232A401343A1F8443130BD00BF05
S2144484E0D88A40206087402000F8FFFF1D4A45F6A2
S2144484F0C8631D4870B5D35A5BBAA0F8483145F6F0
S214448500CA63D45C45F6CC63D55C45F6CB63D15C94
S2144485102B09C5F3C00543EA011145F6CE63D65C84
S21444852045F6CD63D35CDB0043EA5612C4F34003FE
S21444853043EA450304F00105A40843EA850343EAF5
S214448540C403B0F84A4104F47E442343A0F84A31B5
S21444855041EA0233D0F84C21D20DD2051343C0F879
S2144485604C3170BDD88A4020608740201B4945F670
S214448570C9631B4830B5CB5C80F8503145F6CA63B6
S214448580CA5C45F6CD63CD5C45F6CC63CC5C45F61B
S214448590C863C95C93091B0243EA8123C2F3800182
S2144485A043EA8143C2F3C001C2F3401243EAC143E3
S2144485B0D0F8501143EA02532A0905F00F0543EA5E
S2144485C04253084A43EA45630A401343C0F85031CD
S2144485D0230943EA041480F8544130BDD88A402025
S2144485E060874020FF0000E030B545F6C863304C55
S2144485F03049E35A5BBAA1F8183145F6CE63E05CDD
S21444860045F6CF63E25C45F6CA63E55C00F00303D7
S21444861043EA8503C0F3800543EA8523C2F3800515
S21444862043EAC523850943EA0533B1F81A5105F4EC
S21444863040452B43C2F3C005A1F81A3145F6CB6337
S214448640E35C81F81C31C0F3C0031B0243EA4523B4
S21444865002F0030543EA852345F6CC65655D43EAA7
S2144486600533C0F30015C0F3401043EA0553C2F384
S214448670001543EA45539509120943EA8553D1F850
S2144486801C5102F0020225F47F05024325F47F457F
S2144486902B43C1F81C3145F6CD63E35C81F81F31AA
S2144486A091F8203123F003031A4381F8202130BD8A
S2144486B0D88A402060874020074945F6C863074A61
S2144486C0CB581BBAC2F8603145F6CC63CB581BBABC
S2144486D0C2F86431704700BFD88A40206087402083
S2144486E00C4947F664630C48CA5C47F66563CB5C42
S2144486F043EA022247F66263CB5C03F00F0343EA85
S2144487000213D0F86821120D12051343C0F86831DD
S214448710704700BFD88A402060874020064A47F604
S2144487206263D15C47F66363D35C044A43EA01233D
S214448730A2F86C31704700BFD88A4020608740203A
S2144487400C4949F6FC530C48CA5C49F6FD53CB5CCD
S21444875043EA022249F6FA53CB5C03F00F0343EA9A
S2144487600213D0F87021120D12051343C0F870316D
S214448770704700BFD88A402060874020064A49F6A2
S214448780FA53D15C49F6FB53D35C044A43EA0123CB
S214448790A2F87431704700BFD88A402060874020D2
S2144487A010B51B4C208907F091FD1A4907F0E2FDED
S2144487B0194BA27B1860194B60891A6007F086FD36
S2144487C0174907F0D7FD174907F0CAFC07F024F904
S2144487D00DA3D3E9002306F0BFFF07F06DFC124B50
S2144487E0124A1860E37BA08903F00F03136007F076
S2144487F06DFD0F4907F0BEFD0E4907F0B1FC0E4B68
S214448800186010BDAFF30080C3F5285C8FC2D53F17
S21444881060874020CDCCCC3DA01F4020881F402000
S2144488200AD7A33C00C02344941F4020841F402002
S214448830ACC52737ACC5A73E8C1F4020124A134907
S214448840137D03F003000860C3F3830010499B09BB
S214448850086010490B60537D0F49C3F3410008601C
S214448860C3F3C1000D4903F0010308700C490B60C3
S21444887053690C49C3F347330B60D38A0A4AC3F39C
S21444888047131360704700BF60874020741F402022
S214448890701F40206C1F4020641F4020601F4020F3
S2144488A0681F4020541F40205C1F4020074B084A46
S2144488B01B7CC3F300011170C3F34001054AC3F3A4
S2144488C080031170044A1370704700BF60874020CD
S2144488D0521F4020511F4020501F4020FFF7E6BF44
S2144488E008B5FFF7E3FFBDE80840F8F7C5BF174AE9
S2144488F0174992F8243003F003000860C3F381005C
S21444890014490860C3F3011013499B0908601349CE
S2144489100B6092F82530124903F003000860C3F355
S214448920810010490860C3F301100F499B09086091
S2144489300E490B6092F826300D4A03F00301C3F348
S214448940810311600B4A1360704700BF6087402064
S2144489507C1A4020781A4020741A4020701A40200E
S2144489606C1A4020681A4020641A4020601A40203E
S2144489705C1A4020581A402010B5194C208D07F038
S214448980A5FC184907F0F6FC174907F0E9FB174B16
S214448990174A186094F82A30A08D03F00F011B097B
S2144489A01160144A136094F82B30134A323B136018
S2144489B007F08CFC114907F0DDFC114907F0D0FBA9
S2144489C0104B114A186094F82E3003F00F011B091F
S2144489D011600E4A136094F82F200D4B1A6010BD98
S2144489E0608740200AD7A33B0AD723434C1F402026
S2144489F0481F4020441F4020401F40200AD7A33A27
S214448A00F8D323423C1F4020381F4020341F4020C8
S214448A10301F402010B5194C208E07F057FC1849DB
S214448A2007F0A8FC174907F09BFB174B174A18603A
S214448A3094F83230A08E03F00F011B091160144ADB
S214448A40136094F83320134B1A6007F03FFC124926
S214448A5007F090FC114907F083FB114B114A18604C
S214448A6094F8363003F00F011B0911600E4A136068
S214448A7094F837200D4B1A6010BD00BF6087402025
S214448A800AD7A33B0AD723432C1F4020281F402045
S214448A90241F4020201F40200AD7A33AF8D323425D
S214448AA01C1F4020181F4020141F4020101F402029
S214448AB010B5174C208F07F009FC164907F05AFCEE
S214448AC0154907F04DFB154B154A186094F83A3093
S214448AD0A08F03F00F011B091160124A136007F0C0
S214448AE0F5FB114907F046FC104907F039FB104BDB
S214448AF0104A186094F83E3003F00F011B091160C9
S214448B000D4A136094F83F200C4B1A6010BD00BF0A
S214448B10608740200AD7A33B0AD723430C1F402034
S214448B20081F4020041F40200AD7A33AF8D3234204
S214448B30001F4020FC1E4020F81E4020F41E40200B
S214448B4010B53E4C3E4A94F84030B4F8400003F02A
S214448B500101C0F3C7101160C3F34001394A1160E4
S214448B60C3F38201384AC3F341131160374A136092
S214448B7007F0ACFB364907F0FDFB07F0C1FD354B6B
S214448B801860206CC0F3C73007F0A0FB304907F0EC
S214448B90F1FB07F0B5FD304B1860B4F84200C0F363
S214448BA0C71007F093FB2D4907F0DAFA07F0A8FD43
S214448BB02B4B94F8442018602A4B1A6094F845309E
S214448BC0294A03F001011160C3F34001274A1160AA
S214448BD0C3F38001264A1160C3F3C001254A1160DD
S214448BE0C3F30011244A1160C3F34011234A1160B1
S214448BF0C3F38011224ADB091160224A136094F8B9
S214448C004630214A03F001011160C3F340011F4A74
S214448C101160C3F380011E4A1160C3F3C0011D4AAC
S214448C201160C3F300111C4A1160C3F340111B4A80
S214448C30C3F3801311601A4A136010BD6087402046
S214448C40F01E4020EC1E4020E81E4020E41E40203B
S214448C500AD7233CE01E4020DC1E40200000204271
S214448C60D81E4020D41E4020D01E4020CC1E40207B
S214448C70C81E4020C41E4020C01E4020BC1E4020AB
S214448C80B81E4020B41E4020B01E4020AC1E4020DB
S214448C90A81E4020A41E4020A01E40209C1E40200B
S214448CA0981E402038B5264D264B95F8484004F08B
S214448CB00102C4F302101A60C4F34002224B1A6045
S214448CC0C4F38002214B1A60C4F3C002204BE4096B
S214448CD01A6007F0F7FA1F4B1F4A18601F4BA86C20
S214448CE01C6095F84930C0F3473003F00F01C3F3D6
S214448CF00013323811601A4A136007F0E7FA194B2A
S214448D001860B5F84A00C0F34710323807F0DEFA68
S214448D10154B1860B5F84C00A0F5004007F0D6FA9D
S214448D20124B1860B5F84E0007F0D0FA104907F019
S214448D3021FB104907F014FA0F4B186038BD00BFEA
S214448D4060874020941E4020901E40208C1E402069
S214448D50881E4020841E40207C1E4020801E4020CA
S214448D60781E4020741E4020701E40206C1E4020FA
S214448D700AD7233C00004843681E40207047304BC7
S214448D80304A10B593F85940C4F381011170C4F3C6
S214448D9001112D4A1170C4F301012C4AA409117023
S214448DA093F858202A49C2F381100870C2F3011080
S214448DB028490870C2F381002749C2F301020870AB
S214448DC026490A7093F85D202549C2F38100C2F310
S214448DD00102087023490A7093F85E202249C2F3C0
S214448DE003120A7093F85F202049C2F301020A7006
S214448DF093F85A201E4902F003000860C2F381002B
S214448E001C490860C2F301101B49920908601B49BB
S214448E100A6093F85B201A4902F00300C2F3810209
S214448E200860184993F85C000A7007F04FFA164930
S214448E3007F0A0FA154B1860154B1C6010BD00BF18
S214448E4060874020641E4020631E4020621E4020EF
S214448E50611E4020601E40205F1E40205E1E402053
S214448E605D1E40205C1E402070184020241E40207A
S214448E70541E4020501E40204C1E4020481E402079
S214448E80441E402069184020CDCCCC3D3C1E40209A
S214448E90581E4020264A274992F8603003F00700BF
S214448EA00860C3F3C00024490860C3F30010234994
S214448EB00870C3F340102249C3F380130870214955
S214448EC00B70B2F860302049C3F3C7130B60136EBF
S214448ED01E49C3F3C7330B60B2F862301C49C3F370
S214448EE0C1130B6092F863301A49C3F3410008601B
S214448EF0C3F3C1001849C3F34113086017490B6014
S214448F0092F86430164A03F003011160C3F38001FB
S214448F10144A1160C3F3C001134A1160C3F300112D
S214448F20124AC3F340131160114A1360704700BFDE
S214448F3060874020201E40201C1E40201A1E4020D1
S214448F40191E4020181E4020141E4020101E40208B
S214448F500C1E4020081E4020041E4020001E4020B8
S214448F60FC1D4020F81D4020F41D4020F01D4020EC
S214448F70EC1D402010B5194C194A94F8683094F802
S214448F806A00C3F38101C3F301131170154A1370C9
S214448F9094F86930144AC3F301011170C3F3810194
S214448FA0124AC3F381131170114A137007F08AF9F9
S214448FB0104B186094F86B0007F084F90E4B94F845
S214448FC06C2018600D4B1A7094F86D200C4B1A7078
S214448FD094F86E200B4B1A7010BD00BF608740207B
S214448FE0E21D4020D11D4020E11D4020D01D4020E0
S214448FF0E01D4020DC1D4020D81D4020D41D4020CC
S214449000D31D4020D21D402010B50C4CB4F872003D
S21444901007F05CF90A4907F0ADF90A4B1860B4F852
S214449020700007F053F9064907F0A4F9064BB4F864
S21444903074201860054B1A8010BD00BF608740201E
S214449040CDCCCC3DCC1D4020C81D4020C61D402064
S214449050084B0949B3F87A20C2F387020A709A6F1C
S2144490600649C2F309220A8093F87820044B1A7002
S214449070704700BF60874020C41D4020C21D40206A
S214449080C01D402010B5124C124B94F88020B4F802
S21444909081001A6007F01AF90F4907F06BF90F4977
S2144490A007F05EF80E4B1860B4F8840007F00EF92B
S2144490B00C4907F05FF90C4B0C4A186094F886305C
S2144490C003F00F011B091160094A136010BD00BF6D
S2144490D060874020BC1D4020ACC52737ACC5A73EA2
S2144490E0B81D4020CDCCCC3DB41D4020B01D402002
S2144490F0AC1D402010B5114CB4F8880007F0E6F8D3
S2144491000F4907F037F90F4907F02AF80E4B186055
S214449110B4F88A0007F0DAF8094907F02BF9094948
S21444912007F01EF8094B0A4A186094F88C3003F08E
S2144491300F011B091160074A136010BD6087402069
S2144491400AD7A33C00C02344A81D4020A41D4020A9
S214449150A01D40209C1D4020114A124992F8903090
S21444916003F003000860C3F381000F490860C3F3AB
S21444917001100E499B0908600D490B6092F8913026
S2144491800C4903F00100C3F3430308600A490B602B
S214449190D2F89030094AC3F343331360704700BF94
S2144491A060874020981D4020941D4020901D4020FC
S2144491B08C1D4020881D4020841D4020801D40205A
S2144491C0194A1A4992F8943003F003000860C3F32E
S2144491D0810017490860C3F3011016499B090860CB
S2144491E015490B6092F89530144903F00300086063
S2144491F0C3F3810012490860C3F3011011499B0967
S214449200086011490B6092F89630104903F0030049
S214449210C3F3810308600E490B60D2F898300D4AB8
S214449220C3F3833313607047608740207C1D40201F
S214449230781D4020741D4020701D40206C1D402029
S214449240681D4020641D4020601D40205C1D402059
S214449250581D4020541D402010B50E4C0E4B94F81B
S2144492609F0094F89C2000F01F001A6000EB8000DA
S21444927007F02CF8094B1860B4F8A00007F026F85D
S214449280074907F077F8074906F06AFF064B186067
S21444929010BD00BF60874020501D4020381D402030
S2144492A0CDCC4C3D00C0CC44341D402010B50C4CB5
S2144492B0B4F8A60007F00AF80A4907F05BF80A492A
S2144492C006F04EFF094B1860D4F8A800C0F34F00D0
S2144492D0A0F5FF407F3806F0F9FF054B186010BD37
S2144492E0608740200AD7A33C00C02344241D402066
S2144492F01C1D402010B50D4CB4F8AE00C0F30D0054
S21444930006F0E4FF4FF07A5107F034F8084B186043
S214449310B4F8B000C0F30D0006F0D8FF4FF07A5111
S21444932007F028F8034B186010BD00BF6087402044
S214449330141D4020101D402070470B4A0B49B2F8BC
S214449340C40008B5B2F8C030C0F30900C3F38703BD
S2144493500B7006F0BBFF064907F00CF8054906F00B
S214449360FFFE054B186008BD608740200C1D40205A
S214449370CDCCCC3D9A994C42081D402010B5174C94
S214449380B4F8CA00C0F3090006F0A0FF144906F07A
S214449390F1FF144B1860B4F8CC00C0F3090006F093
S2144493A095FF0F4906F0E6FF0F4B1860D4F8CC0043
S2144493B0C0F3093006F08AFF094906F0DBFF0B4B81
S2144493C01860B4F8D000C0F3090006F07FFF0449E3
S2144493D006F0D0FF064B186010BD00BF60874020E3
S2144493E0CDCCCC3D041D4020001D4020FC1C40201C
S2144493F0F81C402038B5154DB5F8D600800906F05F
S21444940065FF134906F0B6FF124906F0A9FEB5F803
S214449410D840114BC4F349041860204606F056FF62
S2144494200E4906F0A7FF0E4B1860D5F8D800C0F3D7
S214449430CF2006F04BFF0B4906F09CFF0A4B186002
S2144494400A4B1C600A4B1C6038BD00BF6087402036
S214449450CDCC4C3D66667241F41C40209A99193E28
S214449460F01C40200AD7233CEC1C4020781C4020AB
S214449470181B402010B5164CB4F8DE00C0F30900A3
S21444948006F024FF134906F075FF134B1860B4F832
S214449490E000C0F3090006F019FF0E4906F06AFF23
S2144494A00E4B1860D4F8E000C0F3C92006F00EFF57
S2144494B0084906F05FFF0A4B1860B4F8E2008009DA
S2144494C006F004FF034906F055FF064B186010BD2E
S2144494D0608740209A99193EE81C4020E41C4020AE
S2144494E0E01C4020DC1C402010B5134CB4F8EA00C5
S2144494F0C0F3C50006F0EAFE104906F03BFF1049EB
S21444950006F02EFE0F4B1860B4F8EC00C0F30B00C8
S21444951006F0DCFE0C4906F02DFF0C4B1860D4F820
S214449520EC00C0F30A3006F0D1FE044906F022FFF0
S214449530074B186010BD00BF60874020CDCCCC3DA3
S214449540CDCC4C40D81C40200AD7233CD41C4020C9
S214449550D01C40207047704710B50E4C0E4B94F804
S2144495600B0194F8082100F01F001A6000EB8000FD
S21444957006F0ACFE094B1860B4F80C0106F0A6FEE3
S214449580074906F0F7FE074906F0EAFD064B186061
S21444959010BD00BF60874020CC1C4020C81C402023
S2144495A0CDCC4C3D00C0CC44C41C402010B50C4C23
S2144495B0B4F8120106F08AFE0A4906F0DBFE0A49B0
S2144495C006F0CEFD094B1860D4F81401C0F34F00E2
S2144495D0A0F5FF407F3806F079FE054B186010BDB5
S2144495E0608740200AD7A33C00C02344C01C4020C8
S2144495F0BC1C402070470B4A0B49B2F8280108B5FA
S214449600B2F82431C0F30900C3F387030B7006F0A5
S2144496105DFE064906F0AEFE054906F0A1FD054B83
S214449620186008BD60874020981C4020CDCCCC3DB7
S2144496309A994C42941C402010B5174CB4F82E010D
S214449640C0F3090006F042FE144906F093FE144B9C
S2144496501860B4F83001C0F3090006F037FE0F492D
S21444966006F088FE0F4B1860D4F83001C0F309307A
S21444967006F02CFE094906F07DFE0B4B1860B4F844
S2144496803401C0F3090006F021FE044906F072FED8
S214449690064B186010BD00BF60874020CDCCCC3D43
S2144496A0901C40208C1C4020881C4020841C402059
S2144496B010B5134CB4F83A01800906F007FE114978
S2144496C006F058FE104906F04BFD104B1860B4F8EF
S2144496D03C01C0F3490006F0F9FD0D4906F04AFE88
S2144496E007F00EF80B4B1860D4F83C01C0F3C720C3
S2144496F006F0ECFD084906F03DFE084B186010BD28
S21444970060874020CDCC4C3D66667241B81C4020F4
S2144497109A99193EB01C40200AD7233CB41C4020DA
S21444972010B50C4CB4F84201C0F3090006F0CEFD67
S214449730094906F01FFE094B1860B4F84401C0F30B
S214449740090006F0C3FD044906F014FE044B1860F5
S21444975010BD00BF608740209A99193EAC1C40203B
S214449760A81C402008B5FFF71BF8FFF767F8FFF77B
S214449770BEF8FFF7E5F9FFF795FAFFF700FBFFF7AA
S21444978089FBFFF7F7FBFFF73FFCFFF761FCFFF7AA
S214449790F3F8FFF73FF9FFF78BF9FFF773FCFFF792
S2144497A0A9FCFFF7D9FCFFF70BFDFFF7E7FDFFF732
S2144497B021FEFFF75FFEFFF73FFFFFF779FFBDE8A7
S2144497C00840FFF7ADBF10B5124CB4F84A01C0F3D9
S2144497D0C50006F07BFD104906F0CCFD0F4906F0A7
S2144497E0BFFC0F4B1860B4F84C01C0F30B0006F0F6
S2144497F06DFD0C4906F0BEFD0B4B1860D4F84C01C9
S214449800C0F30A3006F062FD034906F0B3FD074B89
S214449810186010BD60874020CDCCCC3DCDCC4C40AC
S214449820A41C40200AD7233CA01C40209C1C40205B
S21444983008B5FFF759FEBDE80840FFF7C4BF7047B8
S214449840704708B5084BD3F86801C0F30F1006F00C
S2144498503DFD064906F08EFD054906F081FC06F0FE
S2144498604FFF044B186008BD60874020CDCC4C3D6C
S21444987000C0CC44C01B402008B5084BB3F86C016C
S21444988006F024FD064906F075FD064906F068FC18
S21444989006F036FF044B186008BD00BF60874020C2
S2144498A00AD7A33C00C02344C41B402008B5094B38
S2144498B0D3F87001C0F30F1006F008FD064906F011
S2144498C059FD064906F04CFC06F01AFF044B186096
S2144498D008BD00BF60874020CDCC4C3D00C0CC4482
S2144498E0B41B402008B5084BB3F8740106F0EEFCF0
S2144498F0064906F03FFD064906F032FC06F000FF36
S214449900044B186008BD00BF608740200AD7A33CBC
S21444991000C02344B41B402008B5FFF79DFCFFF766
S214449920C5FCFFF7E7FCFFF708FDFFF715FEFFF75A
S2144499303DFEFFF760FEFFF784FFFFF79DFFFFF74E
S214449940B5FFBDE80840FFF7CDBF1A4B186810B501
S214449950C830194C06F0B6FC184906F0BFFD06F0B0
S2144499605BF80BF061F806F087FB154B1549A4F835
S2144499707801186806F0F6FB134906F0AFFD06F0CA
S2144499804BF80BF051F806F077FB104BA4F87A012D
S2144499901B68A4F87C310E4B186806F03DF80BF0B3
S2144499A043F806F069FB0B4B84F87E011B6884F889
S2144499B07F3110BD801C402060874020CDCCCC3DFC
S2144499C07C1C402000C023440AD7A33C781C40207B
S2144499D0741C4020701C4020324B334A10B5334C24
S2144499E01B78126884F88431314B1202D4F88411FF
S2144499F01B6802F440729B0203F4806313432D4AAF
S214449A001268D20202F4C05213432B4A126852031D
S214449A1002F4C0421343294A1268D20302F4C03205
S214449A201343274A1268520402F460221343254A19
S214449A30127802F0010243EA0253234A127802F0F3
S214449A40030243EA4253214A127802F0070243EAE9
S214449A5002631F4A0A401F491343C4F884311E4B0D
S214449A60186806F07FFB1D4906F038FD05F0D4FF64
S214449A700AF0DAFF06F000FB194BA4F88A011868CE
S214449A8006F020FC134906F06DFB144906F026FD4B
S214449A9005F0C2FF0AF0C8FF06F0EEFAA4F8880103
S214449AA010BD00BFD21D4020601C4020608740206F
S214449AB05C1C4020581C4020541C4020501C402015
S214449AC0201E40201A1E4020F91A4020F81A402032
S214449AD0FF0080F8ACC5A73E4C1C4020ACC52737D9
S214449AE0481C4020184B1949186810B506F0F6FC77
S214449AF0174C05F091FF0AF097FF06F0BDFA154B98
S214449B001249A4F88C01186806F0E8FC05F084FFB6
S214449B100AF08AFF06F0B0FA0F4B0C49A4F88E01FF
S214449B20186806F0DBFC05F077FF0AF07DFF06F0C8
S214449B30A3FA0A4BA4F890011B7884F89331084B97
S214449B401B7884F8923110BDC81D4020CDCCCC3D46
S214449B5060874020CC1D40203C1E4020C41D402031
S214449B60C01D4020174B184A1B7812785B0002F041
S214449B70010203F002031343144A1278920002F0DF
S214449B8004021343124A1278D20002F00802134326
S214449B90104A1278120102F0100213430E4A127849
S214449BA0520102F0200213430C4A1278920102F04A
S214449BB0400213430A4A127843EAC213094A82F817
S214449BC0E4317047251C4020261C4020241C40209D
S214449BD0231C4020221C4020211C4020201C4020C6
S214449BE07E1740206087402038B5254B254D1968A0
S214449BF0254B186806F0B6FA244B044624491868E0
S214449C0006F0B0FA234906F069FC05F005FF0AF0B1
S214449C100BFF06F031FA204B2049A5F8E8011868F6
S214449C2006F0A0FA1E4906F059FC05F0F5FE0AF0C7
S214449C30FBFE06F021FA1B49A5F8EA01204606F089
S214449C404DFC05F0E9FE0AF0EFFE06F015FA164B59
S214449C50A5F8EC01188806F039FB144906F03EFCDA
S214449C6005F0DAFE0AF0E0FE114B1C7806F004FA22
S214449C70C0F30D00A4030443A5F8EE4138BD00BF6D
S214449C80A017402060874020A01F4020A4174020F3
S214449C90000048430AD7233C9C17402000C0234476
S214449CA00AD7A33CCDCCCC3D7C174020CDCC4C3EF3
S214449CB07A1740201C4B1D49186810B506F00EFC58
S214449CC01B4C05F0A9FE0AF0AFFE06F0D5F9194B79
S214449CD0A4F89401186805F09FFE0AF0A5FE06F065
S214449CE0CBF9154B1549A4F89601186806F03AFACC
S214449CF0134906F0F3FB05F08FFE0AF095FE06F0D6
S214449D00BBF9104B1049A4F89801186806F02AFAD3
S214449D100E4906F0E3FB05F07FFE0AF085FE06F0EA
S214449D20ABF9A4F89A0110BD981F4020CDCCCC3D89
S214449D3060874020B8194020A418402000C023441F
S214449D400AD7A33C581B4020000048430AD7233C6C
S214449D50114B1249186810B506F0C0FB104C05F0BC
S214449D605BFE0AF061FE06F087F90E4B0E491B783F
S214449D70A4F89C01A4F89E310C4B186806F0F2F93E
S214449D800B4906F0ABFB05F047FE0AF04DFE06F025
S214449D9073F9A4F8A00110BD08194020CDCCCC3DE1
S214449DA0608740201219402000C023448C1840206D
S214449DB00AD7A33C184B1949186810B506F0D2F9CF
S214449DC0174906F08BFB174C05F026FE0AF02CFECE
S214449DD006F052F9144B1549A4F8A401186806F085
S214449DE0C1F9134906F07AFB05F016FE0AF01CFE8C
S214449DF006F042F90F4BA4F8A6011B6884F8A83174
S214449E000D4B1A680D4B1B6803F00F0343EA02130D
S214449E1084F8A93110BD00BF241D402000C023444F
S214449E200AD7A33C60874020341D402000C0CC4461
S214449E30CDCC4C3D281C4020D81B4020DC1B402069
S214449E40164B1749186810B506F08CF9154906F0F4
S214449E5045FB154C05F0E0FD0AF0E6FD06F00CF96E
S214449E60124B1349A4F8AC01186806F07BF9114963
S214449E7006F034FB05F0D0FD0AF0D6FD06F0FCF8FB
S214449E800D4BA4F8AE011A680C4B1B6803F00F0385
S214449E9043EA021384F8B03110BD00BFC01C402012
S214449EA000C023440AD7A33C60874020C41C4020FB
S214449EB000C0CC44CDCC4C3DC81B4020CC1B4020DD
S214449EC0174B186810B500F28F20164C06F0FAF9B6
S214449ED0154906F003FB05F09FFD0AF0A5FD06F0C4
S214449EE0CBF8124BA4F8B401186800F2666006F08A
S214449EF0E9F90F4906F0F2FA05F08EFD0AF094FDF2
S214449F0006F0BAF80B4BA4F8B6011A680A4B1B685D
S214449F1003F00F0343EA021384F8B83110BD00BFC0
S214449F20C41B4020608740200AD7A33CC01B402067
S214449F30CDCC4C3DB81B4020BC1B4020174B18686A
S214449F4010B500F28F20164C06F0BCF9154906F001
S214449F50C5FA05F061FD0AF067FD06F08DF8124B70
S214449F60A4F8BC01186800F2666006F0ABF90F4925
S214449F7006F0B4FA05F050FD0AF056FD06F07CF8FB
S214449F800B4BA4F8BE011A680A4B1B6803F00F0378
S214449F9043EA021384F8C03110BD00BFB41B40200E
S214449FA0608740200AD7A33CB01B4020CDCC4C3D14
S214449FB0A81B4020AC1B40200A4A0B4B126883F86F
S214449FC0DC210A4A126883F8DD21094A126883F8BC
S214449FD0DE21084A126883F8DF21074A1268C3F86C
S214449FE0E0217047A41B402060874020A01B4020EF
S214449FF09C1B4020981B4020941B40202B4B2C49F4
S21444A00030B51D782B4B05F003051C782A4B04F01D
S21444A01003041878294B00F003001B8881F8C831E4
S21444A020274B1A68274B92001B6802F00C0203F079
S21444A03003031A43244B1B681B0103F030031A43E3
S21444A040224B1B689B01DBB21A43214B1B681B0245
S21444A05003F440731A431F4B1B689B0203F440638C
S21444A0601A431D4B1B681B0303F440531A431B4BF4
S21444A0701B689B039BB21A43194B1B681B0403F4CF
S21444A08040331A43174B1B689B0403F44023134383
S21444A090D1F8C42143EA055302F07C4243EA845390
S21444A0A043EA00631343C1F8C43130BD261B402045
S21444A0B060874020271B4020281B4020241B40202C
S21444A0C08C1B4020901B4020881B4020841B402033
S21444A0D0801B40207C1B4020781B4020741B402063
S21444A0E0701B40206C1B4020124B13491B7803F016
S21444A0F00302124B1B7803F0030343EA8203104A1D
S21444A100127802F0030243EA02130E4A127802F06F
S21444A110030243EA82130C4A127802F0030243EA2B
S21444A1200223B1F8CC2102F47C421343A1F8CC318B
S21444A130704700BF671B402060874020681B402054
S21444A140661B4020651B4020641B4020094B0A497F
S21444A1501A680A4B02F001021B6803F0030343EA41
S21444A160820391F8D82122F00702134381F8D831AC
S21444A170704700BF5C1B402060874020601B402027
S21444A18038B5344B344D1868C83006F09BF833491C
S21444A19006F0A4F905F040FC0AF046FC304B1C6877
S21444A1A0304B64001B6804F0020403F001031C43B4
S21444A1B02D4B1B689B0003F004031C432B4B1B686E
S21444A1C0DB0003F008031C43294B1B681B01DBB26E
S21444A1D01C43284B1B681B0203F440731C43264B4A
S21444A1E01B689B0203F4E0531C43244B1B685B032D
S21444A1F003F4C0431C4305F03FFF214B214903EAC7
S21444A200C0331C43D5F8D03103F000431C431E4BE7
S21444A210C5F8D041186805F0A5FF104906F05EF968
S21444A22005F0FAFB0AF000FC05F026FF174B15492B
S21444A230A5F8D401186805F095FF084906F04EF9CC
S21444A24005F0EAFB0AF0F0FB05F016FFA5F8D60188
S21444A25038BD00BF301B4020608740200AD7233CCF
S21444A2604C1B4020501B4020481B4020441B402091
S21444A270401B40203C1B4020381B4020341B4020C1
S21444A2800080FF7F000048432C1B4020581B402082
S21444A290274B2849186810B505F064FF264906F090
S21444A2A01DF9264C05F0B8FB0AF0BEFB05F0E4FEAB
S21444A2B0234B2449A4F84402186805F053FF224966
S21444A2C006F00CF905F0A8FB0AF0AEFB05F0D4FE48
S21444A2D01E4BA4F846021B68A4F848321C4B1A6866
S21444A2E01C4B02F003021B6803F0010343EA4203DB
S21444A2F0194A126802F0030243EAC203174A126874
S21444A30002F0010243EA4213154A126802F00F02B1
S21444A31043EA8213134A126802F00F0243EA822386
S21444A320B4F84A2202F440421343A4F84A3210BD19
S21444A330681E4020000048430AD7233C60874020DC
S21444A340241D402000C023440AD7A33C181B4020A9
S21444A350581C4020101B4020501C4020041B40200A
S21444A360001B4020FC1A4020234B4FF08E4110B572
S21444A3701B78224C03F00302214B1B7803F00303A3
S21444A38043EA82031F4A127802F0070243EA0213A2
S21444A3901D4A126802F00F0243EAC2131B4A1268AF
S21444A3A002F0010243EAC223194A126802F0030289
S21444A3B043EA0233174A126843EA8233A4F84C321B
S21444A3C0154B1B6884F84E32144B186805F0CAFEC9
S21444A3D005F022FB0AF028FB05F04EFE104BA4F8CD
S21444A3E050021A680F4B1B6803F00F0343EA02132C
S21444A3F084F8523210BD00BFF91A402060874020CE
S21444A400FA1A4020F81A4020F41A4020F01A402045
S21444A410541C4020E81A4020141E40206C1E402045
S21444A420E01A4020E41A4020144B10B5186805F092
S21444A430F3FA134C0AF0F8FA05F01EFE114B84F8B2
S21444A44054021B6884F855320F4B1B68A4F85632E6
S21444A4500E4B186805F0E0FA0AF0E6FA05F00CFE32
S21444A4600B4BA4F858021A680A4B1B6803F00F03F8
S21444A47043EA021384F85A3210BD00BF741C4020CD
S21444A48060874020701C4020481C40204C1C4020C4
S21444A490C81A4020CC1A40201C4A936CC3F3473356
S21444A4A082F88C32B2F84A30C3F3471382F88D32BE
S21444A4B0B2F84230C3F3C71382F88E3292F85C3057
S21444A4C082F88F32124B1968124B01F007011B6851
S21444A4D003F0010343EA41030F49097801F00101FF
S21444A4E043EA01130D49096801F00F0143EA411399
S21444A4F00B49096801F00F0143EA4123B2F8901270
S21444A50001F460410B43A2F89032704760874020C4
S21444A510201E4020EC1D40201A1E4020C41A402015
S21444A520C01A4020FFF7B8BF174B184A1B7812785A
S21444A5305B0002F0010203F002031343144A12784C
S21444A540920002F004021343124A1278D20002F038
S21444A55008021343104A1278120102F01002134301
S21444A5600E4A1278520102F0200213430C4A127823
S21444A570920102F0400213430A4A127843EAC21395
S21444A580094A82F894327047251C4020261C4020F5
S21444A590241C4020231C4020221C4020211C4020F8
S21444A5A0201C40207E17402060874020174B1868A8
S21444A5B010B500F28F20164C05F084FE154905F0C0
S21444A5C08DFF05F029FA0AF02FFA05F055FD124BD7
S21444A5D0A4F82402186800F2666005F073FE0F497A
S21444A5E005F07CFF05F018FA0AF01EFA05F044FD63
S21444A5F00B4BA4F826021A680A4B1B6803F00F0399
S21444A60043EA021384F8283210BD00BFBC1A402027
S21444A610608740200AD7A33CB81A4020CDCC4C3D96
S21444A620B01A4020B41A4020174B186810B500F2F0
S21444A6308F20164C05F046FE154905F04FFF05F0F1
S21444A640EBF90AF0F1F905F017FD124BA4F82C02C9
S21444A650186800F2666005F035FE0F4905F03EFFC7
S21444A66005F0DAF90AF0E0F905F006FD0B4BA4F81C
S21444A6702E021A680A4B1B6803F00F0343EA0213C0
S21444A68084F8303210BD00BFAC1A402060874020AA
S21444A6900AD7A33CA81A4020CDCC4C3DA01A402053
S21444A6A0A41A4020174B186810B500F28F20164C99
S21444A6B005F008FE154905F011FF05F0ADF90AF05E
S21444A6C0B3F905F0D9FC124BA4F83402186800F22A
S21444A6D0666005F0F7FD0F4905F000FF05F09CF9AC
S21444A6E00AF0A2F905F0C8FC0B4BA4F836021A6827
S21444A6F00A4B1B6803F00F0343EA021384F838320C
S21444A70010BD00BF9C1A4020608740200AD7A33C57
S21444A710981A4020CDCC4C3D901A4020941A4020A4
S21444A720174B186810B500F28F20164C05F0CAFD7A
S21444A730154905F0D3FE05F06FF90AF075F905F0F2
S21444A7409BFC124BA4F83C02186800F2666005F0C5
S21444A750B9FD0F4905F0C2FE05F05EF90AF064F94A
S21444A76005F08AFC0B4BA4F83E021A680A4B1B6899
S21444A77003F00F0343EA021384F8403210BD00BFCF
S21444A7808C1A4020608740200AD7A33C881A402071
S21444A790CDCC4C3D801A4020841A40204C4B4FF080
S21444A7A084412DE9F04FDFF864A187B01B788AF81E
S21444A7B0B832484B1B788AF8B932474B186805F0CC
S21444A7C0D1FC4FF0834105F0D5FD05F025F90AF09C
S21444A7D02BF9424B8046894618684FF0844105F071
S21444A7E0C1FC4FF0834105F0C5FD05F015F90AF0AC
S21444A7F01BF93B4B06460F4693F800B0394B3A4993
S21444A8000BF0010B186805F0ADFC384905F066FE00
S21444A81005F002F90AF008F9354B364A1B78CDE9BB
S21444A820000110683449059305F09CFC334905F053
S21444A83055FE05F0F1F80AF0F7F8314A1478314A33
S21444A84004F001041578240305F00105CDE902015E
S21444A8504946404605F010FCC0F30900AD023946AF
S21444A8600543BAF8BA0200F4784005433046AAF8DD
S21444A870BA524FEA8B2505F0FFFBC0F3090BDDE91E
S21444A880000105F0F9FB204A059B45EA0B0B02EA5A
S21444A890C02203F001034BEA020BDAF8BC224BEA6F
S21444A8A0C35302F07F421343DDE90201CAF8BC32C7
S21444A8B005F0E2FBC0F30B000443BAF8C00200F410
S21444A8C060400443AAF8C04207B0BDE8F08F00BF1A
S21444A8D05D1940205C1940205819402050194020EA
S21444A8E04C1940204819402033336F410AD7233C43
S21444A8F04419402040194020CDCCCC42CDCC4C3DD0
S21444A9003C1940205419402000F87F0060874020BE
S21444A910124B1A8DC3F85C22114A1168114A01F091
S21444A9200F01126802F00F0242EA011293F82B104C
S21444A93042EA0122A3F860229A8DC3F864220A4AA6
S21444A94011680A4A126802F00F0242EA011283F8BA
S21444A9506822074A126883F8692270476087402055
S21444A960441F4020481F4020341F4020381F4020AA
S21444A970301F4020114B1A8EC3F86C22104A1168BF
S21444A980104A126802F00F0242EA011283F870225B
S21444A9900D4A126883F871229A8EC3F874220B4AC1
S21444A9A011680B4A126802F00F0242EA011283F859
S21444A9B07822084A126883F87922704760874020D4
S21444A9C0241F4020281F4020201F4020141F4020C2
S21444A9D0181F4020101F40200F4B1A8FC3F87C22AC
S21444A9E00E4A11680E4A126802F00F0242EA011239
S21444A9F083F880229A8FC3F884220A4A11680A4A46
S21444AA00126802F00F0242EA011283F88822074ACB
S21444AA10126883F88922704760874020041F4020CC
S21444AA20081F4020F81E4020FC1E4020F41E4020F4
S21444AA30334B3449F0B51E78334B06F0030691F891
S21444AA405C201D78314B42EA062205F003051C685B
S21444AA502F4B42EA8522240318682E4BA4B20004E6
S21444AA601B78224300F4702003F003072A4B10435C
S21444AA701B7803F0030343EA8703284F3F7807F025
S21444AA80030743EA0713264F3F7807F0030743EAD2
S21444AA908713244F3F7807F0030743EA0723224FE0
S21444AAA03F7807F0030743EA8723204F3F7807F0B1
S21444AAB0030743EA07331E4F3F68BF03BFB23B4317
S21444AAC01C4F43EA06433F7843EA864307F00307AE
S21444AAD043EA065343EA865343EA066343EA8763F4
S21444AAE0D1F8007207F070473B43C1F80032D1F802
S21444AAF004321B0D1B051843C1F80402F0BD00BF09
S21444AB005C1E4020608740205D1E4020101A402076
S21444AB100C1A40205F1E40205E1E4020601E4020CF
S21444AB20611E4020621E4020641E4020631E40205A
S21444AB30581E402069184020204B214A70B51C6896
S21444AB40204BB2F8605004F00F04186892F8603056
S21444AB5005F4FF4592F8641000F00F0003F07F03FD
S21444AB602B43156E05F4FF052B43B2F86250C5F32C
S21444AB70C11543EAC55392F86350C5F3410643EA08
S21444AB804663C5F3C106C5F3411543EAC66343EAC3
S21444AB904573D2F8085205F000452B43C2F80832F4
S21444ABA001F03F03B2F80C1243EA841301F4404127
S21444ABB043EA80230B43A2F80C3270BDE81D4020C4
S21444ABC060874020E41D40201D4B1E4A1B681268C7
S21444ABD09B001D4902F0030203F00C0313431B4A77
S21444ABE01268120102F030021343194A12689201A5
S21444ABF0D2B21343174A1268120202F44072134345
S21444AC00154A1268920202F440621343134A1268C9
S21444AC10120302F440521343114A1268920302F498
S21444AC20703213430F4A1268920402F470121343AC
S21444AC30D1F82022920D92051343C1F82032704772
S21444AC40FC194020001A402060874020F819402014
S21444AC50F4194020F0194020EC194020E81940200F
S21444AC60E4194020E01940201A4B1B49186810B5D7
S21444AC7005F034FC194C04F0CFFE09F0D5FE05F07F
S21444AC80FBF9174B1449A4F81002186805F026FC83
S21444AC9004F0C2FE09F0C8FE05F0EEF9114BA4F824
S21444ACA01202188805F012FB0B4905F017FC04F055
S21444ACB0B3FE09F0B9FE05F0DFF90B4BA4F8140215
S21444ACC01A680A4B1B6803F00F0343EA021384F81E
S21444ACD0163210BDC81D4020CDCCCC3D60874020E8
S21444ACE0CC1D4020C61D40202C1E4020301E402037
S21444ACF0124A92F8783010B582F81832104BD2F8CF
S21444AD0018421878B2F87A30C3F38701936FC3F3C6
S21444AD1009231B0243EA81430A49097801F00F01DB
S21444AD2043EA8163084921400B43C2F8183292F83B
S21444AD301C3260F3030382F81C3210BD6087402047
S21444AD40DA194020DB194020FF0000C0094B0A49AD
S21444AD501A680A4B02F007021B6803F0030343EA2F
S21444AD60820391F8982222F01F02134381F8983206
S21444AD70704700BF581C4020608740204C1B402032
S21444AD80064B10B5064C186805F0BAFCB4F89C326D
S21444AD9060F30903A4F89C3210BD00BF741C402025
S21444ADA060874020094B0A4A1B7812789B00094961
S21444ADB002F0030203F00C03134391F8A02222F09E
S21444ADC00F02134381F8A032704700BFD6194020C3
S21444ADD0D719402060874020044B054993F8A422A5
S21444ADE0097861F3020283F8A42270476087402002
S21444ADF0D5194020044B054993F8A822097861F3F5
S21444AE00030283F8A822704760874020D419402064
S21444AE10F8B53D4B3D4D1B783D4985F8AC323D4B2E
S21444AE20186805F05BFB04F0F7FD09F0FDFD05F03E
S21444AE3023F9394A394B03EA40231068D5F8AC2243
S21444AE40000200F480700343354810400343C5F8BD
S21444AE50AC32344B1B7885F8B032334B1C68334BDA
S21444AE6004F003041F68324B07F001071E68314B99
S21444AE7044EA870406F00106186805F023FA4FF002
S21444AE80814105F077FA05F03BFC2B4A2B4B44EA0C
S21444AE90C606D5F8B01203EA00231068284A80058F
S21444AEA095F8B44200F4800024F00F04034310687D
S21444AEB0244A2643C005126800F4000085F8B462AC
S21444AEC01206034302F0407213431F4A1268920666
S21444AED002F0406213431D4A1268120702F0805281
S21444AEE013431B4A1268520702F000521343194A8E
S21444AEF01268920702F080421343174A0A401343EB
S21444AF00C5F8B032F8BD00BF7C19402060874020A9
S21444AF10CDCCCC3DAC194020B019402000FEFF01FA
S21444AF20FF0000FE7D1940208819402084194020E7
S21444AF3080194020A8194020A419402000FF3F0053
S21444AF40A0194020581C40209819402094194020AD
S21444AF50901940208C194020FF000080084A094B75
S21444AF601278094983F8C422084A0978127883F883
S21444AF70C52293F8C62261F3000283F8C6227047BE
S21444AF80C619402060874020C4194020C519402077
S21444AF90114B12491B6810B5114C84F8E032114B22
S21444AFA01B6884F8E132104B186805F0DBF80F494B
S21444AFB005F094FA04F030FD09F036FD05F05CF82F
S21444AFC00B4A94F8E4321278A4F8E20262F30003DF
S21444AFD084F8E43210BD00BFC019402000C02344AA
S21444AFE060874020BC194020B81940200AD7A33CAB
S21444AFF0B4194020F8B5204B204D186805F062F986
S21444B0004FF0814105F0B6F905F07AFB1C4B044637
S21444B0101F681C4BC4F30D0407F001071E681A4B47
S21444B02044EA8734186844EAC63405F04BF94FF0CE
S21444B030814105F09FF905F063FB144AC0F30D0304
S21444B040A5F8DC421068124A800300F480400343AB
S21444B0501068104AC003126800F4FF00D205034388
S21444B06002F0FF421343D5F8D82202F000421343BD
S21444B070C5F8D832F8BD00BF681940206087402024
S21444B08064194020601940207819402074194020E3
S21444B090701940206C1940200D4B0E4A1B780E49FF
S21444B0A082F8EC320D4B09781B7801F0010182F8E6
S21444B0B0ED320B4B1B785B0003F002030B4392F814
S21444B0C0EE1221F003010B4382F8EE32704700BFC4
S21444B0D03B19402060874020391940203A194020C7
S21444B0E0381940200C4B0D4A1B680D4982F8E8324B
S21444B0F00C4B09781B6801F0030182F8E9320A4BCD
S21444B1001B789B0003F00C030B430849097843EA79
S21444B110011382F8EA327047341940206087402091
S21444B1202F194020301940202E1940202D19402038
S21444B130F8B5254B254C1B78254F84F8F032254B23
S21444B1401B7884F8F132244B1878323005F0BEF878
S21444B150014605F007F805F0D3FA204984F8F202D0
S21444B1600E781F493F780D781E4907F001071E4B9D
S21444B17008781E491A78303009781D4B49001B78E8
S21444B18001F03E01394394F8F37227F03F07394300
S21444B19084F8F31203F03F0102F01F0306F00F0297
S21444B1A043EA411343EAC22305F03F0243EAC2336B
S21444B1B000F03F0243EA4253D4F8F42202F07842C5
S21444B1C01343C4F8F432F8BD2C194020608740205D
S21444B1D0291940202B1940202A194020251940209F
S21444B1E0241940202319402027194020281940209C
S21444B1F02619402038B50C4B0C4C5D68284604F0A4
S21444B2000BFC09F011FC04F037FF0949C4F8D402DA
S21444B210284605F063F904F0FFFB09F005FC04F04A
S21444B2202BFFC4F8D00238BD30464020608740200B
S21444B230000008422DE9F74F374D384E686805F050
S21444B2405FFA86F8F802A86805F05AFA344986F890
S21444B250F902686904F086FF324905F03FF905F0C3
S21444B2604FFA8346A86905F04BFA2D490446E86927
S21444B27004F078FF2B4905F031F9CBF3090B05F0C0
S21444B2803FFA8246286A05F03BFA25498146686AB1
S21444B29004F068FF234905F021F905F031FA8046A9
S21444B2A0A86A05F02DFA1E4900F00107E86804F084
S21444B2B059FF1C4905F012F905F022FAC0F30903B8
S21444B2C02869019305F01CFA019B00F0010043EA4B
S21444B2D08023B6F8FA0200F4784003431248A6F8EE
S21444B2E0FA32A30200EACA2A03F480634FEA4950BA
S21444B2F043EA0B0300F4001043EA0A03034343EA19
S21444B3008853C6F8FC3296F8003367F3000386F891
S21444B310003303B0BDE8F08F3046402060874020BD
S21444B32066667241CDCC4C3D00F81F00084A094B76
S21444B3301278094983F82823084A0978127883F84A
S21444B340292393F82A2361F3000283F82A237047BB
S21444B350221940206087402020194020211940208F
S21444B360114B124A1B68124910B5124C127884F8D5
S21444B3701833114B1B6884F8193394F81C3362F362
S21444B380000384F81C330D4B186804F0EBFE0C499C
S21444B39005F0A4F804F040FB09F046FB04F06CFE0C
S21444B3A0A4F81A0310BD00BF1C19402012194020EF
S21444B3B000C02344608740201819402014194020B8
S21444B3C00AD7A33C284B294910B5294C1B7884F846
S21444B3D01033284B186805F081F804F01DFB09F07B
S21444B3E023FB04F049FE244A244B03EA4023106816
S21444B3F0D4F81023000200F4807003432048104021
S21444B400204A03431268C4F8103312021E4B02F457
S21444B41080721B7884F814331C4B1B685B0203F45D
S21444B420C06313431A4A1268D20202F4C05213434A
S21444B430184A1268520302F400521343164A12681A
S21444B440920302F480421343144A1268D20302F46D
S21444B450C0321343D4F8142322F4FF3222F4807209
S21444B4601343C4F8143310BD10194020CDCCCC3D42
S21444B47060874020081940200C19402000FEFF0138
S21444B480FF0000FE041940201119402000194020F6
S21444B490FC184020F8184020F4184020F0184020AB
S21444B4A03A4B4FF084412DE9F047394E1B7886F8E5
S21444B4B00433384B1B7886F80533374B186804F04A
S21444B4C051FE4FF0834104F055FF05F019F9334B14
S21444B4D00446334993F800A0324B0AF0010A186830
S21444B4E004F040FE304904F0F9FF05F009F92F4B0B
S21444B4F081462F4993F800802E4B08F001081868BF
S21444B50004F030FE2C4904F0E9FF05F0F9F82B4B23
S21444B51005464FF084411F78294BC5F30B0507F0C9
S21444B5200107186804F01EFE4FF0834104F022FF22
S21444B53005F0E6F8234BC0F3090245EA07351878C8
S21444B540C4F3090300F0010043EA8A2342EA802256
S21444B550B6F8060300F4784002431B4800EAC929BB
S21444B560A6F80623D6F8082343EA090302F07F42E6
S21444B57043EAC8531343C6F80833B6F80C3303F407
S21444B58060431D43A6F80C53BDE8F087ED184020F1
S21444B59060874020EC184020E0184020DC1840200B
S21444B5A033336F41D81840200AD7233CD418402060
S21444B5B0CDCCCC42D0184020CDCC4C3DCC184020ED
S21444B5C0E8184020E418402000F87F002DE9F74FA3
S21444B5D0374D384E686805F093F886F84803A868EF
S21444B5E005F08EF8344986F84903686904F0BAFDD4
S21444B5F0324904F073FF05F083F88346A86905F0E2
S21444B6007FF82D490446E86904F0ACFD2B4904F064
S21444B61065FFCBF3090B05F073F88246286A05F0FC
S21444B6206FF825498146686A04F09CFD234904F076
S21444B63055FF05F065F88046A86A05F061F81E498E
S21444B64000F00107E86804F08DFD1C4904F046FF4D
S21444B65005F056F8C0F309032869019305F050F83D
S21444B660019B00F0010043EA8023B6F84A0300F445
S21444B670784003431248A6F84A33A30200EACA2A8B
S21444B68003F480634FEA495043EA0B0300F4001086
S21444B69043EA0A03034343EA8853C6F84C3396F80E
S21444B6A0503367F3000386F8503303B0BDE8F08F99
S21444B6B0304640206087402066667241CDCC4C3D83
S21444B6C000F81F000D4B0E4A1B780E4982F82433AF
S21444B6D00D4B09781B7801F0010182F825330B4B9A
S21444B6E01B785B0003F002030B4392F8261321F009
S21444B6F003010B4382F82633704700BFCB18402023
S21444B70060874020C9184020CA184020C8184020E6
S21444B7100C4B0D4A1B680D4982F820330C4B0978B4
S21444B7201B6801F0030182F821330A4B1B789B0007
S21444B73003F00C030B430849097843EA011382F8E3
S21444B74022337047C418402060874020BC184020ED
S21444B750C0184020BB184020BA184020F8B5254BE6
S21444B760254C1B78254F84F84033254B1B7884F8AA
S21444B7704133244B1878323004F0A8FD014604F0D7
S21444B780F1FC04F0BDFF204984F842030E781F49BB
S21444B7903F780D781E4907F001071E4B08781E496E
S21444B7A01A78303009781D4B49001B7801F03E0169
S21444B7B0394394F8437327F03F07394384F84313D7
S21444B7C003F03F0102F01F0306F00F0243EA411361
S21444B7D043EAC22305F03F0243EAC23300F03F0285
S21444B7E043EA4253D4F8442302F078421343C4F85D
S21444B7F04433F8BDB918402060874020B61840202E
S21444B800B8184020B7184020B2184020B11840203D
S21444B810B0184020B4184020B5184020B318402033
S21444B82008B5FFF785FCBDE80840FFF797BF38B575
S21444B8300C4B0D4C5D68284604F0EEF809F0F4F81D
S21444B84004F01AFC0949C4F83C03284604F046FEB2
S21444B85004F0E2F809F0E8F804F00EFCC4F8380303
S21444B86038BD00BF30464020608740200000084274
S21444B87008B5FEF76AF8FEF7AFF8FEF733F9FEF7B9
S21444B88071F9FEF7B1F9FEF795FAFEF7D9FAFEF725
S21444B89017FBFEF753FBFEF78FFBFEF7AFFBFEF7F7
S21444B8A023FCFEF753FCFEF76BFCFEF7F1FCFEF7B9
S21444B8B05BFDFEF7B9FDFEF737FEFEF777FEFEF7B3
S21444B8C0B3FEFEF7EFFEFEF72BFFFFF721F8FFF778
S21444B8D051F8FFF781F8FFF7ABF8FFF72DF9FFF7BC
S21444B8E0C3F9FFF705FAFFF76FF9FFF72FFAFFF7EB
S21444B8F047FAFFF757FAFFF76FFAFFF77BFAFEF7B8
S21444B9004DFFFFF777FCFFF7CBFDBDE80840FFF798
S21444B9108EBF114B11491B6810B5114C84F8543333
S21444B920104B1B6884F855330F4B186804F01AFC08
S21444B9300E4904F0D3FD04F06FF809F075F804F0EE
S21444B9409BFB0B4A94F858331278A4F8560362F3D8
S21444B950000384F8583310BDAC18402000C023447C
S21444B96060874020A8184020A41840200AD7A33C4B
S21444B970A11840200D4B0E4A1B780E4982F86033BE
S21444B9800D4B09781B7801F0010182F861330B4BAB
S21444B9901B785B0003F002030B4392F8621321F01A
S21444B9A003010B4382F86233704700BFA01840205F
S21444B9B0608740209E1840209F1840209D184020B5
S21444B9C00C4B0D4A1B780D4982F85C330C4B0978B6
S21444B9D01B7801F0030182F85D330A4B1B789B0009
S21444B9E003F00C030B430849097843EA011382F831
S21444B9F05E3370479C184020608740209A18402049
S21444BA009B1840209918402098184020114B124902
S21444BA101B6810B5114C84F86433114B1B6884F8CA
S21444BA206533104B186804F09DFB0F4904F056FD2F
S21444BA3003F0F2FF08F0F8FF04F01EFB0B4A94F8FC
S21444BA4068331278A4F8660362F3000384F8683314
S21444BA5010BD00BF9418402000C023446087402097
S21444BA60901840208C1840200AD7A33C88184020C1
S21444BA700D4B0E4A1B780E4982F86C330D4B0978F1
S21444BA801B7801F0010182F86D330B4B1B785B0089
S21444BA9003F002030B4392F86E1321F003010B43A9
S21444BAA082F86E33704700BF871840206087402076
S21444BAB08518402086184020841840200C4B0D4A98
S21444BAC01B680D4982F870330C4B09781B6801F0EB
S21444BAD0030182F871330A4B1B789B0003F00C0376
S21444BAE00B430849097843EA011382F872337047D6
S21444BAF08018402060874020791840207C184020D9
S21444BB00781840207718402008B5FFF727FAFFF743
S21444BB103FFAFFF77DF9FFF76DFAFFF78BFBFFF768
S21444BB20BBFAFFF7DFFAFFF701FCFFF719FCFFF754
S21444BB3049FCFFF74BFDFFF7C5FDFFF7E9FDFFF7AF
S21444BB40E8FEFFF717FFFFF73BFFFFF75FFFFFF740
S21444BB508FFFBDE80840FFF7B1BF074A0020074BF8
S21444BB60D2F87811D2F87C219962DA62044B93E8D1
S21444BB700600FBF7A1BC00BF60874020D88A40205F
S21444BB8018834600194A1A4892F8843130B492F819
S21444BB90854180F82830C4F3010104F01C03C4F343
S21444BBA041140B4392F8861180F82930D2F8843138
S21444BBB0C3F3C135C1F30013C1F34111DB0143EABA
S21444BBC08503234380F82A3092F8873103F007032D
S21444BBD041EA8301D2F88831C362064B80F82B10C1
S21444BBE0002093E8060030BCFBF766BC6087402024
S21444BBF0D88A4020208346000B4A00200B4BD2F8BC
S21444BC008C119962B2F8901183F82C1092F8921124
S21444BC1092F8932183F82D1083F82E20044B93E852
S21444BC200600FBF749BC00BF60874020D88A402006
S21444BC3028834600084B002093F8E431C3F30002FF
S21444BC4003F0FE031343054A82F82830044B93E876
S21444BC500600FBF731BC00BF60874020D88A4020EE
S21444BC60308346000D480E4AD0F8E8319362B0F867
S21444BC70EC319385B0F8EE31C3F30D0190F8EF3113
S21444BC80002003F0C00382F82E1043EA112382F802
S21444BC902F30044B93E80600FBF70EBC6087402029
S21444BCA0D88A40206083460008B50A4B50200A4A8A
S21444BCB0D3F8A41193F8A8312832116008211371DF
S21444BCC0F8F722FA054B002093E80600BDE8084042
S21444BCD0FBF7F2BB60874020D88A40203883460072
S21444BCE0094B00200949D3F8AC2193F8B0318A6255
S21444BCF003F0F002C3F30303134381F82F30044BDD
S21444BD0093E80600FBF7D8BB60874020D88A4020DB
S21444BD1040834600094B00200949D3F8B42193F8E0
S21444BD20B8318A6203F0F002C3F30303134381F885
S21444BD302F30044B93E80600FBF7BEBB60874020D9
S21444BD40D88A402048834600094B00200949D3F846
S21444BD50BC2193F8C0318A6203F0F002C3F30303B4
S21444BD60134381F82F30044B93E80600FBF7A4BB3B
S21444BD7060874020D88A4020508346000A4A0020E4
S21444BD800A4BD2F8DC1192F8E021996283F82C2011
S21444BD9083F82D2083F82E2083F82F20044B93E835
S21444BDA00600FBF789BB00BF60874020D88A402046
S21444BDB058834600254A264992F8C431C3F3010005
S21444BDC003F0FC03034310B481F8283092F8C531DD
S21444BDD0C3F3010003F0FC03034392F8C60181F861
S21444BDE02930C0F3010400F00C0323438409C0F354
S21444BDF0011081F82A3092F8C73103F003039B01FF
S21444BE0043EA8403034381F82B3092F8C83181F81F
S21444BE102C3092F8C93103F03800C3F302030343CD
S21444BE2081F82D3092F8CA31C3F38300D2F8C83172
S21444BE30C3F3833343EA0013002081F82F30054BC5
S21444BE4010BC93E80600FBF737BB00BF6087402072
S21444BE50D88A4020688346000B490C4A91F8CC3176
S21444BE60C3F3010003F0FC030343002082F82830A8
S21444BE7091F8CD31C3F3010382F82930044B93E89B
S21444BE800600FBF719BB00BF60874020D88A4020D5
S21444BE9070834600084B002093F8D83103F0040220
S21444BEA0C3F301031343054A82F82830044B93E84E
S21444BEB00600FBF701BB00BF60874020D88A4020BD
S21444BEC0788346001049114A91F8D031C3F30000F4
S21444BED003F0FE03034382F8283091F8D13103F08F
S21444BEE07C00C3F301030343002082F82930D1F8D1
S21444BEF0D031C3F3CF335385D1F8D431D362044B16
S21444BF0093E80600FBF7D8BA60874020D88A4020DA
S21444BF108083460019491A48D1F8442200F5FE5356
S21444BF2010B41A6041F6C473B1F84822C25291F86C
S21444BF304A22C2F3C103C2F341041B0143EA840309
S21444BF40C2F30004C2F34012234343EA821341F689
S21444BF50C672835491F84B32C3F38302B1F84A3223
S21444BF60C3F3831343EA021341F6C7728354012092
S21444BF70044B10BC93E80600FBF79EBA608740204B
S21444BF80D88A4020A88346002148224938B590F8EC
S21444BF904C3201F5FE5203F07C04C3F30103234301
S21444BFA090F84D421370C4F30113C4F3C005C4F3B0
S21444BFB081145B0143EA0513B0F84C52C5F3C3152C
S21444BFC02B4341F6C1754B5541F6C273CC5441F6EA
S21444BFD0C37390F84E42CC5441F6C473B0F8504202
S21444BFE0CC5290F8523203F0F000C3F303030343F9
S21444BFF041F6C7700B5408211420F8F7EEF9064BA7
S21444C000012093E80600BDE83840FBF755BA00BF68
S21444C01060874020D88A4020B08346001149124B9E
S21444C02001F5FE52D3F8540210B5B3F858421060E6
S21444C03041F6C47093F85A320C5203F0F000C3F33E
S21444C0400303034341F6C7700B5408211520F8F741
S21444C050C4F9064B012093E80600BDE81040FBF700
S21444C0602BBA00BFD88A402060874020B883460059
S21444C07015491648D1F88C3200F5FE5210B51360B7
S21444C08091F8903203F01E04C3F30003234341F6B1
S21444C090C474035591F89132C3F34304B1F8903213
S21444C0A041F6C771C3F3431343EA041343540821C8
S21444C0B01620F8F792F9064B012093E80600BDE8EF
S21444C0C01040FBF7F9B900BF60874020D88A40206B
S21444C0D0C0834600FFF7CCBF08B5FDF7A9FBF5F7CC
S21444C0E0CCFBFEF7D9F9BDE80840FFF7C1BF084BC3
S21444C0F0012093F89432C3F3000203F0FE03134383
S21444C100044A1370044B93E80600FBF7D5B900BF06
S21444C1106087402098AA4020C883460008B50E4849
S21444C1200E4B00F5FE52D3F8241293F828321160D1
S21444C13003F0F001C3F303030B4341F6C7714354C2
S21444C14008215020F8F749F9054B012093E80600EA
S21444C150BDE80840FBF7B0B9D88A40206087402045
S21444C1608883460008B50E480E4B00F5FE52D3F8B9
S21444C1702C1293F83032116003F0F001C3F303033A
S21444C1800B4341F6C771435408215120F8F725F96B
S21444C190054B012093E80600BDE80840FBF78CB940
S21444C1A0D88A4020608740209083460008B50E48D1
S21444C1B00E4B00F5FE52D3F8341293F83832116021
S21444C1C003F0F001C3F303030B4341F6C771435432
S21444C1D008216020F8F701F9054B012093E8060092
S21444C1E0BDE80840FBF768B9D88A402060874020FD
S21444C1F09883460008B50E480E4B00F5FE52D3F819
S21444C2003C1293F84032116003F0F001C3F3030389
S21444C2100B4341F6C771435408216120F8F7DDF813
S21444C220054B012093E80600BDE80840FBF744B9F7
S21444C230D88A402060874020A0834600174B184A7F
S21444C24003F5FE51B2F85C02088092F8601201F0E1
S21444C250F000C1F30301014341F6C270195441F69C
S21444C260C37192F86102585441F6C471B2F864023C
S21444C270585292F8681201F0F000C1F303010143EA
S21444C28041F6C6701954012092F8691241F6C772F5
S21444C2909954044B93E80600FBF70EB9D88A40201D
S21444C2A060874020D0834600174B184A03F5FE515A
S21444C2B0B2F86C02088092F8701201F0F000C1F3F4
S21444C2C00301014341F6C270195441F6C37192F812
S21444C2D07102585441F6C471B2F87402585292F836
S21444C2E0781201F0F000C1F30301014341F6C67031
S21444C2F01954012092F8791241F6C7729954044BA6
S21444C30093E80600FBF7D8B8D88A402060874020D8
S21444C310D8834600174B184A03F5FE51B2F87C0200
S21444C320088092F8801201F0F000C1F30301014343
S21444C33041F6C270195441F6C370D2F884121954A7
S21444C340090A41F6C470195492F8881201F0F000B4
S21444C350C1F30301014341F6C6701954012092F813
S21444C360891241F6C7729954044B93E80600FBF7CA
S21444C370A3B800BFD88A402060874020E0834600A8
S21444C3802848294990F8003201F5FE5270B5C3F3A7
S21444C390010403F0FC032343137090F80132C3F303
S21444C3A0010403F0FC03234341F6C1740B5541F6E4
S21444C3B0C27390F802422501A609C4F30114CD5471
S21444C3C090F8035205F00303C5F381051B0143EAC5
S21444C3D08603234341F6C37443EA85130B5541F65B
S21444C3E0C47390F80442CC5441F6C57490F80532B0
S21444C3F090F806021D01C3F3031300F00F000D5519
S21444C40043EA001341F6C7700B5408214FF4AE605C
S21444C410F7F7E3FF054B012093E80600BDE87040BC
S21444C420FBF74AB860874020D88A402008844600F4
S21444C4302D4991F8080238B5C0F3001500F00803FA
S21444C4402A4C43EA4513C0F3020504F5FE522B4337
S21444C450C0F34015C0F3801043EA851343EAC01383
S21444C46041F6C1701370B1F80832C3F3C7132354AE
S21444C47041F6C270D1F80832C3F3C733235491F857
S21444C4800B02C0F3C103C0F34105C0F341101B01C6
S21444C49043EA8503B1F80A52C5F3C1152B4343EA70
S21444C4A0801341F6C370235441F6C47091F80C329D
S21444C4B09B00235491F80D32C3F38300B1F80C3239
S21444C4C041F6C771C3F3831343EA00134FF4B060D5
S21444C4D063540821F7F781FF054B012093E80600D3
S21444C4E0BDE83840FAF7E8BF60874020D88A402045
S21444C4F0108446001849194891F8203200F5FE5237
S21444C50010B5C3F3010403F0FC032343137091F8FE
S21444C510213203F03C04C3F30103234341F6C174C0
S21444C520035591F82232C3F38304D1F8203241F6FE
S21444C530C771C3F3833343EA04134354082140F2D8
S21444C5408550F7F74AFF064B012093E80600BDE8FE
S21444C5501040FAF7B1BF00BF60874020D88A402019
S21444C560188446001149124B01F5FE52D3F81002C6
S21444C57010B5B3F81442106041F6C47093F81632FE
S21444C5800C5203F0F000C3F30303034341F6C770B1
S21444C5900B5408214FF4B260F7F71FFF054B0120F8
S21444C5A093E80600BDE81040FAF786BFD88A4020D4
S21444C5B06087402028844600104810B5104C90F8F8
S21444C5C0183204F5FE52137090F81C3203F00F0133
S21444C5D090F81B3240F29550C3F3830343EA0113A9
S21444C5E041F6C77163540821F7F7F7FE054B01205F
S21444C5F093E80600BDE81040FAF75EBF6087402027
S21444C600D88A402030844600084B0120084993F8D5
S21444C610983203F01C02C3F30103134341F6C3727A
S21444C6208B54044B93E80600FAF746BF60874020D5
S21444C630D88A4020E8834600084B41F6C271B3F8D6
S21444C6409C22074BC2F30120585441F6C371012083
S21444C6505A54044B93E80600FAF72EBF60874020EE
S21444C660D88A4020F0834600054B0120054A93F8BB
S21444C670A0321B011370044B93E80600FAF71CBF64
S21444C6806087402098AA4020F8834600074B41F62E
S21444C690C1720749012093F8A43203F007039B00B4
S21444C6A08B54044B93E80600FAF706BF6087402095
S21444C6B0D88A402000844600074B41F6C172074999
S21444C6C0012093F8A832C3F303038B54044B93E836
S21444C6D00600FAF7F1BE00BF60874020D88A4020A3
S21444C6E0208446000D4843F65872B0F8C41208B584
S21444C6F049BA0B4B99521A4490F8C61243F65A70EC
S21444C700C901195403213220F7F7FEFC054B0220D9
S21444C71093E80600BDE80840FAF7CEBE608740209E
S21444C720D88A402038844600114B43F65870114A44
S21444C730B3F8E01249BA10B5115243F65A74B3F836
S21444C740E21293F8E43249BA03F00103115343F674
S21444C7505C719B015354024405214020F7F75DFB6E
S21444C760054B022093E80600BDE81040FAF7A4BE45
S21444C77060874020D88A4020408446003048314A6A
S21444C78090F8B03290F8AC1270B543F6587590F8FD
S21444C790B342535543F65973D15443F65A71D0F8BD
S21444C7A0AC32C3F34F235BBA5352C4F3801304F042
S21444C7B0100141EAC301C4F30103194390F8AD32B2
S21444C7C003F0010341EA4311C4F3810304F0200457
S21444C7D041EA831143F65C73D15490F8B412C1F322
S21444C7E0800601F00803C1F3010143EA06130B4334
S21444C7F090F8B212D0F8B0022343CC09C1F38011AA
S21444C80043EA841343F65D741355C0F30D2343F68D
S21444C8105E74C0F305409B001055642043EA410310
S21444C82043F65F7153542A440821F7F76DFC064BD0
S21444C830022093E80600BDE87040FAF73DBE00BF0C
S21444C84060874020D88A4020488446001F4843F6E4
S21444C85058721F4BB0F8DA12C1F3C71170B5995429
S21444C86043F65974D0F8D8121A44B0F8D852C1F3E3
S21444C870C731C5F30526195590F8DD4204F080010A
S21444C880C4F38014314343F65A76995543F65B71A4
S21444C8905D54B0F8DC5290F8D912C5F3052001F087
S21444C8A04001014343F65C7041EAC411195443F60F
S21444C8B05D716A205D540621F7F726FC054B02207D
S21444C8C093E80600BDE87040FAF7F6BD608740205E
S21444C8D0D88A40205084460038B52C4B43F65870CE
S21444C8E02B4AB3F8B812B3F8C05249BA115293F867
S21444C8F0BE12CC09C5F3032141EA041193F8C142A0
S21444C900C4F3001441EA441193F8BB42C4F38004D0
S21444C91041EA841193F8BD42C4F3800441EAC41149
S21444C92043F65A74115543F65B71B3F8BA425554FC
S21444C93043F65C71C4F30905C4F387045454B3F84E
S21444C940BC12D3F8BC32C1F30904C1F3051141EA61
S21444C950851143F65D755155C3F3CB21C3F3C343E9
S21444C96043EA041343F65E74135543F65F73D15497
S21444C970024408217020F7F7C7FB064B022093E8D1
S21444C9800600BDE83840FAF797BD00BF60874020F0
S21444C990D88A402058844600284A43F65870284986
S21444C9A0B2F8F8325BBA30B40B5243F65A73B2F864
S21444C9B0FA02B2F8FC52C0F30904C0F38700C85424
S21444C9C0C5F3012092F8FB3203F00403034392F8C4
S21444C9D0FD02C0F3800043EAC00392F8FE02C0F3AF
S21444C9E0401043EA001392F8000300F0010043EAC3
S21444C9F0401343F65B7043EA841343F65D740B546A
S21444CA0043F65C73D2F8FC02CD54C0F3C923B2F8A3
S21444CA10FE22C0F347309B010855900943EA9233FF
S21444CA2043F65E728B5443F65F73C8540220054B3C
S21444CA3030BC93E80600FAF73FBD00BF608740204D
S21444CA40D88A402060844600104843F65871104AFD
S21444CA5008B5B0F8EC325BBA535290F8EE3203F0B5
S21444CA600100C3F3400343EA400343F65A701354A9
S21444CA700A444FF444700321F7F7CFF9054B0220DC
S21444CA8093E80600BDE80840FAF716BD60874020E4
S21444CA90D88A402068844600134843F65872134B9D
S21444CAA0B0F8E81249BA10B599521A4490F8EA1206
S21444CAB043F65A70C1F301041C54C1F3031443F6FD
S21444CAC05B70C1F381011C5443F65C701954052114
S21444CAD04FF45470F7F7A1F9054B022093E806008B
S21444CAE0BDE81040FAF7E8BC60874020D88A40206A
S21444CAF070844600254943F65872B1F8F00238B5BA
S21444CB0040BA234B91F8F34298521A44D1F8F402AF
S21444CB1004F00105C4F34404C0F3C53040EAC5102C
S21444CB2043F65A75585543F65B75B1F8F402C0F3AC
S21444CB304510585543F65C7591F8F402C0F304006A
S21444CB405855B1F8F602C0F3022500F4FC6045EAF5
S21444CB50C40443F65D755C5591F8F542C4F3C304CA
S21444CB60204343F65E74185591F8F20243F65F711B
S21444CB70585408214FF46170F7F7C6FA054B022063
S21444CB8093E80600BDE83840FAF796BC6087402034
S21444CB90D88A402078844600094943F65870094AA2
S21444CBA0D1F8D0321BBA13500220D1F8D43243F60F
S21444CBB05C711BBA5350044B93E80600FAF77CBCEE
S21444CBC060874020D88A4020808446000E4845F638
S21444CBD0F062B0F8281308B549BA0C4B99521A4477
S21444CBE090F82A1345F6F260C1F300011954032164
S21444CBF03320F7F789FA064B032093E80600BDE88E
S21444CC000840FAF759BC00BF60874020D88A4020C5
S21444CC1088844600114B45F6F060114AB3F8181361
S21444CC2049BA10B5115245F6F264B3F81A1393F89C
S21444CC301C3349BA03F00103115345F6F4619B01D2
S21444CC405354024405214020F7F744F9054B03208A
S21444CC5093E80600BDE81040FAF72EBC60874020F3
S21444CC60D88A4020908446002248234A90F81013DD
S21444CC7038B590F8143345F6F064135545F6F16329
S21444CC80D15445F6F261D0F81033C3F34F235BBA60
S21444CC90535290F81513C1F34013C1F380151B018A
S21444CCA043EAC503C1F341052B4390F8115305F0FD
S21444CCB0010543EA4513C1F3C10501F0010143EA06
S21444CCC0851345F6F4655355D0F814336520C3F3FD
S21444CCD0C13343EA811145F6F563D1542244082111
S21444CCE0F7F712FA054B032093E80600BDE83840F0
S21444CCF0FAF7E2BB60874020D88A402098844600F2
S21444CD0038B52C4B45F6F0602B4AB3F80413B3F809
S21444CD100C5349BA115293F80A13CC09C5F30321AC
S21444CD2041EA041193F80D43C4F3001441EA441154
S21444CD3093F80743C4F3800441EA841193F8094303
S21444CD40C4F3800441EAC41145F6F264115545F62D
S21444CD50F361B3F80643555445F6F461C4F3090544
S21444CD60C4F387045454B3F80813D3F80833C1F310
S21444CD700904C1F3051141EA851145F6F565515597
S21444CD80C3F3CB21C3F3C34343EA041345F6F66423
S21444CD90135545F6F763D154024408217120F7F73A
S21444CDA0B3F9064B032093E80600BDE83840FAF78B
S21444CDB083BB00BF60874020D88A4020A0844600BA
S21444CDC008B5FEF7CAFEFEF7DDFEFEF715FFFEF7D2
S21444CDD031FFFEF769FFFEF783FFFEF7CFFFFEF74E
S21444CDE0E9FFFFF739F8FFF755F8FFF76BF8FEF75A
S21444CDF039FFFFF78FF8FFF7C7F8FFF70FF9FFF78C
S21444CE0076F9FFF7AFF9FFF7D1F9FFF7F3F9FFF734
S21444CE1085F9FFF713FAFFF747FAFFF77BFAFFF7B0
S21444CE20AFFAFFF705FBFFF79DFBFFF763FBFFF742
S21444CE30C3FBFFF7E9FBFFF7FFFBFFF715FCFFF724
S21444CE4025FCFFF739FCFFF747FDBDE80840FFF730
S21444CE5057BF284A45F6F0602749B2F848335BBACC
S21444CE6030B40B5245F6F263B2F84A03B2F84C5368
S21444CE70C0F30904C0F38700C854C5F3012092F8F0
S21444CE804B3303F00403034392F84D03C0F380008E
S21444CE9043EAC00392F84E03C0F3401043EA00133B
S21444CEA092F8500300F0010043EA401345F6F3605D
S21444CEB043EA841345F6F5640B5445F6F463D2F816
S21444CEC04C03CD54C0F3C923B2F84E23C0F34730C5
S21444CED09B010855900943EA923345F6F6628B5413
S21444CEE045F6F763C8540320044B30BC93E8060069
S21444CEF0FAF7E2BA60874020D88A4020A8844600E1
S21444CF00104845F6F061104A08B5B0F824335BBAC9
S21444CF10535290F8263303F00100C3F3400343EA28
S21444CF20400345F6F26013540A444FF44470032118
S21444CF30F6F7D0FF054B032093E80600BDE808400B
S21444CF40FAF7BABA60874020D88A4020B0844600B0
S21444CF50134845F6F062134BB0F8201349BA10B59F
S21444CF6099521A4490F8221345F6F260C1F301042C
S21444CF701C54C1F3031445F6F360C1F381011C54F9
S21444CF8045F6F460195405214FF45470F6F7A2FFA1
S21444CF90054B032093E80600BDE81040FAF78CBA28
S21444CFA060874020D88A4020B8844600254945F604
S21444CFB0F062B1F8400338B540BA234B91F8434386
S21444CFC098521A44D1F8440304F00105C4F34404C7
S21444CFD0C0F3C53040EAC51045F6F265585545F6E7
S21444CFE0F365B1F84403C0F34510585545F6F46567
S21444CFF091F84403C0F304005855B1F84603C0F30F
S21444D000022500F4FC6045EAC40445F6F5655C5523
S21444D01091F84543C4F3C304204345F6F6641855D3
S21444D02091F8420345F6F7615854082140F285309A
S21444D030F7F76AF8054B032093E80600BDE8384046
S21444D040FAF73ABA60874020D88A4020C08446001F
S21444D05008B5FFF74FFDBDE80840FFF7A7BF08B582
S21444D060F4F70DFCFEF7DCFBBDE80840FFF7F0BF25
S21444D070094945F6F060094AD1F838331BBA1350CB
S21444D0800320D1F83C3345F6F4611BBA5350044BA5
S21444D09093E80600FAF710BA60874020D88A402002
S21444D0A0C8844600114B47F68860114AB3F85413B7
S21444D0B049BA10B5115247F68A64B3F8561393F832
S21444D0C0583349BA03F00103115347F68C619B0168
S21444D0D05354024405214020F6F75AFF054B0420DA
S21444D0E093E80600BDE81040FAF7E6B960874020AA
S21444D0F0D88A4020D0844600104847F68861104AB3
S21444D10008B5B0F860335BBA535290F8623303F014
S21444D1100100C3F3400343EA400347F68A601354CE
S21444D1200A444FF444700321F6F732FF054B0420BB
S21444D13093E80600BDE80840FAF7BEB96087402089
S21444D140D88A4020D8844600134847F68862134B52
S21444D150B0F85C1349BA10B599521A4490F85E1365
S21444D16047F68A60C1F301041C54C1F3031447F61E
S21444D1708B60C1F381011C5447F68C601954052119
S21444D1804FF45470F6F704FF054B042093E806006A
S21444D190BDE81040FAF790B960874020D88A40200E
S21444D1A0E084460008B50A4B49F622620949402005
S21444D1B0B3F866335BBA8B520521074AF6F746FF47
S21444D1C0064B052093E80600BDE80840FAF774B914
S21444D1D060874020D88A4020F8284120E8844600CA
S21444D1E0134849F62062134BB0F8701349BA10B589
S21444D1F099521A4490F8721349F62260C1F3010416
S21444D2001C54C1F3810449F62360C1F303111C5432
S21444D21049F62460195405214FF45470F6F716FF66
S21444D220054B052093E80600BDE81040FAF744B9DC
S21444D23060874020D88A4020F8844600104849F643
S21444D2402061104A08B5B0F86C335BBA535290F874
S21444D2506E3303F00100C3F3400343EA400349F648
S21444D260226013540A444FF444700321F6F7EEFE4A
S21444D270054B052093E80600BDE80840FAF71CB9BC
S21444D28060874020D88A4020F084460008B5FFF7DF
S21444D29029FAFFF749FAFFF771FAFFF7D7FAFFF7CB
S21444D2A0D3FBFFF7F9FBFFF791FCFFF7B3FCFFF75F
S21444D2B0DBFCFFF725FEFFF74BFEFFF7F3FEFFF719
S21444D2C01BFFFFF741FFFFF76DFFFFF7B7FFBDE812
S21444D2D00840FFF785BF08B5FCF71EFBF4F7ABFA2A
S21444D2E0FEF712FCBDE80840FFF7D0BF7047704712
S21444D2F070477047064AB2F82032B2F8681003F412
S21444D3004043C1F30D010B43A2F82032704700BFDF
S21444D31060874020044BB3F81221A3F82422B3F8C4
S21444D3200C21A3F82622704760874020044BB3F8AC
S21444D330A620A3F82C22B3F8A020A3F82E227047E8
S21444D3406087402070477047054BB3F86C21A3F8BC
S21444D3503422D3F86821C2F30F12A3F8362270475A
S21444D36060874020054BB3F87421A3F83C22D3F8D9
S21444D3707021C2F30F12A3F83E2270476087402004
S21444D380054BB3F86C21A3F8B421D3F86821C2F353
S21444D3900F12A3F8B621704760874020054BB3F8B8
S21444D3A07421A3F8BC21D3F87021C2F30F12A3F85A
S21444D3B0BE2170476087402008B5FFF7E1FFFFF7BE
S21444D3C0EDFFFFF797FFFFF7A5FFFFF7AFFFFFF768
S21444D3D0BBFFBDE80840FFF7C5BF08B5FCF7C2F978
S21444D3E0F4F72AFAFEF744FAFFF7E6FFBDE80840EA
S21444D3F0FFF7E6BC70477047704770470B4AD2F851
S21444D400C431D2F894101B0DC1F313011B050B4312
S21444D410D2F89810C2F8C43101F47F11D2F8C8315A
S21444D42023F47F130B43C2F8C8317047608740200B
S21444D43008B5F9F7E1F8BDE80840F8F707BB7047C8
S21444D440F4F7F7B9FFF747BFFFF7C7BFFBF748BA8C
S21444D4507047074A1378632B96BF01330023DBB229
S21444D4601370044A136801331360FEF735BE00BFD9
S21444D470E84B41200021402008B5FAF739F8BDE8CA
S21444D4800840F6F799BA08B5F7F704FBFFF7E7FD47
S21444D4904CF24053044AD058B0FA80F0BDE80840F5
S21444D4A04009F9F723B900BFEC4B41207047704759
S21444D4B030B53D4C85B03D48237801A90193019B86
S21444D4C01B020193019A637813440193019B1B0248
S21444D4D00193019AA37813440193019B1B02019381
S21444D4E0019AE3781344019323790293029B1B0227
S21444D4F00293029A637913440293029B1B0202939B
S21444D500029AA37913440293029B1B020293029A43
S21444D510E37913440293237A0193019B1B020193FC
S21444D520019A637A13440193019B1B020193019A67
S21444D530A37A13440193019B1B020193019AE37A55
S21444D54013440193237B0293029B1B020293029A89
S21444D550637B13440293029B1B020293029AA37BAF
S21444D56013440293029B1B020293029AE37B1344E6
S21444D570029342F21273019342F21373029300F041
S21444D580B0FB04F1100004F1080104F1180208236A
S21444D59014F8015B013B00F8015B11F8015B02F8EB
S21444D5A0015BF5D105B030BD6C114220808080000F
S21444D5B00C4A0823002102F1280030B402F1080581
S21444D5C002F12004013B02F8011B05F8011B13F08D
S21444D5D0FF0304F8011B00F8011BF3D130BCFFF72E
S21444D5E067BF00BF6C1142204F4BF0B51B688BB031
S21444D5F002934E4B1A6803925A6804929B680593AA
S21444D60042F21273029A9A4200F08980484800F027
S21444D61013FBFFF7CDFF002346480AAA50F8231011
S21444D62002EB83020133082B42F8201CF5D1002379
S21444D63040480AAA50F8231002EB83020133082B11
S21444D64042F8201CF5D102990025039A049B0598BC
S21444D650394C00903948264600F0EEFA029B38488A
S21444D6601B0E2370029B1B0C6370029B1B0AA37049
S21444D670029BE370039B1B0E2371039B1B0C63717D
S21444D680039B1B0AA371039BE371049B1B0E23722B
S21444D690049B1B0C6372049B1B0AA372049BE372D9
S21444D6A0059B1B0E2373059B1B0C6373059B1B0A70
S21444D6B0A373059BE37300F0B6FA013516F8010B25
S21444D6C000F0DAFA082DF8D11E4D002600F0CBFA09
S21444D6D01D482F4600F0A7FA013617F8010B00F054
S21444D6E0CBFA082EF8D100F0BEFA184B002203F10C
S21444D6F0080703F1100003F118019446013214F8A8
S21444D700016B15F801EB082A03F8016B07F801EBE7
S21444D71000F8016B01F801CBF0D10BB0F0BD0C481A
S21444D72000F08AFA77E700BF80808000848080001B
S21444D730A28C4600108080006C114220C68C4600A5
S21444D740E38C460074114220ED8C46007C11422046
S21444D750B88C4600194A08211948F0B592F8A53104
S21444D76000F1100C00F1080500F11807012B9CBFCE
S21444D770002382F8D431002310F8014B01391CF8F9
S21444D780016B17F801EBB4422E7818BF013344EA14
S21444D790060418BFDBB2764505F8014B1CBF0133BF
S21444D7A0DBB211F0FF01E7D133B1B2F8BE301BB99A
S21444D7B0BDE8F040FFF77CBEF0BD00BFA811422094
S21444D7C06C1142201FB5144B01A953F820305A1E41
S21444D7D0073312F8010F9A4201F8010BF9D19DF86C
S21444D7E004300024502B8DF80C4007D0432B0CD02B
S21444D7F0422B0DD0552B08BF4FF440040DF10500C5
S21444D80000F04CFA204404B010BD4FF48004F5E711
S21444D8104FF40004F2E700BF082140202DE9F04F02
S21444D8205C4D8DB082462B6805F1080806AC09A904
S21444D83063F07C4340462E46A9462B604246082366
S21444D84016F8017B013B04F8017B9BB210F8017B80
S21444D85001F8017B002BF3D1BAF10A0F0BD14146F4
S21444D8604C4C0823FF20013B04F8010B01F8010B44
S21444D8709BB2002BF7D1484BC8240021013C03F847
S21444D880011BA4B2002CF9D126464449DFF808B15E
S21444D89004F1080380279BB200932B781F4203D1E0
S21444D8A098F800301F4248D051F824300DF10C0C43
S21444D8B0581E073310F801EF98420CF801EBF9D1E3
S21444D8C04FF000038DF814309DF80C30502B59D08F
S21444D8D0432B59D0422B5AD0552B34D14FF44003C6
S21444D8E00DF10D00019300F0D9F9019B95F800C0A5
S21444D8F0184498F800302A4A3B404FEA102E2749ED
S21444D90018BF082317EA0C0F4FEA104C18BF43F011
S21444D91001030BF806C006F1010C1FFA8CFC0BF849
S21444D9200CE006F1020C1FFA8CFC0BF80C00F01C01
S21444D930043680B2B6B20BF800300134009B7F0840
S21444D940A4B2A342A9D1013508F1010895429FD15A
S21444D950BAF10A0F0FD19DF81A30BDF8182089F88D
S21444D9600230A9F800209DF82630BDF8242089F816
S21444D9700A30A9F80820084B002230469A550DB0C4
S21444D980BDE8F08F0023ABE74FF48003A8E74FF4DD
S21444D9900003A5E76C1142203E2240200821402087
S21444D9A074114220F0B50D4C0822002004F10805FD
S21444D9B014F8016B082380210E4202D12F78394295
S21444D9C001D0013080B2013B49089BB2002BF3D111
S21444D9D0013A013592B2002AEAD1F0BD6C114220D8
S21444D9E02DE9F04FDFF8B480002685B08346A8F1D1
S21444D9F0080A3446284B022E4FF080094FF00002A6
S21444DA0034BF082703272744BFB29AF8001019EA00
S21444DA10010F04D198F8001019EA010F2DD053F8DD
S21444DA20241001AD481E073110F801CF814205F895
S21444DA3001CBF9D19DF804108DF80C20502914D050
S21444DA40432914D0422915D055291CD14FF44005FA
S21444DA500DF1050000F022F905440F4B00225D4508
S21444DA600BD1E0B205B0BDE8F08F0025F0E74FF4E7
S21444DA708005EDE74FF40005EAE701344FEA59091B
S21444DA80A4B2A742C1D1013608F101080AF1010A3D
S21444DA90082EB0D1FF20E5E708214020741142202B
S21444DAA02DE9FF4700240746204EA146022C4FF09E
S21444DAB0000834BF4FF0080A4FF0030A336801A940
S21444DAC05A1E073312F8010F9A4201F8010BF9D196
S21444DAD09DF804308DF80C90502B0DD0432B15D068
S21444DAE0422B16D0552B17D001340436082CDDD1E2
S21444DAF0FF2004B0BDE8F08700250DF1050000F0D6
S21444DB00CDF80544BD420AD1E0B2F2E74FF48005B1
S21444DB10F3E74FF40005F0E74FF44005EDE708F16E
S21444DB2001081FFA88F39A45C8D8DDE70821402043
S21444DB302DE9F04FDFF8C490002585B08346A9F15F
S21444DB4008082C462B4A022D4FF0800A4FF000015D
S21444DB5034BF082703272744BFB298F800001AEAC0
S21444DB60000F04D199F800001AEA000F32D052F898
S21444DB7024000DF1040C461E073016F801EFB0429F
S21444DB800CF801EBF9D19DF804008DF80C105028E0
S21444DB9018D0432818D0422819D0552820D14FF4FD
S21444DBA040060DF1050000F079F80644124B0021BA
S21444DBB05E45104A0ED15955E0B21D44297205B04F
S21444DBC0BDE8F08F0026ECE74FF48006E9E74FF413
S21444DBD00006E6E701344FEA5A0AA4B2A742BCD18B
S21444DBE0013509F1010908F10108082DABD1FF20E0
S21444DBF0E5E700BF082140206C1142207411422002
S21444DC007047092894BF30303730C0B2704707B5E4
S21444DC1001220DF107018DF80700002013F0C8FB20
S21444DC2003B05DF804FB10B5441E14F8010F00B9A8
S21444DC3010BDFFF7ECFFF8E70FB400B5C3B044AA35
S21444DC4002A852F8041B019204F066FC002302A8C2
S21444DC508DF805318DF80631FFF7E5FF43B05DF8E2
S21444DC6004EB04B070470D2008B5FFF7D0FF0A2038
S21444DC70BDE80840FFF7CBBF10B504460009FFF7E0
S21444DC80C0FFFFF7C4FF04F00F00FFF7BAFFFFF72B
S21444DC90BEFF2C20BDE81040FFF7B9BF002330B5C7
S21444DCA01A46441E184614F8011F392908D82F2945
S21444DCB00AD95D1C01F00F0303EB00102B4606E067
S21444DCC0A1F14105052D06D900B943B10822013218
S21444DCD0072AE8D930BD5D1CA1F13703ECE71D46A1
S21444DCE0EAE7002070470000034A92F89E3001336A
S21444DCF082F89E30704700BFA811422010B52A4CC7
S21444DD0094F89A30642B94BF0133002384F89A30F5
S21444DD1094F8C63043B1013BDBB284F8C6301BB935
S21444DD2084F8C53084F88A3194F8C73053B1013B3F
S21444DD30DBB284F8C7302BB994F88A21032A08BF8B
S21444DD4084F88A31B4F8E4315BB1013B9BB2A4F861
S21444DD50E43133B9012284F8CF3184F8C13184F8F0
S21444DD60A52194F8C231013384F8C231FFF7F2FC9E
S21444DD7094F8A13123B1002084F8A10101F01FFCDE
S21444DD80B4F8BE3073B1013B9BB2A4F8BE304BB975
S21444DD9084F88A3184F8C53084F8A33184F8C131D4
S21444DDA084F8DC3110BD00BFA8114220034A92F823
S21444DDB09830013382F89830704700BFA81142204B
S21444DDC070470323002010B5064CA4F8EC3104F148
S21444DDD054020823E16CF8F713FB002384F89530CB
S21444DDE010BD00BFA8114220024B0022C3E91522F1
S21444DDF0704700BFA811422030B5224B00220124B0
S21444DE004FF4FB604FF4FA61082583F8A541A3F864
S21444DE109820A3F8B420C3F8D420A3F8CA20A3F8C3
S21444DE20CC2083F88121A3F8822183F88C2183F8BF
S21444DE309C21C3F8A02183F8D62183F8DB2183F8FC
S21444DE40DC21A3F8E42183F8EA21A3F8C220C3F82E
S21444DE50C420D864196083F89450A3F8C621C3F844
S21444DE60D02183F8D421C3E972424FF40C14C3E999
S21444DE702E22C3E96122C3F8C04183F8C421C3E912
S21444DE802B1030BDA8114220144B002293F88D115C
S21444DE9083F88A21E1B90322A3F8861183F8542033
S21444DEA093F8882142F0400283F8552093F89C2149
S21444DEB0012A01BF7F2283F85520002283F89C2143
S21444DEC0B3F8862152BAA3F8562000229A657047C2
S21444DED046F60362A3F85420E8E700BFA8114220A0
S21444DEE0054B3022A3F854200A2283F856200D22EC
S21444DEF083F8C720704700BFA8114220034B012275
S21444DF0083F8C5200B2283F8C6207047A811422008
S21444DF1008B5FFF783FC0330284B81B2284AC0B2C9
S21444DF2007291DD85921C3F8982183F8540083F84B
S21444DF30551093F89E1183F85610FF2183F8571016
S21444DF40117883F85810517883F859109178D2781C
S21444DF5083F85A1083F85B200422A3F8CA2008BD2D
S21444DF60A3F8CC10090AC3F8982141F0100183F8AD
S21444DF70550083F85410592183F8561093F89E118F
S21444DF8083F85710FF2183F85810117883F85910F6
S21444DF905178927883F85A1083F85B200322A3F8CA
S21444DFA0CA20012283F8C520022283F88A2121222E
S21444DFB083F88C21222283F88821D0E7A8114220B6
S21444DFC03E224020024B002283F85420704700BF74
S21444DFD0A811422038B5CB1C40F6FF749BB2A3422E
S21444DFE028BF2346174C1D0A84F855306223A4F8EC
S21444DFF0CC1045F0100584F8580084F85630030ACF
S21444E00084F85450022163F00F03C4F8982184F82E
S21444E01057300123A4F8CA301378A4F8CA1084F8F9
S21444E0205930537884F85A300323A4F8CA30937886
S21444E03084F85B30FFF762FF212384F88A1184F862
S21444E0408C3138BDA8114220F0B5C84C87B094F83E
S21444E050C2310133DAB21B064ABF002384F8C22118
S21444E06084F8C231B4F8C63113B1013BA4F8C631C2
S21444E07094F8A03123B1002384F8A031FFF798FA2E
S21444E08094F88A51012D40F0288194F888312E2B3B
S21444E0903DD146F60362A4F854206289A4F856207B
S21444E0A094F88D210D2A0BD1002384F88A3101235C
S21444E0B084F8953040F2F513A4F8BE3007B0F0BDAE
S21444E0C00E2AF4D194F88911A9480491A9490391D8
S21444E0D0B4F8CA10CDE9012194F8C5202946009227
S21444E0E0B4F88421FFF7A8FD94F88931012B03D1B5
S21444E0F0002001F064FAD7E7022B03D1002001F098
S21444E10079FAD1E7FF2BCFD184F8CB51CCE7222B39
S21444E110CAD1B4F88431B3F5A06F6BD1964D0022C2
S21444E120964915F8010B134601321F2892B204D9BA
S21444E130322A01F8010BF4D11346E2182C213A2076
S21444E14082F8E4105A1C422114FA82F282F8E4104F
S21444E1509A1C4F2114FA82F282F8E410DA1C14FA5C
S21444E16082F282F8E4101A1D542114FA82F282F8DC
S21444E170E4105A1D562114FA82F282F8E410991DCE
S21444E180DA1D14FA81F192B281F8E4007C490878E9
S21444E19042281FD022444E2182F8E41003F108029C
S21444E1A0302114FA82F282F8E41003F10A010933AA
S21444E1B0202289B214FA83F383F8E42063180022F9
S21444E1C001314FF4A06083F8E42089B26B4AFFF72C
S21444E1D001FF6CE70B466B4D1878114601321F2839
S21444E1E092B2EBD901332144AB4281F8E400F3D137
S21444E1F01146E3E7644EB4F8862106EB4316B4F8BA
S21444E20086C14FEA122E3789D0B29CFA9CFCF2683B
S21444E210FB1C99B2DBB207292FD984F85530C1F3D9
S21444E2200321622384F857E041F0100184F8580033
S21444E23084F85630002384F854100221A4F8CA30D7
S21444E240C4F89821A4F8CC701378A4F8CA5084F87B
S21444E25059305378A4F8CA1084F85A30937884F81E
S21444E2605B300323A4F8CA30FFF748FE322384F811
S21444E2708A1184F8C630212374E0622184F854302D
S21444E280A4F856C0013384F855100021C4F89821E8
S21444E290DBB2A4F8CA10A4F8CC701078A4F8CA501C
S21444E2A084F85800507884F859000220A4F8CA002C
S21444E2B0907884F85A000320A4F8CA00D27884F8E8
S21444E2C05B200422A4F8CA20DAB2082A3FF4ECAE53
S21444E2D0E218013382F85410F6E7022D7FF4EEAECE
S21444E2E094F8C530002B7FF4E9AE94F88831222B9D
S21444E2F07FF4DDAE94F8C430012B06D9023BDBB282
S21444E30084F8C430002B7FF4D9AE94F8C330072188
S21444E31094F88C212E27B4F8CC50D4F8986113483E
S21444E32084F8C43084F85420B4F8CA300139013033
S21444E330AB4238BF16F803C003F101032CBF80F884
S21444E340547080F854C09BB211F0FF01A4F8CA3050
S21444E350EAD19D4202F10103DBB298BF84F88A11E8
S21444E3602F2B88D884F88C31A1E600BFA811422010
S21444E370E68F460040134220000144008C1242209F
S21444E380201040003910400040874600FFF75CBE2E
S21444E39038B51B4C6389A4F89E31FFF713FE94F8F6
S21444E3A09E5105F0F703022B05D10123002584F87E
S21444E3B09D31284638BD012D0FD145F6061384F805
S21444E3C05650A4F8543094F89F3184F85730FFF7E9
S21444E3D0E9FA40BAA4F85800EBE7032D12BF47F613
S21444E3E0027345F6021384F856504FF001051BBFDE
S21444E3F0A4F854301223A4F8543084F85630D8E79E
S21444E400A811422008B5FFF7DDFD0B4B4CF2025233
S21444E410A3F854209A7A012A83F8562004D100227D
S21444E42083F8D421012008BD022A01D10122F7E74E
S21444E4307F2283F85520F5E7A8114220064B47F67D
S21444E4400372A3F85420012283F8560083F8571029
S21444E45083F89C21704700BFA8114220074B93F8CD
S21444E460D621132A09D093F8A521032A1FBF7F2259
S21444E47083F8D621012283F89C217047A8114220B4
S21444E480002310B56B4C84F8D63194F8CE30222B4A
S21444E49007D194F8D531032B09D0132384F8D63109
S21444E4A005E0202B14D194F8D531022BF5D894F8F6
S21444E4B0D63163B147F6037284F857300123A4F883
S21444E4C0542094F8CE2084F89C3184F8562010BD0D
S21444E4D0102B0BD194F8D531022BDED1A37A03F05E
S21444E4E07F03013B022BE2D91223D7E7852B12D1B7
S21444E4F0A37A013B012B84BF122384F8D63194F8C7
S21444E500D531022B02D0132384F8D63194F8D601A1
S21444E510FFF7A4FFCBE7272B05D194F8D53103F0BA
S21444E520FB03022BB8E7192B18D194F8D531012BED
S21444E530B3D0A27A0A2AF4D0032AF2D0022AAAD066
S21444E540042A08D1062BA8D1A37B012BAFD0FF2BDE
S21444E550ADD03123A2E7012AC6D19CE7282B1DD192
S21444E56094F8D511A27A032902F07F0305D0002B34
S21444E570C9D0032BC7D0022902D0591E0129C2D9BB
S21444E58012F07C0F01D01223BEE7E27A013A022A47
S21444E590BCD90BB1032BB9D13123B5E7142B1CD10D
S21444E5A094F8D531042B7FF478AFE07AA37A00EB65
S21444E5B00323207B00EB03206FF07F439842C4F88C
S21444E5C0D0013FF474AF1C4B98423FF470AFFFF752
S21444E5D067FAFF287FF46BAFBBE73E2B11D194F864
S21444E5E0D531022B7FF459AFA37A13F07F0F4FF443
S21444E5F0FA7318BF1222A4F8E43118BF84F8D6215F
S21444E60055E7312B09D194F8D531062B3FF645AF63
S21444E610A37A013B022B9CD849E72E2B05D194F8CC
S21444E620D531022B7FF639AF41E70F2B3FF63FAF8C
S21444E630112333E7A8114220FF0040004FF287130E
S21444E6409842134B0ED10A290AD1002283F8D621C8
S21444E65093F8D621003A18BF012283F8DB2170478D
S21444E6601322F3E74FF28B12904201D10429EBE7D1
S21444E6704FF29512904201D10329E5E74FF29312E7
S21444E6809042F9D04FF28C129042DED10729DBE754
S21444E690A81142200B4B024693F90A00997A0028A7
S21444E6A0B3BF01F07F02012083F855200020B8BF95
S21444E6B09A724FF00102A8BF83F8540083F8A5214C
S21444E6C0704700BFA8114220274B014610B593F966
S21444E6D00A009A7A0028BBBF02F07F02002001207D
S21444E6E09A729A7A541E022C31D8062483F855100E
S21444E6F0022A4FF0000183F854404FF4997483F88B
S21444E7005620A3F858404FF0F40483F8571083F883
S21444E7105A404FF4FA7483F8A521A3F8E44112D181
S21444E720124A1278422A06D102F5800202F6DF72B5
S21444E73012784F2A03D0012283F89C2103E0012259
S21444E740084683F8CA21002283F8CF2110BD47F635
S21444E7500372A3F8542093F8CE2083F8562012224E
S21444E76083F85720E7E700BFA81142202010400056
S21444E77010B5214CA37AE07A00EB032080B2B0F5C2
S21444E780754FA4F886010BD14FF4A063A4F88431E6
S21444E7900123002084F88A31222384F8883111E04A
S21444E7A0B0F5704F12D300F0A9FD4FF6FF739842B0
S21444E7B009D10223012084F85430637A43F040039D
S21444E7C084F8553010BDA4F88401E1E740F2DF73C5
S21444E7D0D4F8E001C01A47F60373A4F8543018BFBF
S21444E7E0012094F8CE3084F85630312384F85730DC
S21444E7F0012384F89C31E5E7A81142202DE9F04135
S21444E8004E4C2E23A27AE07A84F88831130900EB22
S21444E8100220217B0E2B84F88D3180B284F8891136
S21444E820A4F886010DD10123002084F88A3194F897
S21444E830DB31012B71D1424A626584F89C31BDE8D4
S21444E840F081B0F5704F13D300F0C3FD0F2302469A
S21444E850A4F8840184F88D314FF6FF73984204D0AF
S21444E860384E06EB4013D96921B9032384F8DB31CB
S21444E8700120DCE794F8CF11012901D00223F5E703
S21444E880002084F89C0194F8DB010028F0D19B68B2
S21444E89094F8D5010333DBB2984207D013232A48B1
S21444E8A084F8DB1184F8D631FFF7C6F9B4F884311E
S21444E8B00027DFF89C80042506EB4313A4F8CA70AF
S21444E8C0DA689B68C4F89421A4F8CC30B4F8CA300B
S21444E8D018F8011BD4F89421D154B4F8CA30B4F8CB
S21444E8E0CC2001339BB29A42A4F8CA30C0D9002047
S21444E8F0FFF7CAFA94F89C3184F8DB7143B9B4F84C
S21444E900843106EB4313DB69012B08BF84F8A1313D
S21444E910013D15F0FF05D9D1AAE7022B03D10B4BD5
S21444E9206365012389E7032B01BF03F1445303F5D1
S21444E930391303F57C53636581E700BFA811422071
S21444E940037F2E134087460037904600037F2E33BE
S21444E950B4114220204B014630B593F90A009A7A06
S21444E9600028BBBF02F07F02002001209A72DA7AA8
S21444E97002F0FD04012C22D19A7A02F0FD05012D05
S21444E98011D183F8DC5193F8A521012A4FF00202F5
S21444E99083F854201AD87F225A7222229A7200226E
S21444E9A083F8DC2130BD12B983F8DC21EBE7022A78
S21444E9B006BF002083F8DC4183F89C41E3E7022A43
S21444E9C01FBF7F225A7212229A72DCE79A7A83F821
S21444E9D0551083F85620E5E7A81142207047704743
S21444E9E07047704750B123230549013B00284FEA3E
S21444E9F040009BB2B8BF4840002BF6D1704700BFDA
S21444EA0069696C6CF8B56C4B064693F8A5211C46B0
S21444EA10012A0BD847F60372A3F854205A7A83F88F
S21444EA2056207F2283F8572001253DE0997A01F04D
S21444EA30FB05012D4AD1062384F8550084F8561068
S21444EA4084F8543094F8CF31012B2FD101292DD19D
S21444EA500023A4F8A631A4F8A83194F8A6610129A5
S21444EA6094F8A72194F8A83118BF022184F85820B6
S21444EA7002EB062294F8A90184F8593003EB0223EA
S21444EA8084F85A0000EB032084F85760FFF7AAFF87
S21444EA90030E84F8A631030C40BA84F8A731012348
S21444EAA0A4F8A80184F8C1312846F8BD94F8C231C8
S21444EAB003F1110284F8A63184F8A72103F1220257
S21444EAC0343384F8A82184F8A931C6E7022DABD1A3
S21444EAD093F8C121012A4FF0000210D083F8C121D7
S21444EAE047F603720125A3F8542093F8CE2083F802
S21444EAF09C5183F85620242283F85720D4E783F881
S21444EB00C121DA7A93F8A6319A420AD1227B94F844
S21444EB10A7319A4205D1B4F8A821B4F80D309A42E8
S21444EB201DD047F603730629A4F8543094F8CE3023
S21444EB3084F856304FF0350384F857304FF00103CD
S21444EB4084F89C317FF470AF1C4B1B78422B08D062
S21444EB5001231B4884F89C31FFF76EF801E0062930
S21444EB60F2D094F89C51002D7FF45EAFA37A02272E
S21444EB7084F8556084F8563084F85470FFF721F9C9
S21444EB80A37A062B0ED101230E4884F8CF7184F85D
S21444EB90CA31FFF748F80B48FFF745F80948FFF72E
S21444EBA042F881E794F8A531023B012B9CBF012330
S21444EBB084F8CF3178E700BFA811422020104000E7
S21444EBC04B904600A9904600114B002293F89C11A6
S21444EBD083F8D621012904BF7F2183F89C2193F82A
S21444EBE0CE2008BF83F85510312A0DD193F8D5119D
S21444EBF0062903D9132283F8D62103E0997A0139EA
S21444EC000229F8D801207047342AFBD11222F2E7B1
S21444EC10A811422070B5674C0025637A264694F8BE
S21444EC20DD2184F8CE30237A84F89C519A4284F8C5
S21444EC30D53101D800200FE0013B062BFAD8FFF768
S21444EC401FFC94F89C31012B0FD1D4F8E02140F2FC
S21444EC50DF739A4201D0012070BD94F8D631113B3F
S21444EC60012BF8D884F89C51E4E7627A94F8CE30C5
S21444EC70102A43F0400003D1BDE87040FFF724BD9E
S21444EC80202A03D1BDE87040FFF704BD852A03D18E
S21444EC90BDE87040FFF7B6BB2A2B0AD1E37A84F866
S21444ECA0C33146F60223A4F85430A37A84F8563087
S21444ECB0D1E7222B04D16220BDE87040FFF758BD4F
S21444ECC02E2B04D16E20BDE87040FFF797BD282B4D
S21444ECD004D16820BDE87040FFF73CBE2F2B0ED110
S21444ECE046F60673344AA4F854300623013B12F819
S21444ECF0011B13F0FF0382F84B10F7D1ABE7142B3C
S21444ED0015D1FFF75FF9D4F8D0016FF07F439842EE
S21444ED1002D02A4B984207D1012386F8A03145F207
S21444ED200143A6F8543096E7FEF702FFF7E7272B91
S21444ED3004D16720BDE87040FFF764BE192B03D1A9
S21444ED40BDE87040FFF724BB312B0BD11C4A072388
S21444ED50013B12F8011B13F0FF0382F8DA10F7D1D7
S21444ED60712079E7112B0FD145F20213A4F85430E1
S21444ED70A37A84F85630FFF724F81248FEF753FF78
S21444ED801148FEF750FF66E73E2B0FD194F90A1060
S21444ED90A37A0029FFF64EAF022142F0400284F8DF
S21444EDA0563084F8541084F8552054E7FEF79CFFF8
S21444EDB040E700BFA8114220B2114220FF004000A5
S21444EDC0B1114220559046006A90460038B5424CF0
S21444EDD00F2384F88D312546237A217B03F00F02D6
S21444EDE0637AE07A03EB022304F1E40201EB0020A9
S21444EDF0C4F8942142F2030280B2A4F8CC30A4F8BA
S21444EE008A2194F8CE202F2A23D1033B2E22A4F81D
S21444EE107A019BB284F8882104F22F12A4F8860162
S21444EE20A4F8CC3084F87931A37BC4F8942184F8D0
S21444EE3031310423627BA4F8CA30E37B84F87C2116
S21444EE4084F82F1184F8302184F83231FFF748F8DB
S21444EE5014E0A4F8860100F051FA4FF6FF73984286
S21444EE600ED147F603723123A5F8542095F8CE20E8
S21444EE7085F8D63185F8562085F85730012038BDB8
S21444EE80164B03EB4013DA69002AEAD02E22A4F884
S21444EE90840184F88821032284F88A21DA689B68EE
S21444EEA0C4F89421A4F8CC300123A4F8CA30637B78
S21444EEB01370B4F8CA30D4F89421591CA4F8CA1074
S21444EEC0A17BD154B4F8CA30D4F89421591CA4F880
S21444EED0CA10E17BD154B9E7A811422040874600C6
S21444EEE008B51A4B0022197A83F88D2101F00F00D9
S21444EEF0597AA3F8842101EB00219A7AC82983F829
S21444EF0088211A7B88BFC82183F8E520A3F8CC1053
S21444EF10D97A02EB01205A7B83F8E41083F8E62082
S21444EF209A7BA3F8860142F2030083F8E720DA7B53
S21444EF30A3F88A0183F8E82005220548A3F8CA20E6
S21444EF40C3F89401FEF7CCFF012008BDA811422067
S21444EF503E224020184B0022987A83F8D62183F824
S21444EF609C21A0F12E0283F8CE00D1B208291DD8E8
S21444EF7040F24912CA40D24312F0010216D12E285A
S21444EF8083F8DB2114D193F8A521012A02D993F8FA
S21444EF90CF216AB97E2283F8D62102F17E2202F579
S21444EFA0381285325A65012283F89C210120704725
S21444EFB00020FFF70BBF00BFA8114220002340F2F9
S21444EFC0F51210B5884C84F8983084F89C31A4F82F
S21444EFD0BE204FF4FA72C4E915332368A4F8E4213A
S21444EFE0B3F5FA6F17D1431E04F10802073013F83D
S21444EFF0011F984202F8011BF9D14FF4FA63C4F892
S21444F000E031227A12F0F0032BD1FFF703FE0028FA
S21444F01040F08B804CE040F2DF72934220D103787C
S21444F02013F0F00F1CD14278A2F11003DBB2182B78
S21444F03011D9852A01D03E2A12D140F2DF736B4A99
S21444F040C4F8E031431E073013F8011F834202F828
S21444F050011BF9D1D5E7664A22FA03F3DB07ECD461
S21444F06010BD102B02D1FFF775FFD0E7202B40F0E0
S21444F0708F8094F8CE302E3BD9B206295CD84923EB
S21444F080CB40DB4313F0010356D194F88A1103298D
S21444F0900ED194F8DD11072910D8B4F8CA300139D6
S21444F0A01944B4F8CC30994202D2002384F88A3109
S21444F0B0002384F89C3184F89830D1E794F88B1177
S21444F0C0914205D14B4884F88A31FEF7ACFDEFE710
S21444F0D084F88B210D2284F8C72094F8DB2132B9BA
S21444F0E0E218D4F89411507AB4F8CA208854B4F884
S21444F0F0CA20B4F8CC10013292B29142A4F8CA2085
S21444F10042D894F8DB31012B1AD147F60372A4F89F
S21444F110542094F8CE2084F85620132284F857209E
S21444F12084F89C31002384F8DB3194F89C31012B1D
S21444F13004BF7F2384F85530012384F89530B7E71D
S21444F140022B0CD147F60373A4F8543094F8CE300F
S21444F15084F85630332384F857300123E0E7002000
S21444F160FEF792FEB4F88421234B94F89C1103EBEB
S21444F17042132248DA69012A08BF84F8A12194F888
S21444F180A131FEF759FDCDE70133072BA5D18FE713
S21444F190302B8DD194F8DD31022B86D9312A03D118
S21444F1A00B2384F8C63083E794F8C5305BB9322A1B
S21444F1B009D146F20323A4F85430B4F886315BBA36
S21444F1C0A4F856304CE7A37A0021312A03F103030E
S21444F1D084F8C51084F8C610DBB284F8C33084F8CB
S21444F1E0C4303FF662AF63E7A8114220B011422014
S21444F1F0130204017A9046004087460092904600E7
S21444F2000A4810B5FEF718FD72B64FF00053084989
S21444F2101022084C0848C3E90012FEF70DFDF2F729
S21444F22000FB2046FEF708FDFBE700BFA49046001F
S21444F2307154CA3DCB904600B190460038B52C4B2D
S21444F24093F8C8211C4632B9FEF7D6FD2948BDE8D6
S21444F2503840FEF7E8BC93F89820002A3FD00022B6
S21444F26093F89D1183F8982081B193F89E0183F812
S21444F2709D21FEF74DFE012384F8953040F2F513A8
S21444F280A4F8BE30BDE83840FEF79BBD93F89550D1
S21444F290002DF3D1184A13780133DBB2022B01D880
S21444F2A0137038BD1570FEF7CFFE94F8993094F875
S21444F2B0C22101330132DBB284F8C221042B84F824
S21444F2C099300CD984F89950FEF718FDB4F89C3060
S21444F2D0C72B96BF0133A4F89C50A4F89C3094F8EE
S21444F2E0CA2194F8CB311343DBD0FFF789FF00BF24
S21444F2F0A8114220DA904600042240204FF2280308
S21444F300984218D84FF20F03984259D9A0F5704046
S21444F310113817280DD8DFE800F056292B2D2F3149
S21444F32031333537393B3D3F4143454547494B4D9E
S21444F3304F51042070474FF29313984245D00CD84F
S21444F3404FF28713984242D04FF288124FF6FF731B
S21444F350904214BF1846012070474FF295124FF65C
S21444F360FF73904214BF1846022070470620704729
S21444F3700720704708207047092070470A207047C6
S21444F3800B2070470C2070470D2070470E207047A6
S21444F3900F20704710207047112070471220704786
S21444F3A01320704714207047152070471620704766
S21444F3B01720704718207047192070471A20704746
S21444F3C04FF6FF70704705207047032070470020B3
S21444F3D07047FFF793BF1C280146F0B585B037D871
S21444F3E03F4B420103EB40169C584FF6FF739C423A
S21444F3F02ED0F369012B2BD1756804F50004B3684D
S21444F400AD082246009337482B46FEF715FCD6E94E
S21444F41003639A1E012A1DD8002315E036F82310EC
S21444F420023389B2029102990904029150880299E2
S21444F43001440291918889B2039103990904039186
S21444F440D188039A0A4403929D4206EB8302E5D888
S21444F45005B0F0BD043B012B3FD90027BD4206EB67
S21444F4608701F5D916F82730204602370834DBB230
S21444F4700293029B1B0602934A78029B03EB0243C9
S21444F48002938A78029B03EB02230293CB78029A78
S21444F490134402930B79DBB20393039B1B0603933B
S21444F4A04A79039B03EB024303938A79039B03EB5A
S21444F4B002230393CB7902A9039A13440393FEF7DA
S21444F4C010FCCBE756F8231002330291526803929D
S21444F4D09D4206EB8302F5D8BAE70023F8E700BF5F
S21444F4E040874600E59046001C28014630B403D9C0
S21444F4F02C4830BCFEF7A0BB42012B4B03EB40101C
S21444F5009B584FF6FF7293421FD0C269012A1CD102
S21444F5100169072919D0826803F50003C468881E68
S21444F520012814D852080234002191420DD253F8CF
S21444F530040B050C24F8025C4D1C954205D202319E
S21444F54080B28A4224F8040BEFD830BC70470439A2
S21444F550012925D822F0030222449442F5D053F8D8
S21444F560041B44F8041BF8E75858050E25704D1C38
S21444F570AA42EAD9C0F3074565708D1CAA42E4D96D
S21444F580C0F30725A570CD1CAA42DED90431C0B20B
S21444F59004348A4204F8010CD7D99142E4D3D4E720
S21444F5A00021FAE7069146004087460010B500243D
S21444F5B0A0B20134FFF798FF1D2CF9D110BD1FB53A
S21444F5C00024A0B20134FFF706FF1D2CF9D1074BE7
S21444F5D002A902934FF47C730393054B019301985D
S21444F5E0FEF77FFB002004B010BD00BF55EFCDAB47
S21444F5F01000800008B508B9FFF7D8FF002008BD02
S21444F600124B00B51B688BB00293114B1A680392D9
S21444F6105A6804929B6805930299039A049B05983A
S21444F62000900C48FEF708FB039BB3F57C7F06D19D
S21444F6300948FEF701FB01200BB05DF804FB0748C0
S21444F640FEF7FAFA4FF0FF30F6E700BF10008000EE
S21444F65014008000169146002E91460039914600CB
S21444F66008B5FFF7CDFF012805D1FFF79FFFBDE89A
S21444F6700840FDF7B9BFFFF7C3FF0128F5D00020C7
S21444F680FFF79DFFFFF7BCFFF1E700BF10F8012B23
S21444F69011F8013B012A28BF9A42F7D0D01A704786
S21444F6A0034613F8012B002AFBD1181A0138704779
S21444F6B001F0FF01102A2BDB10F0070F08D010F8DA
S21444F6C0013B013A8B422DD010F0070F42B3F6D1DE
S21444F6D0F0B441EA012141EA014122F007047FF0F7
S21444F6E000070023F0E80256083C85EA010586EA4E
S21444F6F0010685FA47F5A3FA87F586FA47F6A5FA8A
S21444F70087F68EB9EED1F0BC01F0FF0102F0070295
S21444F71032B110F8013B013A83EA010313B1F8D140
S21444F7200020704701387047002D06BF3546033821
S21444F730073815F0010F07D1013015F4807F02BF5A
S21444F740013015F4C03F0130F0BC0138704700BFAB
S21444F75081F0004102E000BF83F0004330B54FEA39
S21444F76041044FEA430594EA050F08BF90EA020FA6
S21444F7701FBF54EA000C55EA020C7FEA645C7FEA39
S21444F780655C00F0E2804FEA5454D4EB5555B8BF5C
S21444F7906D420CDD2C4480EA020281EA030382EACD
S21444F7A0000083EA010180EA020281EA0303362D5F
S21444F7B088BF30BD11F0004F4FEA01314FF4801C32
S21444F7C04CEA113102D0404261EB410113F0004F44
S21444F7D04FEA03334CEA133302D0524263EB4303FB
S21444F7E094EA050F00F0A780A4F10104D5F1200E99
S21444F7F00DDB02FA0EFC22FA05F2801841F10001F4
S21444F80003FA0EF2801843FA05F359410EE0A5F1C7
S21444F81020050EF1200E012A03FA0EFC28BF4CF0F8
S21444F820020C43FA05F3C01851EBE37101F00045AE
S21444F83007D54FF0000EDCF1000C7EEB00006EEBBB
S21444F8400101B1F5801F1BD3B1F5001F0CD3490845
S21444F8505FEA30004FEA3C0C04F101044FEA44529C
S21444F86012F5800F80F09A80BCF1004F08BF5FEA23
S21444F870500C50F1000041EB045141EA050130BD03
S21444F8805FEA4C0C404141EB0101013C28BFB1F515
S21444F890801FE9D291F0000F04BF01460020B1FA60
S21444F8A081F308BF2033A3F10B03B3F120020CDA33
S21444F8B00C3208DD02F1140CC2F10C0201FA0CF011
S21444F8C021FA02F10CE002F11402D8BFC2F1200C76
S21444F8D001FA02F120FA0CFCDCBF41EA0C0190402C
S21444F8E0E41AA2BF01EB0451294330BD6FEA040475
S21444F8F01F3C1CDA0C340EDC04F11404C4F1200260
S21444F90020FA04F001FA02F340EA030021FA04F371
S21444F91045EA030130BDC4F10C04C4F1200220FAC8
S21444F92002F001FA04F340EA0300294630BD21FA06
S21444F93004F0294630BD94F0000F83F4801306BFCC
S21444F94081F480110134013D4EE77FEA645C18BFC0
S21444F9507FEA655C29D094EA050F08BF90EA020F57
S21444F96005D054EA000C04BF1946104630BD91EA4F
S21444F970030F1EBF0021002030BD5FEA545C05D152
S21444F9804000494128BF41F0004130BD14F5800491
S21444F9903CBF01F5801130BD01F0004545F0FE4105
S21444F9A041F470014FF0000030BD7FEA645C1ABF3A
S21444F9B0194610467FEA655C1CBF0B46024650EA71
S21444F9C0013406BF52EA033591EA030F41F400219D
S21444F9D030BD00BF90F0000F04BF0021704730B523
S21444F9E04FF4806404F132044FF000054FF00001F8
S21444F9F050E700BF90F0000F04BF0021704730B5B9
S21444FA004FF4806404F1320410F0004548BF40428D
S21444FA104FF000013EE700BF42004FEAE2014FEAE2
S21444FA2031014FEA02701FBF12F07F4393F07F4FBD
S21444FA3081F06051704732F07F4208BF704793F0C0
S21444FA407F4F04BF41F40021704730B54FF46074D3
S21444FA5001F0004521F000411CE700BF50EA0102D6
S21444FA6008BF704730B54FF000050AE050EA01027F
S21444FA7008BF704730B511F0004502D5404261EBEF
S21444FA8041014FF4806404F132045FEA915C3FF430
S21444FA90D8AE4FF003025FEADC0C18BF03325FEACD
S21444FAA0DC0C18BF033202EBDC02C2F1200300FA7E
S21444FAB003FC20FA02F001FA03FE40EA0E0021FAA3
S21444FAC002F11444BDE600BF70B54FF0FF0C4CF491
S21444FAD0E06C1CEA11541DBF1CEA135594EA0C0F43
S21444FAE095EA0C0F00F0DEF82C4481EA030621EA7E
S21444FAF04C5123EA4C5350EA013518BF52EA0335B9
S21444FB0041F4801143F4801338D0A0FB02CE4FF06A
S21444FB100005E1FB02E506F00042E0FB03E54FF09A
S21444FB200006E1FB03569CF0000F18BF4EF0010E92
S21444FB30A4F1FF04B6F5007F64F5407404D25FEA8E
S21444FB404E0E6D4146EB060642EAC62141EA555141
S21444FB504FEAC52040EA5E504FEACE2EB4F1FD0C83
S21444FB6088BFBCF5E06F1ED8BEF1004F08BF5FEA01
S21444FB70500E50F1000041EB045170BD06F00046B3
S21444FB8046EA010140EA020081EA0301B4EB5C0460
S21444FB90C2BFD4EB0C0541EA045170BD41F4801158
S21444FBA04FF0000E013C00F3AB8014F1360FDEBF7D
S21444FBB0002001F0004170BDC4F10004203C35DA59
S21444FBC00C341BDC04F11404C4F1200500FA05F3DC
S21444FBD020FA04F001FA05F240EA020001F000427D
S21444FBE021F0004110EBD37021FA04F642EB0601F3
S21444FBF05EEA430E08BF20EAD37070BDC4F10C041D
S21444FC00C4F1200500FA04F320FA05F001FA04F2E0
S21444FC1040EA020001F0004110EBD37041F10001CC
S21444FC205EEA430E08BF20EAD37070BDC4F12005D7
S21444FC3000FA05F24EEA020E20FA04F301FA05F23F
S21444FC4043EA020321FA04F001F0004121FA04F2E7
S21444FC5020EA020000EBD3705EEA430E08BF20EAB7
S21444FC60D37070BD94F0000F0FD101F000464000F1
S21444FC7041EB010111F4801F08BF013CF7D041EA73
S21444FC80060195F0000F18BF704703F00046520077
S21444FC9043EB030313F4801F08BF013DF7D043EA48
S21444FCA00603704794EA0C0F0CEA135518BF95EAFE
S21444FCB00C0F0CD050EA410618BF52EA4306D1D185
S21444FCC081EA030101F000414FF0000070BD50EAA4
S21444FCD0410606BF1046194652EA430619D094EA2E
S21444FCE00C0F02D150EA013613D195EA0C0F05D118
S21444FCF052EA03361CBF104619460AD181EA03016C
S21444FD0001F0004141F0FE4141F470014FF0000023
S21444FD1070BD41F0FE4141F4780170BD70B54FF0BE
S21444FD20FF0C4CF4E06C1CEA11541DBF1CEA13553E
S21444FD3094EA0C0F95EA0C0F00F0A7F8A4EB050420
S21444FD4081EA030E52EA03354FEA013100F0888017
S21444FD504FEA03334FF0805545EA131343EA1263E0
S21444FD604FEA022245EA111545EA10654FEA002695
S21444FD700EF000419D4208BF964244F1FD0404F54E
S21444FD80407402D25B084FEA3202B61A65EB0305AA
S21444FD905B084FEA32024FF480104FF4002CB6EB67
S21444FDA0020E75EB030E22BFB61A754640EA0C00E7
S21444FDB05B084FEA3202B6EB020E75EB030E22BF27
S21444FDC0B61A754640EA5C005B084FEA3202B6EB68
S21444FDD0020E75EB030E22BFB61A754640EA9C0027
S21444FDE05B084FEA3202B6EB020E75EB030E22BFF7
S21444FDF0B61A754640EADC0055EA060E18D04FEAB5
S21444FE00051545EA16754FEA06164FEAC30343EA54
S21444FE1052734FEAC2025FEA1C1CC0D111F4801F21
S21444FE200BD141EA00014FF000004FF0004CB6E71A
S21444FE3011F4801F04BF01430020B4F1FD0C88BFB9
S21444FE40BCF5E06F3FF6AFAEB5EB030C04BFB6EBC4
S21444FE50020C5FEA500C50F1000041EB045170BDB7
S21444FE600EF0004E4EEA113114EB5C04C2BFD4EBE4
S21444FE700C0541EA045170BD41F480114FF0000E68
S21444FE80013C90E645EA060E8DE60CEA135594EAE4
S21444FE900C0F08BF95EA0C0F3FF43BAF94EA0C0FE7
S21444FEA00AD150EA01347FF434AF95EA0C0F7FF45C
S21444FEB025AF104619462CE795EA0C0F06D152EAB0
S21444FEC003353FF4FDAE1046194622E750EA410694
S21444FED018BF52EA43067FF4C5AE50EA41047FF4A5
S21444FEE00DAF52EA43057FF4EBAE12E74FF0FF3C0A
S21444FEF006E000BF4FF0010C02E000BF4FF0010CDB
S21444FF004DF804CD4FEA410C7FEA6C5C4FEA430C53
S21444FF1018BF7FEA6C5C1BD001B050EA410C0CBFA2
S21444FF2052EA430C91EA030F02BF90EA020F002004
S21444FF30704710F1000F91EA030F58BF994208BF6B
S21444FF4090422CBFD8176FEAE37040F00100704728
S21444FF504FEA410C7FEA6C5C02D150EA013C07D17F
S21444FF604FEA430C7FEA6C5CD6D152EA033CD3D0CA
S21444FF705DF8040B704700BF8446104662468C46C4
S21444FF801946634600E000BF01B5FFF7B7FF0028F7
S21444FF9048BF10F1000F01BD4DF808EDFFF7F4FF20
S21444FFA00CBF012000205DF808FB00BF4DF808EDAB
S21444FFB0FFF7EAFF34BF012000205DF808FB00BFCE
S21444FFC04DF808EDFFF7E0FF94BF012000205DF8F0
S21444FFD008FB00BF4DF808EDFFF7CEFF94BF0120A5
S21444FFE000205DF808FB00BF4DF808EDFFF7C4FF9E
S21444FFF034BF012000205DF808FB00BF4FEA410CE7
S2144500007FEA6C5C02D150EA013C0AD14FEA430CC8
S2144500107FEA6C5C02D152EA033C02D14FF0000005
S21445002070474FF0010070474FEA410212F5001243
S21445003015D211D56FF47873B3EB625212D94FEAE5
S214450040C12343F0004343EA505311F0004F23FACF
S21445005002F018BF404270474FF00000704750EA24
S214450060013005D111F0004008BF6FF000407047E1
S2144500704FF00000704700BF4A0011D212F500123B
S21445008011D20DD56FF47873B3EB62520ED44FEAA6
S214450090C12343F0004343EA505323FA02F0704726
S2144500A04FF00000704750EA013002D14FF0FF3064
S2144500B070474FF0000070474FEA4102B2F1E04307
S2144500C024BFB3F5001CDCF1FE5C0DD901F0004CF5
S2144500D04FEAC0024CEA5070B2F1004F40EB830045
S2144500E008BF20F00100704711F0804F21D113F171
S2144500F03872BCBF01F00040704741F480114FEAAA
S2144501005252C2F11802C2F1200C10FA0CF320FA32
S21445011002F018BF40F001004FEAC1234FEAD3234F
S21445012003FA0CFC40EA0C0023FA02F34FEA4303B9
S214450130CCE77FEA625307D150EA01331EBF4FF042
S214450140FE4040F44000704701F0004040F0FE405D
S21445015040F40000704700BF80F0004002E000BF5A
S21445016081F0004142001FBF5FEA410392EA030F58
S2144501707FEA226C7FEA236C6AD04FEA1262D2EBA2
S2144501801363C1BFD218414048404140B8BF5B42A7
S214450190192B88BF704710F0004F40F4000020F040
S2144501A07F4018BF404211F0004F41F4000121F056
S2144501B07F4118BF494292EA030F3FD0A2F10102A0
S2144501C041FA03FC10EB0C00C3F1200301FA03F1DE
S2144501D000F0004302D5494260EB4000B0F5000F01
S2144501E013D3B0F1807F06D340084FEA310102F1C0
S2144501F00102FE2A51D2B1F1004F40EBC25008BF72
S21445020020F0010040EA03007047490040EB00003B
S214450210013A28BFB0F5000FEDD2B0FA80FCACF13C
S214450220080CB2EB0C0200FA0CF0AABF00EBC25069
S21445023052421843BCBFD0401843704792F0000F57
S21445024081F4000106BF80F400000132013BB5E7AA
S2144502504FEA41037FEA226C18BF7FEA236C21D020
S21445026092EA030F04D092F0000F08BF0846704785
S21445027090EA010F1CBF0020704712F07F4F04D153
S214450280400028BF40F00040704712F100723CBF66
S21445029000F50000704700F0004343F0FE4040F490
S2144502A0000070477FEA226216BF08467FEA23634E
S2144502B00146420206BF5FEA412390EA010F40F439
S2144502C0800070474FF0000304E000BF10F0004385
S2144502D048BF40425FEA000C08BF704743F096436C
S2144502E001464FF000001CE050EA010208BF704787
S2144502F04FF000030AE000BF50EA010208BF70470E
S21445030011F0004302D5404261EB41015FEA010C22
S21445031002BF84460146002043F0B64308BFA3F11A
S2144503208053A3F50003BCFA8CF2083AA3EBC253FC
S21445033010DB01FA02FC634400FA02FCC2F120021B
S214450340BCF1004F20FA02F243EB020008BF20F052
S2144503500100704702F1200201FA02FCC2F12002B8
S21445036050EA4C0021FA02F243EB020008BF20EAAD
S214450370DC7070474FF0FF0C1CEAD0521EBF1CEADB
S214450380D15392EA0C0F93EA0C0F6FD01A4480EAC9
S214450390010C400218BF5FEA41211ED04FF00063B2
S2144503A043EA501043EA5111A0FB01310CF00040DE
S2144503B0B1F5000F3EBF490041EAD3715B0040EA04
S2144503C0010062F17F02FD2A1DD8B3F1004F40EBD4
S2144503D0C25008BF20F00100704790F0000F0CF0A7
S2144503E0004C08BF49024CEA502040EA51207F3A6B
S2144503F0C2BFD2F1FF0340EAC250704740F4000046
S2144504004FF00003013A5DDC12F1190FDCBF00F036
S21445041000407047C2F10002410021FA02F1C2F1E4
S214450420200200FA02FC5FEA310040F1000053EA80
S2144504304C0308BF20EADC70704792F0000F00F0CE
S214450440004C02BF400010F4000F013AF9D040EAD4
S2144504500C0093F0000F01F0004C02BF490011F468
S214450460000F013BF9D041EA0C018FE70CEAD15366
S21445047092EA0C0F18BF93EA0C0F0AD030F0004CE6
S21445048018BF31F0004CD8D180EA010000F000409A
S214450490704790F0000F17BF90F0004F084691F058
S2144504A0000F91F0004F14D092EA0C0F01D1420292
S2144504B00FD193EA0C0F03D14B0218BF084608D15B
S2144504C080EA010000F0004040F0FE4040F40000A5
S2144504D0704740F0FE4040F4400070474FF0FF0C38
S2144504E01CEAD0521EBF1CEAD15392EA0C0F93EA7F
S2144504F00C0F69D0A2EB030280EA010C49024FEAD1
S214450500402037D04FF0805343EA111143EA101389
S2144505100CF000408B4238BF5B0042F17D024FF441
S214450520000C8B4224BF5B1A40EA0C00B3EB510F1C
S21445053024BFA3EB510340EA5C00B3EB910F24BF05
S214450540A3EB910340EA9C00B3EBD10F24BFA3EB8A
S214450550D10340EADC001B0118BF5FEA1C1CE0D152
S214450560FD2A3FF650AF8B4240EBC25008BF20F005
S214450570010070470CF0004C4CEA50207F32C2BF59
S214450580D2F1FF0340EAC250704740F400004FF0F6
S2144505900003013A37E792F0000F00F0004C02BF27
S2144505A0400010F4000F013AF9D040EA0C0093F0F1
S2144505B0000F01F0004C02BF490011F4000F013B4B
S2144505C0F9D041EA0C0195E70CEAD15392EA0C0FB3
S2144505D008D142027FF47DAF93EA0C0F7FF470AFEB
S2144505E0084676E793EA0C0F04D14B023FF44CAF2E
S2144505F008466EE730F0004C18BF31F0004CCAD1C3
S21445060030F000427FF45CAF31F000437FF43CAFFE
S2144506105FE700BF4FF0FF3C06E000BF4FF0010C20
S21445062002E000BF4FF0010C4DF804CD4FEA400202
S2144506304FEA41037FEA226C18BF7FEA236C11D04C
S21445064001B052EA530C18BF90EA010F58BFB2EBFF
S214450650030088BFC81738BF6FEAE17018BF40F07F
S214450660010070477FEA226C02D15FEA402C05D133
S2144506707FEA236CE4D15FEA412CE1D05DF8040BB8
S214450680704700BF844608466146FFE70FB5FFF74B
S214450690C9FF002848BF10F1000F0FBD4DF808ED03
S2144506A0FFF7F4FF0CBF012000205DF808FB00BFF4
S2144506B04DF808EDFFF7EAFF34BF012000205DF84E
S2144506C008FB00BF4DF808EDFFF7E0FF94BF01209B
S2144506D000205DF808FB00BF4DF808EDFFF7D2FF98
S2144506E094BF012000205DF808FB00BF4DF808EDDB
S2144506F0FFF7C8FF34BF012000205DF808FB00BFA8
S21445070042000ED2B2F1FE4F0BD34FF09E03B3EB31
S214450710126209D44FEA002343F0004323FA02F05D
S21445072070474FF00000704712F1610F01D1420249
S21445073002D14FF0FF3070474FF00000704700BFC2
S21445074053B94AB9002908BF00281CBF4FF0FF31EE
S2144507504FF0FF3000F0A6B9ADF1080C6DE904CEB8
S21445076000F03EF8DDF804E0DDE9022304B070470A
S21445077038B505460C462846214600220023FFF795
S21445078015FC28B928462146BDE8384000F00AB889
S214450790284604F1004100F005F8404261EB41016E
S2144507A038BD00BFD0B50C4B002206460F46FFF7B6
S2144507B08BF9FFF761FC0446FFF70CF9074B00225F
S2144507C0FFF782F902460B4630463946FEF7C4FF28
S2144507D0FFF752FC2146D0BD0000F03D0000F04139
S2144507E02DE9F047089D0E4604468C46002B40F002
S2144507F081808A42174645D9B2FA82F24AB1C2F199
S214450800200106FA02F320FA01F1974041EA030C6B
S21445081094404FEA174E230CBCFBFEF6B9B20EFBCE
S21445082016CC43EA0C4306FB01F0984209D9FB185F
S21445083006F1FF3C80F01581984240F21281023E57
S2144508403B441B1AA4B2B3FBFEF00EFB103344EA3E
S214450850034400FB01F1A14209D93C1900F1FF33DD
S21445086080F00181A14240F2FE8002383C44641A81
S21445087040EA064000211DB1D4400023C5E90043A7
S214450880BDE8F08702B9FFDEB2FA82F2002A4FD100
S214450890CB1B4FEA174E1FFA87F80121B3FBFEFC28
S2144508A0260C0EFB1C3346EA034608FB0CF3B34204
S2144508B007D9BE190CF1FF3002D2B34200F2EB80E5
S2144508C08446F61AA3B2B6FBFEF00EFB106643EA64
S2144508D0064408FB00F8A04507D93C1900F1FF334C
S2144508E002D2A04500F2D2801846A4EB080440EA9E
S2144508F00C40C0E78B4208D9002D00F0AF800021A0
S214450900C5E900060846BDE8F087B3FA83F1002935
S21445091049D1B34202D3824200F2BB80841A66EBC9
S214450920030301209C46002DAAD0C5E9004CA7E745
S214450930C2F120039740D8409140DE404FEA174E1B
S21445094008434FEA104CB6FBFEF11FFA87F80EFB3C
S21445095011664CEA064601FB08F3B34204FA02F474
S21445096009D9BE1901F1FF3C80F08E80B34240F2B2
S2144509708B8002393E44F31A86B2B3FBFEF00EFB7B
S214450980103346EA034600FB08F3B34207D9BE19BF
S21445099000F1FF3C74D2B34272D902383E44F31A92
S2144509A040EA01417AE7C1F1200703FA01F422FA49
S2144509B007F31C4320FA07F906FA01F34FEA144CED
S2144509C0FE4049EA03094FEA1943B6FBFCFE1FFA07
S2144509D084F80CFB1E6643EA06460EFB08FAB2454B
S2144509E002FA01F200FA01F308D9A6190EF1FF3012
S2144509F048D2B24546D9AEF1020E2644A6EB0A06C3
S214450A001FFA89F9B6FBFCF00CFB106649EA064668
S214450A1000FB08F8B04507D9A61900F1FF3C2DD2D2
S214450A20B0452BD90238264440EA0E40A6EB0806C8
S214450A30A0FB02894E45C446CE4618D315D075B39D
S214450A40B3EB0C0266EB0E0606FA07F722FA01F33D
S214450A50CE401F43C5E90076002111E729462846C2
S214450A600EE76646EDE6184601E74345E7D2B8EB9E
S214450A70020C69EB04040138A646E0E76046D3E776
S214450A8060468CE78646B9E7614674E702383C44DB
S214450A902BE7084647E7ACF1020C3E4411E72946EA
S214450AA0EEE600BF704700BF2DE9F04788B0002B43
S214450AB01F461446B8BF03F10043129A109DDDF851
S214450AC04CA0B6BF1F4600232D231370149B23F05E
S214450AD02008B8F1460F05D0B8F1450F00D10135CD
S214450AE0022300E0032307AA049206AACDE902A240
S214450AF0CDE9003522463B4601F0A6FDB8F1470F45
S214450B00064602D1119BDB0722D5B8F1460F06EB08
S214450B10050910D13378302B0AD100220023204610
S214450B203946FFF739FA18B9C5F10105CAF8005034
S214450B30DAF8003099440022002320463946FFF76C
S214450B402BFA08B1CDF81C903022079B4B4507D3AE
S214450B50079B159A9B1B3046136008B0BDE8F08787
S214450B60591C07911A70F0E7F7B503460029B8BF38
S214450B70494203F8022BB4BF2D222B220929427085
S214450B802ADD0DF10704A4460A27A6460A4691FB28
S214450B90F7F607FB16153035632A04F1FF340EF8D1
S214450BA0015C3146F1DC3031AEF1020504F8011C3A
S214450BB0441C294661450AD30DF10902A2EB0E02F3
S214450BC0654588BF00221344181A03B0F0BD11F8D6
S214450BD0012B04F8012FEDE7302330318370C170C7
S214450BE0031DF1E72DE9F04F91B00C46DDF868801E
S214450BF016461F46054602F04DFE036809931846FD
S214450C00FEF74EFD00230E93D8F800300A900733C2
S214450C1023F0070303F1080294F81890D4F800B0BF
S214450C20C8F80020D3E90023C4E91223D4E9128A80
S214450C302AF000430B930B999C4B4FF0FF324046EE
S214450C40FFF7DCF970BB994B0B994FF0FF324046E6
S214450C50FFF7B6F930BB0022002340465146FFF762
S214450C60A5F910B12D2384F84330914B9148B9F13D
S214450C70470F94BF98468046032323612BF0040311
S214450C8023604FF0000A009733460FAA21462846B0
S214450C9000F0D2F9013040F08F804FF0FF3011B0B0
S214450CA0BDE8F08F4246534640465146FFF7A6F903
S214450CB040B1BAF1000FBCBF2D2384F843307E48BF
S214450CC07E4BD4E763685A1C09F0DF0142D1062300
S214450CD06360002206920EAACDE904920DAA4BF453
S214450CE0806303920DF13302CDE9013223606368D8
S214450CF000934246534628460B91FFF7D5FE0B997F
S214450D00472980460D9908D1C81C02DB636899427D
S214450D1040DDA9F102095FFA89F9B9F1650F1FD8D7
S214450D2001394A4604F150000D91FFF71DFF0E9A12
S214450D301318012A8246236102DC2268D20701D5B0
S214450D40013323619DF83330002B9CD02D2384F846
S214450D50433098E74729BCD1002BBAD10123B7E7E2
S214450D60B9F1660F18D1002963680BDD216113B907
S214450D702268D00702D501330B442361A1654FF0A5
S214450D80000ADFE713B92268D20701D50233F4E734
S214450D900123F2E74FF067090E9B994205DB23686E
S214450DA02161D807EAD54B1CE7E70029D4BFC1F136
S214450DB0020201221344E0E723685A0507D4236953
S214450DC0424631462846B84701302BD165E7B9F14A
S214450DD0650F40F2DC80D4E9120100220023FFF7BC
S214450DE0DBF8002833D0364A012331462846B84733
S214450DF001303FF452AFDDE90D239A4202DB23680A
S214450E00D8070FD5DDE9092331462846B8470130CE
S214450E103FF443AF4FF0000804F11A090E9B013B1F
S214450E20434509DC23689B0700F10181E0680F9B79
S214450E309842B8BF184632E701234A463146284607
S214450E40B84701303FF429AF08F10108E6E70D9BA6
S214450E50002B37DC1A4A012331462846B84701306D
S214450E603FF41BAFDDE90D23134302D12368D907B1
S214450E70D8D5DDE9092331462846B84701303FF441
S214450E800CAF4FF0000904F11A0A0D9B5B424B4527
S214450E9001DC0E9B94E70123524631462846B84767
S214450EA001303FF4FAAE09F10109EEE7FFFFEF7FA7
S214450EB0469146004A914600529146004E9146005C
S214450EC0569146000E9AA36D9A42A8BF1A46002A26
S214450ED0914637DC4FF0000B29EAE97904F11A020E
S214450EE0D4F858A0AAEB09035B4533DCDDE90D23AE
S214450EF09A423BDB2368DA0738D40E9A0D99A2EB63
S214450F000A03A2EB01099945A8BF9946B9F1000F16
S214450F1034DC4FF0000829EAE97904F11A0ADDE9DC
S214450F200D239B1AA3EB090343457FF77BAF0123AC
S214450F30524631462846B84701303FF4AEAE08F132
S214450F400108ECE71346314642462846B847013085
S214450F50C0D1A2E60123314628460B92B847013058
S214450F603FF49BAE0B9A0BF1010BB9E7DDE909237C
S214450F7031462846B8470130BFD18EE64B4608EB8A
S214450F800A0231462846B8470130C2D185E60E9A50
S214450F90012A01DCDB0737D5012342463146284680
S214450FA0B84701303FF479AEDDE909233146284696
S214450FB0B84701303FF471AED4E912010022002350
S214450FC0FEF7EAFFD8B90E9B08F10102013B314610
S214450FD02846B84701300ED15FE601234A463146DA
S214450FE02846B84701303FF458AE08F101080E9B35
S214450FF0013B4345F1DC534604F15002E1E64FF030
S214451000000804F11A09F2E701234246DFE7012307
S2144510104A4631462846B84701303FF43EAE08F1C9
S2144510200108E3680F995B1A4345F0DCFEE64FF08E
S214451030000804F11909F4E72DE9F04716469946E4
S2144510408A680B69DDF820809342B8BF1346336043
S21445105091F8432007460C460AB1013333602368AE
S214451060990642BF336802333360256815F0060596
S21445107006D104F1190AE36832689B1AAB4226DCAE
S21445108094F84320131E226818BF012392062BD4DA
S21445109004F1430249463846C04701301ED023680E
S2144510A0E568326803F00603042B08BFAD1AA3684B
S2144510B022690CBF25EAE57500259342C4BF9B1AF5
S2144510C0ED1800261A34B5421AD1002008E001234F
S2144510D0524649463846C047013003D14FF0FF30A7
S2144510E0BDE8F0870135C6E7E1185A1C302081F87F
S2144510F04300224494F8451082F843100233C7E76C
S2144511000123224649463846C0470130E6D00136D7
S214451110D9E700002DE9FF470C469146277E0C99F6
S214451120782F80469A4604F1430207D8622F0AD89C
S214451130002F00F0D880582F00F0A38004F1420617
S21445114084F842703AE0A7F16303152BF6D801A060
S21445115050F823F0AD114500C11145003D1145003D
S2144511603D1145003D1145003D114500C111450065
S2144511703D1145003D1145003D1145003D114500D9
S214451180CD124500F1114500AF1245003D11450011
S2144511903D114500EF1245003D114500F111450052
S2144511A03D1145003D114500B71245000B681A1D17
S2144511B01B680A6004F1420684F842300123A3E026
S2144511C0256808682E0600F104030AD505680B60F5
S2144511D0002D03DA2D236D4284F843305E480A23FA
S2144511E019E015F0400F05680B6018BF2DB2EFE704
S2144511F00B682568181D0860280601D51D6802E09D
S2144512006906FBD51D8854486F2F0CBF08230A2353
S214451210002184F843106668A660002EA2BF2168A8
S21445122021F0040121600DB9002E4DD01646B5FBC0
S214451230F3F103FB1157C75D06F8017D2F46BB4208
S2144512400D46F4D9082B0BD12368DF0708D523694B
S21445125061689942DEBF302306F8013C06F1FF3649
S214451260921B2261CDF800A04B4603AA2146404674
S214451270FFF7E2FE01304CD14FF0FF3004B0BDE839
S214451280F087354884F8457023680E681F0656F87B
S214451290045B0E6014D5D90744BF43F02003236092
S2144512A01DB9236823F0200323601023B0E7236885
S2144512B043F0200323607823284884F84530E3E745
S2144512C05E0648BFADB2E6E71646BBE70B6826683E
S2144512D060691D1D0D6035061B6801D5186002E066
S2144512E07106FBD51880002323611646BAE70B68BE
S2144512F01A1D0A601E68626800213046FEF7D8F956
S21445130008B1801B606063682361002384F843301E
S214451310A8E72369324649464046D0470130ABD018
S21445132023689B0713D4E068039B9842B8BF1846CA
S214451330A4E70123324649464046D04701309BD074
S2144513400135E36803995B1AAB42F2DCEBE700250F
S21445135004F11906F5E700BF589146006991460025
S2144513602DE9F04F87B0174603938B685A1EB2F5A2
S214451370AE7F83BF6FF4AE755B190293002386BFBD
S21445138040F25D138B6002930B688B46002543F451
S214451390F0634BF81C3BCDE9045580460C465E464B
S2144513A0AA46A9460195A26852B13B681B784E2BC2
S2144513B064D8402B3CD8A3F12B01C8B20E283AD9A5
S2144513C0B9F1000F03D0236823F4807323600AF134
S2144513D0FF3ABAF1010F00F213815E4500F205812E
S2144513E00125284607B0BDE8F08FA3F161020D2A16
S2144513F0E6D801A151F822F037154500C11345003E
S214451400C1134500C1134500971545006F154500A6
S214451410C1134500C113450045154500C113450098
S214451420C1134500C1134500C1134500FD144500D1
S214451430A3F14102DBE70E29C2D801A050F821F0FE
S214451440EF144500C1134500EF14450083154500CC
S214451450C11345009D144500D9144500D9144500CF
S214451460D9144500D9144500D9144500D91445006A
S214451470D9144500D9144500D91445006E2B09D812
S214451480602BB2D8542B77D0592B99D1072D97D1AD
S214451490082529E0742B6FD0792BF6E72168C80517
S2144514A01AD5029B21F08001216009F101091BB183
S2144514B0013B01320293A260A368013BA360236906
S2144514C0013323617B68013B002B7B6040F38480BE
S2144514D03B6801333B6066E71AEB050F7FF470AF58
S2144514E0226822F4C072226006F8013BE4E72268CF
S2144514F010067FF565AF22F08002F4E7BAF1000FDB
S2144515000ED1B9F1000F0ED1226802F4E061B1F5B3
S214451510E06F08D122F4F06222604FF0010AE3E75B
S214451520BAF1020F55D0012D02D0042D7FF448AFF5
S2144515300135EDB2D8E7BAF1010F7FF441AF4FF070
S214451540020AD1E77DB9B9F1000F7FF43CAF2268B6
S21445155002F4E061B1F5E06F7FF439AF22F4F06252
S21445156022600125C0E7032DE2D0052DDEE7022DDA
S2144515707FF426AF0325B7E7062D7FF421AF072571
S214451580B2E7226891057FF51BAF22F420722260F0
S214451590CDF80490A8E7226802F4A061B1F5806F03
S2144515A006D050057FF50CAFB9F1000F3FF40FAFED
S2144515B0910558BF019922F4F06258BFA9EB010185
S2144515C042F4C07258BFCDE9041622604FF00009B8
S2144515D08AE74FF0030A87E7D4F880313946404614
S2144515E0984700283FF4DFAEEAE6D4F87C3116F893
S2144515F0011D3A46404698472369013B2361ECE680
S2144516006B1E062B25D8022D36D85E457FF6E8AEEE
S214451610D4F87C3116F8011D3A464046984723696A
S214451620013B2361F1E70298D4F87C3110F8011D9F
S21445163002903A46404698472369013B23610AF1A2
S214451640FF3A5FFA8AFABAF1020FECD1033DEDB2E2
S214451650761B2368DA052FD55B0510D55E457FF6E4
S214451660BFAED4F87C3116F8011D3A464046984739
S2144516702369013B2361F1E7AA460296DFE716F8A0
S214451680011C2369652903F1FF3306F1FF35236104
S2144516900CD045290AD0D4F87C313A46404698477E
S2144516A0236916F8021C013BB51E2361D4F87C312C
S2144516B03A46404698472E46256815F0100559D1B6
S2144516C03570236803F4C063B3F5806F1CD1019B66
S2144516D04B45A3EB090224D100225946404600F06B
S2144516E083FED4F800C0039B1CF0020F1B68064619
S2144516F00F4621D003991A1D0A601B68C3E9006787
S214451700E3680133E3606CE6049B002BE4D005995F
S2144517100A232A460131404600F0E6FE049B059E14
S214451720C21A04F26F139E4228BF04F5B7761249D3
S214451730304600F029F8CFE71CF0040F03F1040EFD
S21445174003D00399C1F800E0D7E7039AC2F800E052
S214451750D3F8008002460B46FEF750FC28B10748F2
S21445176000F00EF8C8F80000CAE730463946FEF7DE
S214451770A3FCF7E7002534E67A914600648C4600DC
S214451780004870470000C07F0EB400B59AB01BAB4A
S214451790019005906FF0004109480691039109496B
S2144517A053F8042B04910068009301A902F0E4FD68
S2144517B0019B00221A701AB05DF804EB03B070471F
S2144517C0182340200802FFFF2DE9F0410F469046BA
S2144517D002F084FB04460D46B8F1000F11D0C7F35E
S2144517E00A53C3F16B03002B0BDD1B0503F17F5535
S2144517F0002405F5401522462B46FEF765F90446B6
S2144518000D4620462946BDE8F08100000000000050
S2144518102DE9F04FA1B09B4600231C939E4B179293
S2144518201F68824638460E46FDF73AFF4FF00008D9
S21445183004464FF000091B961B9B1A782B2A4CD062
S2144518403AD80D2A33D8082A33D8002A3DD0002363
S2144518500C931B9D2B78302B40F0A9806B7803F0BA
S214451860DF03582B66D10C9B01931CAB00938B4A28
S214451870CDF808B01DAB1BA9504601F01FFD10F072
S2144518800706044605D0062E29D1013500231B95AB
S2144518900C93179B002B40F08E850C9BD3B142468C
S2144518A009F100431046194621B0BDE8F08F202ABD
S2144518B0CDD101331B93BFE72D2AC8D101220C9207
S2144518C05A1C1B925B78002BC3D1179B1B96002B8B
S2144518D040F06F8542464B46E4E70022EFE71C9A08
S2144518E03AB135211EA802F0F0FB1C99504602F08D
S2144518F031F8013E042E06D8DFE806F00A03141731
S2144519000A00DDE91E892107C3D549F00049C0E72D
S214451910DDE91E831D9A23F4801302F2334243EA1F
S2144519200259F0E7DFF87891EDE76FF000494FF0A0
S214451930FF38E8E71B9B5A1C1B925B78302BF9D087
S214451940002BA6D0012307931B9B08930023CDE9C4
S21445195005339B460A221B980578A5F13003D9B274
S214451960092926D92246394602F01CFE002832D0DF
S21445197000202B465C4604900246652B01D0452B3D
S21445198013D11CB9079B03439FD000241B9E731C91
S2144519901B9373782B2B78D02D2B7BD00027A3F168
S2144519A03001092940F282801B9600259EE00023DF
S2144519B0C9E7BBF1080FD5BF0699059902FB013368
S2144519C002FB013300F10100D4BF069305930BF1EA
S2144519D0010B1B90BFE71B9B1A191B921B5DBBF1A6
S2144519E0000F36D004905C46A3F13002092A12D97E
S2144519F00122C2E71B9B5A1C1B925B780130302B99
S214451A00F8D0A3F13102082A00F2DA841B9A049032
S214451A10002008920446303B00F1010213D0049999
S214451A2011440491224605190A21954213D12218DC
S214451A30082A04F1010404441BDC06990A2202FB29
S214451A400133069300221B9B591C1B915B7810465D
S214451A50CAE75846D3E7082A04DC069F4F4306974D
S214451A600132E2E7571C102FDEBF059F4F4305970F
S214451A70F6E7102CDFBF05990A2202FB01330593D2
S214451A80E0E70023049301227CE70027B31C1B9361
S214451A90B37884E70127F9E7E0924600809146004F
S214451AA00000F07F1B9B591C1B915B78302BF9D0AF
S214451AB0A3F1310108293FF678AFA3F1300C1B9B03
S214451AC009934FF00A0E1B9B591C1B915B78A3F19B
S214451AD03005092D35D9099D491B082944F61F654A
S214451AE002DC6545A8BF654607B16D42002C4CD162
S214451AF0079901437FF4CDAE002A7FF4E6AE692B05
S214451B0026D023DC492B23D04E2B7FF4DEAE9C49D2
S214451B101BA801F00FFE00283FF4D7AE1B9B1B7891
S214451B20282B2CD197491EAA1BA801F017FE05287D
S214451B3025D11F9BDDF8788043F0FF4949F4E0093D
S214451B40A7E60EFB0C3CACF1300CBCE76E2BDCE795
S214451B508D491BA801F0EEFD00283FF4B6AE1B9B51
S214451B608A49013B1BA81B9301F0E4FD10B91B9B5A
S214451B7001331B93DFF824924FF0000889E684482A
S214451B8002F00AFD8046894683E6049B0698EB1AD2
S214451B90BBF1000F08BFA346102C07932646A8BFE7
S214451BA01026FDF717FF092C8046894613DD794B2D
S214451BB003EBC60353E91223FDF786FF80460598D7
S214451BC08946FDF707FF02460B4640464946FDF760
S214451BD0C5FD804689460F2C36DC079B002B3FF417
S214451BE058AE22DD162B09DC6A4C04EBC304D4E957
S214451BF0000142464B46FDF767FFC3E7079AC4F127
S214451C002503934220DB634DC4F10F0405EBC40165
S214451C1042464B46D1E90001FDF756FF079B1C1B84
S214451C2005EBC405D5E90023E5E7079B16330BDB33
S214451C30049B584A5D1B02EBC505D5E90023404683
S214451C404946FEF76BF89DE7079BA61B1E44002EEC
S214451C5071DD16F00F030AD04E4901EBC30142462B
S214451C604B46D1E90001FDF72FFF8046894636F001
S214451C700F0650D0B6F59A7F27DD4FF0000BCDF80E
S214451C8010B0CDF820B0CDF818B02223DFF80C916F
S214451C90CAF800304FF00008089B002B3FF4F9AD1A
S214451CA01C99504601F056FE0699504601F052FEE4
S214451CB00499504601F04EFE0899504601F04AFEFA
S214451CC05946504601F046FEE3E5002336114046A8
S214451CD049461F46012E21DC0BB1804689462E4BD0
S214451CE0A9F1547903EBC70742464B46D7E90001AD
S214451CF0FDF7EAFE294B0A460B4029498B428046AA
S214451D00BBD8A1F580118B4286BFDFF898904FF07F
S214451D10FF3802F15479002305937EE0F20707D594
S214451D201D4B03EBC703D3E90023FDF7CDFE012387
S214451D3001377610CEE7EED0764216F00F020AD07F
S214451D40144B03EBC20340464946D3E90023FDF74F
S214451D50E5FF804689463611DDD01F2E24DD4FF03F
S214451D60000BCDF810B0CDF820B0CDF818B0222332
S214451D704FF000084FF00009CAF800308CE700BF66
S214451D8053914600949146004B914600D4924600A6
S214451D90648C460020934600F89246000000F07F8B
S214451DA00000A07CFFFFEF7F16F0100318BF6A23E4
S214451DB0B34F0593404649460023F20704D5D7E975
S214451DC00023FDF781FE0123761007F10807F4D1BD
S214451DD00BB180468946059BBBB1C9F30A53C3F18F
S214451DE06B03002B494610DD1F2B40F32881342B0F
S214451DF0DEBF203B4FF0FF3202FA03F34FF00008F8
S214451E00CCBF4FF05C7903EA010900220023404627
S214451E104946FEF7C1F80028A1D1069B00930899CC
S214451E2023465A46504601F0EAFD089000283FF4FE
S214451E3024AF049B5D1B079B002BB4BF2B4600239A
S214451E400E93079B4FF0000B23EAE3731693CDF8EA
S214451E5010B0089B5046596801F048FD069000288A
S214451E603FF413AF089B1A69023203F10C01920046
S214451E700C3001F02DFD1EAB01931DAB0093424681
S214451E804B465046CDE90A8902F0A2F81C90002838
S214451E903FF4FBAE0121504601F03DFE049003465B
S214451EA000283FF4F2AE1D9D1E9A002DABBF0E9B3B
S214451EB0169B169C0E9EACBFEE185C1B059BED1A3A
S214451EC01544704B013D9D42C2F1360280F2C980F1
S214451ED05B1B1F2BA2EB03024FF0010700F3B680F6
S214451EE007FA03F30F930025B718059BBE42144423
S214451EF01C443346A8BF3B46A342A8BF2346002BF7
S214451F00C2BFFF1AE41AF61A0E9B002B17DD04997A
S214451F101A46504601F0A4FE049000283FF4B5AE9C
S214451F2001461C9A504601F0FFFD099000283FF4F3
S214451F30ACAE1C99504601F00DFD099B1C93002F35
S214451F4000F39380079B002B08DD169A06995046AA
S214451F5001F086FE069000283FF497AE002C08DD7B
S214451F6006992246504601F0C9FE069000283FF4E1
S214451F708CAE002E08DD04993246504601F0BEFE72
S214451F80049000283FF481AE069A1C99504601F00D
S214451F902FFF834600283FF478AE0024C368049993
S214451FA0C4600D9301F009FFA04271DA0D9B53EA18
S214451FB0080340F09780C9F31303002B40F0928046
S214451FC029F000431B0D1B05B3F1D66F40F28A80FE
S214451FD0DBF8143023B9DBF81030012B40F3828050
S214451FE059460122504601F089FE0499834601F080
S214451FF0E4FE002876DD0599234A4B46002900F085
S214452000928002EA0901B1F1D66F00F38C80B1F1F6
S2144520105C7F7FF7ACAE1D4A0023CDE914324046BF
S214452020DDE914234946FDF74FFD0B46034308BF3C
S21445203022238046894608BFCAF8003030E64FF06E
S214452040FF3202FA03F303EA0808DEE6C5F17F45E8
S21445205005F57F0505F57B45E23507FA05F50F9746
S21445206042E7012300250F933EE71C993A46504622
S21445207001F044FE1C9000287FF464AF05E600BFDF
S214452080A891460002FCFFFF0000F07F0000503993
S214452090CDF8249066D10D9AC9F313035AB39C4ADA
S2144520A093422CD1059B404603B39A4A4B461A4069
S2144520B0B2F1D46F4FF0FF311BD8120DC2F16B034E
S2144520C001FA03F398421AD1934B099A9A4202D1E0
S2144520D001303FF4DAAD8F4B099A1A4002F5801964
S2144520E04FF00008059B002B95D1D9E54FF0FF33FF
S2144520F0E8E70B46E6E753EA08033FF47CAFE5B16D
S214452100099B1D42EED00D9B059A40464946C3B1F4
S214452110FFF75AFB02460B46DDE90A01FDF71EFBB3
S21445212080468946DEE71340A3F580136FEA1359C8
S2144521306FEA09594FF0FF38D4E70F9B13EA080FAB
S214452140E0E7FFF741FB02460B46DDE90A01FDF7EE
S21445215003FB0022002380468946FDF71DFF002825
S214452160C0D004E60499584601F081FF00224FF09E
S214452170804306460F46FDF723FF002875D00D9B86
S214452180002B47D0654F0026644D099B23F000433E
S2144521901B0D1B050F930F9A614B9A4240F0C88062
S2144521A0DDE90A23CDE91423099BA3F1547940467A
S2144521B0494601F093FE02460B4630463946FDF742
S2144521C083FC42464B46FDF7C9FA0B465149554AEC
S2144521D01940914280465ED90B9B02F15472934258
S2144521E003D10A9B01333FF450ADDFF82C914FF0F5
S2144521F0FF381C99504601F0ADFB0699504601F054
S214452200A9FB0499504601F0A5FB5946504601F0F6
S214452210A1FB1EE6B8F1000F19D1099BC3F31303C2
S214452220E3B93E4B002230463946FDF7BFFEC8B9F6
S2144522303D4B002230463946FDF746FC04460D46E2
S21445224005F1004318941993DDE918679DE7B8F141
S214452250010F03D1099B002B3FF489AD334F002670
S214452260002491E70D9C304DEAE72F4B002230467F
S2144522703946FDF729FC0D9B04460D4633B901F159
S214452280004310901193DDE910677EE702460B4642
S214452290CDE91023F7E703F15479059B002BA8D128
S2144522A029F000430F9A1B0D1B059A42A1D12046E3
S2144522B02946FEF75DFAFDF7D9FB02460B46204652
S2144522C02946FDF749FA0D9AC9F3130343EA08036D
S2144522D0134304460D4666D009A3D3E90023FDF70C
S2144522E065FE00287FF4DCAC07A3D3E9002320462F
S2144522F02946FDF779FE00283FF47BAFD0E400BFC2
S2144523009535A094FFFFDF3F35E5AF350000E03F4C
S214452310FFFF0F000000F07FFFFFEF7F0000F03F5C
S2144523200000E07FFFFF9F7C0000E03F0000F0BF1D
S214452330059B13B30F9BB3F1D46F1ED826A3D3E9E1
S214452340002320462946FDF73BFE90B12946204608
S214452350FDF792FE012838BF0120FDF73BFB0D9B9C
S21445236004460D46D3B901F1004312901393DDE9B7
S21445237012670F9A07F1D6639F1ADDE90A0101F045
S214452380ADFD02460B4630463946FDF79DFBDDE979
S2144523900A23FDF7E3F9804689467EE702460B4663
S2144523A0CDE91223E3E70EA3D3E90023FDF7FEFDAF
S2144523B0A1E700230C93179A1B9B1360FFF76DBA92
S2144523C0652B3FF45EAB452B3FF45BAB0122FFF735
S2144523D08FBB00BFAFF300800000C0FFFFFFDF41AB
S2144523E09535A094FFFFCF3F014BFFF711BA00BFCD
S2144523F0802340202DE9F0473A4E86468C46604677
S2144524001CF8014BA55D15F00805F8D12D2C33D1E8
S2144524109CF800404FF0010800F1020C002B5CD000
S214452420102B0CD1302C0AD19CF8000000F0DF00B0
S21445243058284DD19CF8014010230CF1020C08F1A8
S2144524400047013F0026B7FBF3F9304603FB197AF0
S214452450A4F13005092D18D82C46A34224DD751C59
S21445246007D081451DD301D1A2451ADB00FB0340A9
S21445247001261CF8014BEBE72B2C08BF9CF80040C7
S214452480A84608BF00F1020CC8E7A4F14105192D7E
S21445249001D8373CE1E7A4F16105192D04D8573C2E
S2144524A0DBE74FF0FF36E4E7731C06D12223CEF870
S2144524B00030384642B9BDE8F087B8F1000F00D085
S2144524C04042002AF7D00EB10CF1FF311160F2E719
S2144524D03024002BB3D10823B1E7302CA4D00A23EF
S2144524E0ADE700BFD1914600FFF784BF00B59BB06E
S2144524F0019105916FF000410691039105490491BC
S21445250001A901F039FF019B00221A701BB05DF846
S21445251004FB00BF0802FFFF13460A460146024871
S2144525200068FFF7E3BF00BF182340202DE9F74FAB
S21445253003690C69A3420746C0F28180013C01F15C
S214452540140800F1140505EB8403019358F824306C
S21445255055F8242001339A424FEA840B08EB840948
S214452560B2FBF3F631D34FF0000E4046AC46F2468A
S21445257050F8042B93B206FB03E34FEA134E9BB287
S214452580AAEB0303120CDCF800A006FB02E213FAE2
S2144525908AF34FEA124E1FFA82FADCF80020CAEB9D
S2144525A0124202EB23429BB243EA024381454CF872
S2144525B0043B4FEA224ADBD255F80B302BB9019B38
S2144525C0043B9D421A462ED33C61384601F0F5FB46
S2144525D0002824DB013628464FF0000C58F8042B1B
S2144525E0D0F800E093B2ACEB0303120C13FA8EF36B
S2144525F0C2EB1E4202EB23429BB243EA0243C1456D
S21445260040F8043B4FEA224CE8D255F8242005EB27
S214452610840322B9043B9D421A460AD33C613046A0
S21445262003B0BDE8F08F1268043B002ACCD1013CCC
S214452630C7E71268043B002AF0D1013CEBE70020CF
S214452640EEE70000000000002DE9F04F446A99B01F
S21445265016461F46CDE90467DDF8948005463CB925
S214452660102001F01BF9C0E9014468620460C460AB
S2144526706B6A196851B15A684A60012393408B606A
S214452680284601F067F96B6A00221A603B1EB9BFFF
S21445269023F0004305930023C8F80030DDF8149076
S2144526A0A74BBCBF0122C8F8002033EA090319D15D
S2144526B0249A42F20F731360C9F31303334300F0B1
S2144526C06D85269B53B99F4B23E09F4B0393083359
S2144526D0269A1360039819B0BDE8F08F994B03937B
S2144526E00333F5E7DDE90434CDE90C34DDE90C01C7
S2144526F000220023FDF750FC804660B1249A012352
S2144527001360269B002B00F04685904B269A136057
S214452710013B0393DEE716AB019317AB00932846C0
S214452720DDE90C2301F054FCC9F30A548346002C1A
S2144527307ED00D9BCDF84C80C3F31303DDE90C0129
S21445274043F07F5141F44011A4F2FF34804B002200
S214452750FDF702F874A3D3E90023FDF7B5F974A392
S214452760D3E90023FCF7FAFF064620460F46FDF759
S21445277041F971A3D3E90023FDF7A6F902460B46B6
S21445278030463946FCF7EAFF06460F46FDF74CFC51
S21445279000228246002330463946FDF707FC48B1FD
S2144527A05046FDF727F932463B46FDF7F5FB08B997
S2144527B00AF1FF3ABAF1160F57D8664B03EBCA0330
S2144527C0D3E90023DDE90C01FDF7F0FB00284ED0E8
S2144527D00AF1FF3A00230F93169B1C1B631E0993B1
S2144527E045BFC4F101030693002300234CBF09935C
S2144527F00693BAF1000F3CDB099BCDF838A053444D
S214452800099300230A93229B092B00F2B580052BDA
S214452810C4BF043B2293229BA3F10203CCBF0024F2
S2144528200124032B00F2B480DFE803F02D987AA448
S214452830DDE916431C4404F23243202BC3BFC3F1E3
